:020000040000FA
:040000006FD00400B9
:101000006F00907E00000000000000009020002093
:10101000AA220020A9BDF9F56C23002000000000E1
:10102000000000006C230020902000200000000041
:101030000000000090200020000000009020002010
:101040000000000090200020902000209020002030
:101050009020002090200020582F00209424002071
:101060000000000090200020902000201E2400207E
:1010700090200020D22300209020002090200020EB
:101080009020002090200020902000209020002020
:101090009020002001A04111B7170040985F3AC688
:1010A000945F3247E39CE6FE3245410182800111A4
:1010B00013078008F337078093F787083EC20100C3
:1010C0000100B7170040930570052380B70413068D
:1010D00080FA2380C7040100010083C6B70493F699
:1010E000F60DA385D704238007049246F3A6068055
:1010F0000100010093760502D5CEF336078093F602
:10110000860836C4010001002380B7042380C70489
:1011100001000100B70614007D89558D88C70100C4
:1011200001000100010023800704A246F3A6068007
:101130000100010073370780137787083AC6010062
:1011400001002380B7042380C704010001000100CF
:1011500001003727004093061005A303D7802380A2
:101160000704B247F3A70780010001009307800836
:10117000F3B7078093F787083ECE01000100B71749
:101180000040130770052380E704130780FA2380CB
:10119000E7040100010003C7B70413670708A3852C
:1011A000E70423800704F247F3A70780010001004A
:1011B0000561828093760504BDC6F336078093F6F9
:1011C000860836C8010001002380B7042380C704C5
:1011D00001000100B7061400938606047D89558D31
:1011E00088C7010001000100010023800704C246F6
:1011F000F3A6068001000100733707801377870884
:101200003ACA010001002380B7042380C70401000B
:1012100001003727004093062005A303D7802380D1
:101220000704D24781B773370780137787083ACC12
:10123000010001002380B7042380C70401000100DE
:1012400098471367070C98C723800704E24719BF24
:101250000111814601468145114506CE97000000E7
:10126000E780605893078008F3B7078093F78708F3
:101270003EC601000100B717004013077005238028
:10128000E704130780FA2380E7040100010003C785
:101290006704136717002383E70423800704B2471A
:1012A000F3A7078001000100F2400561828041112F
:1012B000814601468145114597000000E780A05214
:1012C00013078008F337078093F787083EC40100AF
:1012D0000100B7170040130670052380C70493066A
:1012E00080FA2380D70401000100FD552396B70240
:1012F00023800704A245F3A5058001000100733790
:101300000780137787083AC6010001002380C704CD
:101310002380D7040100010003C767041367170087
:101320002383E70423800704B247F3A70780010063
:10133000010001A0B1473305F50201007D1575FDDF
:101340008280411122C426C206C6AA8401446317C2
:101350009400B24022449244410182800504130566
:10136000803E420497000000E78000FD4180C5B741
:101370009305000273A04580824573901534924016
:101380002242B2424243D2436244F2440255925551
:101390002256B2564257D2576258F25806499649D9
:1013A000264AB64A464BD64B664CF64C065D965DD1
:1013B000265EB65E465FD65F09617300203041113C
:1013C000B7170040985F3AC6945F3247E39CE6FE49
:1013D000324541018280B71700401307000323887C
:1013E000E702854717170000232EF74673002030C9
:1013F000411122C42D6426C24AC006C637190040D6
:101400001304A4AAB704002023208900976000E0F9
:10141000E78040359C408297976000E0E780803409
:10142000E5B737370040834747009146BD8B639E41
:10143000D702B73600401306F00F973500009385AA
:10144000651F9737000083D7E72E03C7A6001377E1
:10145000F70F1DE3B7E70400BC4F09468945171590
:1014600000000345A5F7829731A099466394D70001
:10147000834757007300203003C786001377F70FA8
:10148000E365F6FC13851700AE97173800002313A9
:10149000A82A2380E70075B7B787004003C7670015
:1014A000098B6309071003C77700930600031377BE
:1014B0000703630DD70817380000034878771736FD
:1014C00000001306E6730547B30606012380E60015
:1014D00083C577001737000013078774429793F589
:1014E000F50F2300B70003C58700973500009385EB
:1014F0002572C2951375F50F2380A50003470700D9
:1015000089451377F703630CB70C63E7E50A6306B5
:10151000071A8545630CB7129737000083C75771C8
:101520003307F600034707001377F70F19CB85073A
:1015300093F7F70F3D476363F71A17370000A309C6
:10154000F76EB787004009472383E700B78700405D
:1015500083C77700E207E18763DE0704973700005F
:1015600083C7176D17370000130787693E978546B5
:101570002300D700173700001307876A3E979306AA
:1015800000032300D70017370000130767683E9752
:10159000A14685072300D70093F7F70F3D47636403
:1015A000F71417370000A305F768B787004009470D
:1015B0002383E70073002030930610026300D70EE8
:1015C000930620026305D70693060002E316D7F4BC
:1015D00003C727021377C70F13672700D5A803C7D0
:1015E00067001377070465CB03C7A702173800000D
:1015F00013088842173500001305C539134707083B
:101600002385E70203C7A7021377370F1367870005
:101610002385E702814713070004B305F5008C41D9
:10162000B306F80091078CC2E399E7FEF5B503C74E
:10163000A702134707042385E70203C7A70213770E
:10164000C70F136727002385E702F9B503C76700B3
:101650001377070449C303C767021738000013084C
:10166000682F173500001305A526134707082383A5
:10167000E70203C767021377370F136787002383D7
:10168000E702814713070004B305F5008C41B30658
:10169000F80091078CC2E399E7FEBDBD03C767025E
:1016A000134707042383E70203C767021377C70FB3
:1016B000136727002383E70285B503C76700137705
:1016C000070411CB03C727021377370F136787006F
:1016D0002381E70291B5238006003DBD97370000C6
:1016E000A3880754B9BD97370000A383075475BD7D
:1016F0002303048015472303E48001002302A48010
:10170000828083076480E3CE07FE23030480828007
:1017100083076480E3CE07FE03454480828083070D
:101720006480E3CE07FE2302A4808280411126C498
:101730004AC24EC006C61377F50BAD47AA892E895B
:101740009544630CF700194597000000E78080FA84
:1017500097000000E78020FB8D444E859700000035
:10176000E78040F9FD59FD1463983401B240A2446A
:101770001249824941018280135509011375F50F01
:1017800097000000E780E0F92209F1BF011126CCA3
:1017900006CEB704080097000000E780C0F61545A4
:1017A00097000000E78000F597000000E78080F6D2
:1017B00097000000E78000F62AC697000000E78047
:1017C00080F432459377150089EB13651500137586
:1017D000F50FF240E24405618280FD14E9F0014515
:1017E000CDBF397126DC4ADA4ED852D656D45AD2F9
:1017F0005ED006DE62CE66CCB7E700E07D5783AAF6
:10180000070022C603AA470023A0E71823A2E7186F
:10181000B7170040130770052380E704130780FA09
:101820002380E70483C74704930B75FFB684E20760
:1018300093FBFB0F8546AA892E8B32893724004003
:10184000E187015763FA76016308D50089461307DB
:1018500000026313D5000157D98F93F7F70FB71C18
:1018600000402382FC0411472303E4801305F00F9A
:1018700097000000E78000E8094C97000000E7802F
:1018800080E863657C15B7050700DA9537870700A0
:10189000795563FEE504B3879500636AF704370B57
:1018A0000800A94733EB65016395F90881E8814495
:1018B00097000000E78020E5268515A8DA85094510
:1018C00097000000E780C0E605090345F9FFFD1415
:1018D000050B97000000E780C0E481C49377FB0FFD
:1018E000E5F797000000E780A0EA69F17D55B7179A
:1018F0000040130770052380E704130780FA238054
:10190000E70403C74704418B2382E704F250B7E79B
:1019100000E023A0571123A24711E2543244525948
:10192000C259325AA25A125B825B724CE24C21615C
:101930008280A547639BF90685691309F00FB306FA
:101940009900B3742B01B6941349F9FFB37499004D
:10195000856B33796901416B9387F9FFB3F72701F1
:1019600099E363FC340193D94900C147E3E637FFAB
:101970003DBF0569C1697D19D9B71305800D63881D
:101980006901130500026384790113051008CA85F3
:1019900097000000E780C0D997000000E78040DF93
:1019A00031D54E99B38434416DBFDA852D4597000A
:1019B0000000E780E0D7CA94E30B99EE0509970091
:1019C0000000E78020D5A30FA9FEFDB79387F9FF9C
:1019D00093F7F70F636DFC0C83C71C0413073008E3
:1019E0006315F706370708006361EB06B3079B0032
:1019F000B706100063FBD704334BEB0089476399AC
:101A0000F9068980D549E38404EADA850945970017
:101A10000000E780E0D111090327C9FF9147232087
:101A2000E48003076480E34E07FE23033481FD173F
:101A3000EDFBFD14110B81C49377FB0FE9FF9700B9
:101A40000000E780E0D461F155B5B717004003C747
:101A50005704B70708001377070219E3B787070091
:101A60007955E376FBE833079B00E3F9E7F841B5E6
:101A70008547E380F9F0DA852D4597000000E7807F
:101A800020CB9389F4FFE38404E297000000E78011
:101A900060C893F7390091EB83260480032709007F
:101AA00093074900E396E6E03E89CE84D9BFB54767
:101AB0006399F9001305900B97000000E78080C33D
:101AC000FDB3B1471305B00AE388F9FE9947639760
:101AD000F904B7050800B365BB002D459700000069
:101AE000E78000C581448D4BA14997000000E78045
:101AF00060C263967401832704802320F900850463
:101B0000E39534FF8327048013172B0163550700E7
:101B10002312F90069BB2322F90051BB9D47639F43
:101B2000F90281451305B00497000000E78040C02A
:101B3000BD442320090023220900FD59970000001D
:101B4000E78040BD93F77400CA9703C70700FD14F0
:101B5000398D2380A700E39334FF91BBA14763979E
:101B6000F90697000000E780A0C28144630D0B00D6
:101B70008D479304C0036308FB00930400056304CE
:101B80008B01930440041375C507E30295D21945F0
:101B900097000000E78000B697000000E780A0B63D
:101BA000054597000000E780E0B426859700000017
:101BB000E78020B7094597000000E78080B69700CE
:101BC0000000E780E0BCE31405CE0DB39147639FAE
:101BD000F9001305600697000000E780A0B19700A8
:101BE0000000E78040B213059009F9B5E38109CC04
:101BF000F1547DB9BD660147173600001306C620B3
:101C0000938606A685458347060093F7F70F91C391
:101C100082800507E3F9E6FE973700002386B71EAA
:101C2000DDB77D166206618693178601E18763D46E
:101C3000070001458280931726003307F500AE9711
:101C400018439C4363E7E7007D16E37FF7FC7D556F
:101C5000828005458280FD15E205E18513978501A7
:101C6000618793F7F50F63480700FD15139725006B
:101C70002A97584365D713851700620561858280CE
:101C80003308B5021C4283A80600B335B502C297DB
:101C900033B50701AE98469585486367B5006394F0
:101CA000A50063E3070181480C43C6950CC388C2B5
:101CB0001CC2828081471397870161876343B70005
:101CC0008280139727002A97232007008507E5B70E
:101CD0008147014793968701E18663C5B6001335B6
:101CE0001700828093962700AA9694428507558F05
:101CF000D5B793D755408A07AA979C430545331516
:101D0000B5007D8D828017F3FFDFE702833D2A84D3
:101D100097000000E78060F405C5931725003E9406
:101D20000327C4FF814711EB7D1516053E9542053B
:101D3000418517F3FFDF6700033D05838507E5B79E
:101D40000145C5BF81471397870161876343C7007A
:101D5000828013972700B386E50094422A9785076F
:101D600014C3D5B77D1662066186014793178601B5
:101D7000E18763D50700133517008280931726008B
:101D8000B306F500AE9794429C437D16B58F5D8FE8
:101D9000F1BF8A05AA9501476363B500828083A6D7
:101DA000C5FFF11593D71600D98F9CC11397F60183
:101DB000E5B72A830148014701456343D700828084
:101DC000B387050183A80700B30706019C43C697A4
:101DD000AA976384F80033B517010507B308030118
:101DE000620723A0F80061871108C1BF2A83014759
:101DF0008147014563C3D70082803388E50083288B
:101E00000800330EE600032E0E003388A840330886
:101E1000C8416384080133B508018507B308E300AE
:101E2000E20723A00801E1871107E9B717F3FFDFF5
:101E3000E702232B0111B286B2842E86AA850A8579
:101E400097000000E780C0FA2A84A6850A859700DB
:101E50000000E78020E833348000060413351500C5
:101E6000018D056117F3FFDF6700E32917F3FFDF3B
:101E7000E702A3244111AA89AE8A328BB68402C23A
:101E800002C402C60144131C8401135C8C416349E3
:101E90009C02939B1400FD1B0549138CF4FFF15C1D
:101EA00033048901620461846340740792478E049D
:101EB000CE9423AEF4FE410117F3FFDF67006323E6
:101EC00013192400B30B2B01014A93172A00D6974C
:101ED00083A50B0088437800340050009700000071
:101EE000E78040DA050A93178A01E187F11BE35E78
:101EF000FCFC92474E9905042320F900A2473EC2FC
:101F0000B24702C63EC441B7131A8901135A8A4127
:101F1000131D240093178A01E18763CF970092472E
:101F20000A044E941CC0A24705091379F90F3EC25A
:101F3000B24702C63EC4ADB7B3079A0313152A00D1
:101F400056950841780034005000050AEA97DA9760
:101F50008C4397000000E780E0D26DBF197106C284
:101F600012C416C61AC81ECA22CC26CE2AD02ED219
:101F700032D436D63AD83EDA42DC46DECAC0CEC2C9
:101F8000D2C4D6C6DAC8DECAE2CCE6CEEAD0EED2F9
:101F9000F2D4F6D6FAD8FEDA971500009385058CB0
:101FA0008841E700050092402242B2424243D243B8
:101FB0006244F244025592552256B2564257D257C5
:101FC0006258F25806499649264AB64A464BD64BBD
:101FD000664CF64C065D965D265EB65E465FD65F45
:101FE0000961730020300000972100209381810156
:101FF000175100201301018117F5FFFF1305C500DC
:102000009705002093850500171600201306C6FDCE
:1020100063FAC5008322050023A055001105910530
:10202000E3EAC5FE17050200130585F497150020A5
:102030009385C5FB171600201306C66563FAC50015
:102040008322050023A0550011059105E3EAC5FE92
:1020500017150020130505649745002093858526F4
:102060006377B500232005001105E36DB5FEFD4241
:10207000739002BC8D4273904280B722000093821D
:10208000828873900230970200209382A2F793E235
:102090003200739052309752000093828286739080
:1020A00012346FB0F47573002030397101436EC67D
:1020B00019A0397141536AC866CA62CC5ECE19A0B4
:1020C000397101535AD056D252D44ED64AD826DA54
:1020D00022DC06DE33016140828241114AC026C201
:1020E00022C406C68282B24D4101024D924C224C5E
:1020F000B24B4101024B924A224AB2494101024984
:1021000092442244B240410182803D432A87637356
:10211000C3029377F700BDEFADE5937606FF3D8AE6
:10212000BA960CC34CC30CC74CC74107E36BD7FE30
:1021300011E28280B306C3408A0697020000969699
:102140006780A6002307B700A306B7002306B700E1
:10215000A305B7002305B700A304B7002304B70005
:10216000A303B7002303B700A302B7002302B700FD
:10217000A301B7002301B700A300B7002300B700F5
:10218000828093F5F50F93968500D58D9396050182
:10219000D58D61B7939627009702000096968682A8
:1021A000E78086FA9680C1171D8F3E96E374C3F8C8
:1021B000A5B73367B500FD530D8B79E7B7877F7FF0
:1021C0009387F7F710419441B372F6003363F6003A
:1021D000BE92B3E262006397720C6318D606504158
:1021E000D441B372F6003363F600BE92B3E26200EC
:1021F0006398720A631BD60410459445B372F600C7
:102200003363F600BE92B3E262006391720A631E0A
:10221000D6025045D445B372F6003363F600BE9241
:10222000B3E26200639A72086311D60210499449BE
:10223000B372F6003363F600BE92B3E262006393BA
:1022400072085105D105E30FD6F6131706019397CF
:102250000601631CF7001357060193D706013305E7
:10226000F7409375F50F91E982804183C18333056F
:10227000F7409375F50F91E182801377F70F93F78D
:10228000F70F3305F74082800346050083C605003B
:10229000050585056313D60065FA3305D6408280AF
:1022A00011059105E312D6FE014582802105A105A5
:1022B000E31CD6FC014582803105B105E316D6FC4E
:1022C000014582804105C105E310D6FC01458280AD
:1022D000B717004003C777051377E70FA38BE70411
:1022E000130700F8A38DE7043D47238CE704130789
:1022F0005003A38CE70403C7A7051377D70F238DDB
:10230000E7048280B717004003C7E7020D89411137
:102310001377C70F498F93068008F3B6068093F6AC
:10232000860836C601000100930670052380D70495
:10233000930680FA2380D704010001002387E70277
:1023400023800704B247F3A7078001000100410181
:10235000828041112A83014E930E407E130F001993
:10236000930F400663E56E129308001913034006AD
:10237000B3781503854E0D4FA14F337365020D8958
:102380001335150063EFBE121308F6FF79467298F5
:102390004208135808013307C70213D61700BE07B7
:1023A00032976146B3F6C60213068070B386C60242
:1023B0003697A166F58F42075D8FB716004083C739
:1023C000F60293F70708A303F1000346710083C7E1
:1023D000F60293F70708E394C7FE83477100B71628
:1023E000004093F7F70F6388071293078008F3B74D
:1023F000078093F787083EC401000100B71700402B
:10240000930670052380D704930680FA2380D704AF
:102410000100010023AA070383C6170393E60608F9
:10242000A388D70223800704A247F3A707800100EF
:1024300001001166B71700407D16D45BC85F938515
:102440004703A98EF18EF5FA93068008F3B606804D
:1024500093F6860836C601000100930670052380B6
:10246000D704930680FA2380D7040100010098C1A5
:1024700003C7170313670704A388E7022380070431
:10248000B247F3A7078001000100410182807D135C
:102490003368E3039308E016630E08003368F30320
:1024A0009308D016630808009378330093B8180097
:1024B0009388D81633081E01131E0801135E0E01FF
:1024C00055B56393E5030548638608000148630337
:1024D00003002A8871087298FD15131E0801C205B1
:1024E000135E0E01C18179BD13F8150063F4BF00BE
:1024F0007908D5B713381800E5BF83C7F60293F7FC
:102500000708A303F1000346710083C7F60293F79F
:102510000708E394C7FE8347710093F7F70FF1DFD5
:10252000E9B531714AD966CB06DF22DD26DB4ED70D
:1025300052D556D35AD15ECF62CD6AC96EC7AA8C26
:1025400002D897100000E78020B12A8993078008FD
:10255000F3B7078093F787083EDA01000100B71749
:102560000040130770052380E704130780FA2380D7
:10257000E7040100010003C7F7021377770FA38771
:10258000E70203C7F70213678700A387E7022380E8
:102590000704D257F3A70780010001000545970003
:1025A0000000E78060D6130780C13347E902116A53
:1025B00093070AE893065002BD69930BA004814A71
:1025C000014B13048008930470057D1AB347F90288
:1025D0003307D7023EC0FD873ECC938709A69309F7
:1025E000803E3347F7023AC27D873AC43347390306
:1025F0008549B399990193D93940B306D702B30BF2
:102600007703B3C6F602B3CBFB0236C6FD8636C8E7
:1026100093D6FB4136CEB7460F0093860624334946
:10262000D9028566938606FAB3969601B389E902C4
:10263000130760553309D90293060010B389E902E4
:102640003349D902B3C9F9029316390036CA37198A
:102650000040FD8636D0930D090493D7F9413ED250
:10266000F336048093F6860836DC010001009307F8
:1026700070052380FD00930680FA2380DD000100B1
:1026800001008346390593F6860FA309D9048346D2
:10269000390593E61600A309D90423800D00E256FC
:1026A000F3A6068001000100130C80FA116DF336C9
:1026B000048093F6860836DE01000100930770055A
:1026C0002380FD0023808D01010001008346390530
:1026D000216693E60602A309D90483560905B3E6E9
:1026E000A6012318D90483560905D18E2318D904CD
:1026F00023800D00F256F3A60680010001008346F8
:10270000390593F606026381061A03463905218AC4
:102710006DDE081897100000E7800098733604807B
:1027200013768608B2C20100010023809D00238039
:102730008D0101000100B717004003C6370513766D
:10274000F60DA389C70403C6370513660602A389DD
:10275000C704835609052166B3E6A6012318D904E8
:1027600083560905D18E2318D90423800D0096467F
:10277000F3A60680010001008346390593F60602A0
:10278000638B061483463905A18AEDFE970000206D
:10279000E7806090AA8636D497000020E780A08F5B
:1027A000A256E30AD5FE835609054255B3E6A601B3
:1027B0002318D90497100000E780C08F834639059D
:1027C000A18AEDDE03560905834629058247337643
:1027D000CA00B306DA0293D5F641B296B388F64042
:1027E000E24733B8C6002E983308F840A247B3B684
:1027F00016013308D84063C70701631DF8009247EC
:1028000063FA1701C247634FF80E63950701B24799
:1028100063EAF80E894663E9660FF24693151800DD
:1028200013D3F8015E8613951800B365B30042D642
:1028300046D497C00100E78080DA3258050B137B3D
:10284000FB0F63470001631A0838A25863870838F2
:1028500013081500B336A800B69513D6F5013298C3
:10286000B336C800AE9613581800FE06B3E606014C
:102870007336048013768608B2C6010001002380F7
:102880009D0023808D01010001000356C902B2960C
:10289000C206C1822316D90223800D00B646F3A6D4
:1028A00006800100010021B5F336048093F6860806
:1028B000B6C00100010023809D0023808D0101002E
:1028C00001008346390593E60602A309D904238053
:1028D0000D0086460DB5F336048093F68608B6C41F
:1028E0000100010023809D0023808D010100010073
:1028F0008346390593E60602A309D90423800D0017
:10290000A646BDB5E30B0BF0F336048093F68608BC
:10291000B6C801000100930680FA23809D00238041
:10292000DD00010001008346390593F5FC0F93F6A5
:10293000860FA309D90483463905CD8EA309D9048E
:1029400023800D00C646F3A6068001000100130592
:1029500080FA03463905930639051D8A631C9629BA
:102960007336048013768608B2CC0100010013068A
:1029700080FA23809D002380CD000100010003C662
:1029800006001376F60D2380C60003C60600136604
:1029900006022380C600835609051166D18E2318CE
:1029A000D904835609052166D18E2318D9042380C2
:1029B0000D00E646F3A6068001000100130680FA2A
:1029C0008346390593F60602638006268346390559
:1029D000130C3905A18AFDDA081897000000E7807A
:1029E000A06BF336048093F68608B6D00100010090
:1029F000930680FA23809D002380DD000100010002
:102A000083460C00116693F6F60D2300DC00834626
:102A10000C0093E606022300DC0083560905D18EE4
:102A20002318D904835609052166D18E2318D904A9
:102A300023800D008656F3A60680010001001306D0
:102A400080FA8346390593F60602638A0620834698
:102A50003905A18AEDFE97F0FF1FE780C0632A8C3D
:102A600097F0FF1FE7802063E30C85FF835609057D
:102A700011664255D18E2318D90497000000E780D3
:102A800060638346390513063905A18AFDDAF336FA
:102A9000048093F68608B6D401000100930680FAFC
:102AA00023809D002380DD00010001008346060095
:102AB00093F6F60D2300D60023800D00A656F3A64C
:102AC0000680010001008356090503462905D24707
:102AD000B376DA003306CA021305800C9355F6412B
:102AE0003696330DF6408257333CD6002E9C333653
:102AF000A601330CFC40330CCC40330885039256BE
:102B00004E86B335A5033305A503C29597C00100D2
:102B1000E780E0AC63468001631E0C16630C0D1663
:102B2000130615003335A6002E959356F5013696FB
:102B3000B335D600AA959396F50105828585D18E89
:102B40006346B000639D051A638B061A0356C902DB
:102B500015823305D6003336C500B2956348B00000
:102B6000639105241306F00F637DA622894663F363
:102B7000561593078008F3B7078093F78708BED6EA
:102B80000100010037170040930770052300F70488
:102B9000930780FA2300F704010001008356C7025F
:102BA00089678117D58FC207C1832316F7022300D7
:102BB0000704B657F3A7078001000100FA506A54D2
:102BC000DA544A59BA592A5A9A5A0A5BFA4B6A4C49
:102BD000DA4C4A4DBA4D296182801308F5FF33352E
:102BE000A800FD152E951356F5013298B336C8008E
:102BF000AA9695B9F336048093F68608B6CA010002
:102C0000010023809D002380AD0001000100834668
:102C10003905CD8EA309D90423800D00D646F3A62D
:102C200006800100010035B3F336048093F6860870
:102C3000B6CE0100010023809D002380CD0001005D
:102C400001008346390593E60602A309D9042380CF
:102C50000D00F646F3A606800100010095B3F33699
:102C6000048093F68608B6D20100010023809D00FF
:102C70002380CD00010001008346390593E606025A
:102C8000A309D90423800D009656F3A606800100FF
:102C9000010045BB9306F5FF33B5A600FD152E9543
:102CA0009355F501AE96B3B5B600AA951396F50106
:102CB000858269B5F336048093F68608B6D801009C
:102CC0000100930680FA23809D002380DD0001002F
:102CD00001008356C9020566011693F6F60FD18EE0
:102CE000C206C1822316D90223800D00C656F3A660
:102CF000068001000100850A93FAFA0F95B233E6C7
:102D0000B60045C20356C9023305D0403338A0008F
:102D1000B305B040B385054115826345B000D1E1EC
:102D20006371A608894663F0560593078008F3B7D8
:102D3000078093F78708BEDA01000100B71700404B
:102D4000130770052380E704130780FA2380E70444
:102D50000100010003D7C7027D8B2396E702238081
:102D60000704D65781BDF336048093F68608B6DC97
:102D700001000100930680FA23809D002380DD007E
:102D8000010001008356C9020566011693F6F60F8D
:102D9000D18EC206C1822316D90223800D00E656C9
:102DA000B9B793078008F3B7078093F78708BEDEAB
:102DB0000100010037170040930770052300F70456
:102DC000930780FA2300F704010001000356C702AD
:102DD00093975600B297C207C1832316F7022300C8
:102DE0000704F657C1BB914763EEB70217D701003E
:102DF0001307471C8A05BA959C41BA978287B71773
:102E0000004003A7470B1345F5FF698F23AAE70A84
:102E100003A7070B698F23A8E70A03A7070A798D81
:102E200023A0A70A8280B717004083A6470B134749
:102E3000F5FFF98E23AAD70A83A6070B558D23A881
:102E4000A70A83A6070A758F23A0E70A8280B7170F
:102E5000004003A7470B498F23AAE70A03A7070BE4
:102E60001345F5FF45BFB717004083A6470B13472F
:102E7000F5FF758F23AAE70A03A7070A598D4DB7F7
:102E8000B717004003A7470B498FEDB7914763EE93
:102E9000B70217D70100130727138A05BA959C417B
:102EA000BA978287B717004003A7470D1345F5FF70
:102EB000698F23AAE70C03A7070D698F23A8E70CE6
:102EC00003A7070C798D23A0A70C8280B7170040B9
:102ED00083A6470D1347F5FFF98E23AAD70C83A6C7
:102EE000070D558D23A8A70C83A6070C758F23A06B
:102EF000E70C8280B717004003A7470D498F23AA2C
:102F0000E70C03A7070D1345F5FF45BFB7170040B2
:102F100083A6470D1347F5FF758F23AAE70C03A778
:102F2000070C598D4DB7B717004003A7470D498FC0
:102F3000EDB7797122D43714004026D24AD0035914
:102F400024028354040206D64209C2044ECE52CC57
:102F500056CA13590901C1802DE11379F9F793F489
:102F6000F49F4209C20413590901C18093078008E4
:102F7000F3B7078093F787083EC401000100930769
:102F800070052300F404930780FA2300F404010081
:102F90000100231124032310940223000404A247F8
:102FA000F3A7078001000100B25022549254025945
:102FB000F249624AD24A45618280B7F507008146EC
:102FC0003000B105194597000020E7808081A247B5
:102FD00013972701E34A07FC1369090893E40440A7
:102FE00093098008F3B7098093F787083EC0010072
:102FF0000100930A700523005405130A80FA230088
:10300000440501000100231124032310940223002E
:1030100004048247F3A7078001000100294597F0C7
:10302000FF1FE7802031F3B9098093F989084EC268
:1030300001000100230054052300440501000100A4
:103040008357040293E707202310F40223000404AB
:103050009247B9B7B7170040884742054181937737
:10306000050491EB9377F5013755E80113050580C9
:103070003345F50282809377050C130700046397AC
:10308000E7009377F50137459C1CCDB72165130503
:1030900005D0828037E700E01C435443A183E20659
:1030A000D58F1CC1FD572320F7182322F7188280E3
:1030B00013178500B7E700E023A0E710618123A282
:1030C000A7108280B7F700E08847CC47828081470D
:1030D00037370040A14663C4C7003285828003456C
:1030E000B740E38EA6FE3385F5000345050085074E
:1030F0002304A740CDB797070020938727EF9C4371
:10310000173700201307071C3E95636EE50017373D
:1031100000201307274F6368A70017070020232705
:10312000A7EC3E858280FD57EDBF8280411122C40D
:1031300006C62A8497000000E78000F22947B307FB
:10314000E502B2408D83B3D7870222449507B3D7F7
:10315000E70237370040C207C1832316F700410159
:103160008280411137150E0006C697000000E780E7
:1031700020FCB7370040130770F82381E7000D47A4
:10318000A381E70013070004A380E7000547238716
:10319000E700B24041018280373700408347270073
:1031A0001A0593F7F703C98F93F7F70F2301F70079
:1031B0008280B737004003C7170019C9D98DA38093
:1031C000B70003C70700136787002380E7008280EA
:1031D00093C5F5FFF98DA380B7008280AE872A875B
:1031E000B736004021463738004089E71703000012
:1031F0006700E3F383C8B600E30916FF05078348B9
:10320000F7FFFD17C20723041801C183F9BF41115D
:1032100022C406C62A8497000000E780E0E329471D
:10322000B307E502B2408D83B3D7870222449507E6
:10323000B3D7E70237370040C207C1832316F740F0
:1032400041018280716541111305052006C6970072
:103250000000E78000FCB7370040130770F82381B7
:10326000E7400D47A381E74013070004A380E74030
:1032700005472387E740B24041018280CC4141119C
:1032800006C6328503C6150083C5050022064D8E8D
:1032900042068D654186138875A2630C0611634B47
:1032A000C804138845A26300060D634AC8009385CD
:1032B00035A26301B6082390060029464DA0138865
:1032C00055A26305060D938565A2E316B6FE8D45EE
:1032D0001D4663E6E5081146198E63F3C7003E8676
:1032E000B7E704002390C600FC4797D501009385FB
:1032F000E5CF9DA0138895A263030611634E060DCA
:103300001388A5A263000613938505A5E315B6FAF5
:1033100099451D4663E5E504198E63F3C7003E86B3
:10332000B7E704002390C600FC479705002093856B
:1033300025D61DA09D451D4663E3E5022146198E55
:1033400063F3C7003E86B7E70400FC472390C6003E
:103350009705002093858534BA9582970146B2403F
:10336000328541018280AD451D46E3EAE5FE3146E6
:10337000198E63F3C7003E86B7E704002390C600AA
:10338000FC4797D501009385E5C8F9B7B1451D46BF
:10339000E3E7E5FC3546198E63F3C7003E86B7E7E1
:1033A00004002390C600FC4797D50100938585C78C
:1033B00065B78D451D46E3E4E5FA1146198E63F3C2
:1033C000C7003E86B7E704002390C600FC4797D5A8
:1033D0000100938565C249B78D451D46E3E1E5F8D7
:1033E0001146198E63F3C7003E86B7E704002390A9
:1033F000C600FC4797D50100938585C4B1BFA5459C
:103400001D46E3EEE5F42946198E63F3C7003E86B8
:10341000B7E704002390C600FC4797D501009385C9
:1034200065BE1DBFB5451D46E3EBE5F23946198E75
:1034300063F3C7003E86B7E704002390C600FC474D
:1034400097D50100938585B901BFB7E7040003A3B1
:103450000713970600209386A6C24146A545170587
:1034600000201305E5B802832D455DE703C505007F
:103470000947631FE50803A84500411106C6034735
:10348000180032850346080022074168518F9308CF
:1034900028FE6307170563E9E800051863030703BF
:1034A00023900600294591A8130648FE630AC70425
:1034B0001518E31707FF15463E87637BF60015478F
:1034C00001A8130600023E876374F600130700028A
:1034D000B7E704002390E600FC471316070111A884
:1034E0003E8691C30546B7E70400FC472390C6001B
:1034F0004206CC45418282970145B240410182801B
:10350000130600083E87E375F6FC13070008C9B7E9
:103510002390060005458280828041677917630405
:10352000E504411122C406C685472A84639FF5003D
:10353000B7E7040022852244B24003A3871397050E
:1035400000209385E52F4101028389476399F500A7
:10355000B7E7040083A7070B8545829771D9B2406E
:103560002244410182808280797126D252CCAE847D
:103570002A8A97D501009385A5AE17D501001305BA
:10358000A5B006D63AC622D44AD0368432894ECE69
:1035900097B00100E780E04FA28517D50100130521
:1035A000A5AF97B00100E780C04E294597B0010054
:1035B000E780005383C7840093F70702F9E383C9C8
:1035C00004008947054532476396F908D44083C70C
:1035D000160083C60600A207D58FC166138616FEA5
:1035E000638CC7028D16638FD7068D6693862690EF
:1035F00029456391D706B7E70400A286225403A3A6
:103600004714B250F2494A86A6850259925452850F
:10361000624A8547456102832D450DEF93070002FD
:10362000354563E98702B7E70400FC47C844130641
:103630000002CA8582978149970700209387072156
:103640009C43014581CB9C4391C74E852286CA8508
:1036500082970145B250225492540259F249624A6B
:10366000456182802D457DF79307700F3545E3E373
:1036700087FEB7E70400FC47C8442286CA858297C4
:1036800065BF2145C1BF411122C437E4040083272F
:10369000841326C2AA84416506C697050020938537
:1036A000251A7D1582978327C40A17050000130584
:1036B00005E78588829795C0032304132244B2400E
:1036C000924497060020938626AE4146C5451705CD
:1036D00000201305659C41010283B24022449244BC
:1036E00001454101828019C59707002023A0A71634
:1036F00001458280454582801147636AA70A97D6B3
:1037000001009386A6940A0536951841411106C614
:103710003697AE87B2850287130700026145639D25
:10372000E700B7E70400FC47130600021705002076
:10373000130545F782970145B24041018280054754
:103740006145E39BE7FEB7E70400FC470546170524
:103750000020130525F7F9BF1307700F6145E39D9E
:10376000E7FCB7E70400FC471306700F17050020BD
:10377000130585F5C1B7130700086145E39EE7FA15
:10378000B7E70400FC4713060008170500201305DF
:1037900025034DB715476145E390E7FAB7E7040005
:1037A000FC471546170500201305C50961B70945F3
:1037B0008280411126C2B7E4040083A7C41322C447
:1037C0004AC006C62E8497050020938565072A897E
:1037D0008297058905C5970700209387E78B83D7D4
:1037E000A70BA28503A3440D2310F4002244B2408A
:1037F00092444A850249014641010283B240224473
:103800009244024949454101828097070020238163
:1038100007049707002023AF0702B717004003A74C
:10382000070CB706C0FFFD16758F23A0E70C03A792
:10383000070DB7064000558F23A8E70C03A7070C18
:103840003D9B23A0E70C03A7070D1367070123A8DF
:10385000E70C8280B717004003A5470C83A7470CED
:10386000598113451500C18B058999E3136525001E
:103870009707002083C7C7FD6380A7029707002032
:103880002388A7FC11C9970700209387A7FC03A3EF
:1038900007006303030002838280114517F3FFFFD3
:1038A000670063C8011122CC06CE3714004026CA37
:1038B0004AC84EC652C483447405034AB4058349BA
:1038C00084050349940597F0FFFFE780A0A0834794
:1038D000A40593F4F40F137AFA0F93E71700230D5E
:1038E000F40493F9F90F1379F90FB717004003C7E0
:1038F000A705058B6DFF03D5C705A38D4705238C51
:103900003705A38C2705A38B9704F2406244D24469
:103910004249B249224A05618280411193970501CB
:1039200022C406C626C2C1872E8463DC0700B7E422
:103930000400FC54829719C1BC5482972165218DE3
:1039400015A893F7150013C515008DE793F725000B
:103950009DC797000000E78020F0B7E70400BC4F48
:103960001306000A894517050020034525EF8297B5
:1039700013452400B240224492444101828093972F
:10398000250163D80702B7E4040083A7C41E829709
:1039900097000000E780A0F0BC4C375607001306E4
:1039A0000630896517050020034545EB82970965B8
:1039B00079B7939715010145E3DE07FA17C50100B2
:1039C0001305857597B00100E7808024B7E70400F0
:1039D000BC4F13060064916517050020034505E8F8
:1039E00082971165A9BF1D71A2CC37E404005C5C0D
:1039F000485886CE494697C501009385656D8297E4
:103A000011E917C501001305E56D97B00100E780C6
:103A1000202001A0B7F600E0795798CAFD57DCCA0C
:103A20000567B7E700E023A0E7101306F00290C295
:103A300023A0E718010001003707002018471306EC
:103A4000000481459706002023A8E6E04157A38A99
:103A5000E7403C4408088297970700209387077D3A
:103A60003EC8856713870740938757D1231AE10023
:103A70002312F1021307B00F97F7FFFF9387C76474
:103A80002310E1023ED81547970700009387C7E14E
:103A9000B7F50700A30FE1003EDC054797070000DC
:103AA0009387E7DF81463000E10519452301E102F4
:103AB0003EDE97F0FF1FE780C0D218088147994685
:103AC00030003E960346060085070507A30BC70096
:103AD000E398D7FEC24791C70357410185676373D7
:103AE000F70001A0B7E7040083A7470A08088297F8
:103AF000AA8511C917C501001305056097B001001B
:103B0000E78020F901A0F6406644256182804111DA
:103B100026C2B7E4040083A7040806C622C417051A
:103B200000001305C5DF829717040020130404D397
:103B30002300A40097000000E780800297000000A7
:103B4000E780E0CC03450400224403A38405B2408F
:103B5000924413060032896541010283797106D6C9
:103B600022D413078008F337078093F787083EC2F3
:103B700001000100B7170040930570052380B704CA
:103B8000130680FA2380C7040100010083C6F702F0
:103B900093F6A60FA387D702238007049246F3A6C5
:103BA00006800100010073370780137787083AC445
:103BB000010001002380B7042380C7040100010035
:103BC00003C7F70213672700A387E70223800704D0
:103BD000A247F3A7078001000100054597E0FFFF1A
:103BE000E780807297000000E78060CB0147814644
:103BF0008147054685451305407E97E0FFFFE78036
:103C0000807537E404003C44680051468145829742
:103C1000B707C0A83EC8B787E803938707D03ECA56
:103C200097E7FF1F9387A7793EC67C586800829765
:103C3000B250225445618280411197D5010093858D
:103C4000E5AF17C501001305254406C697B001006E
:103C5000E78020E417D50100130505C797B00100E0
:103C6000E78020E3B2402945410117B30100670016
:103C700023E7411197D50100938585AD17C5010054
:103C80001305854006C697B00100E78080E017D590
:103C90000100130525C297B00100E78080DFB24024
:103CA0002945410117B30100670083E3411122C494
:103CB00006C6834705002A849DC797D501009385D2
:103CC000E5AE17C501001305253C97B00100E7805C
:103CD00040DC4C4017D50100130545D197B00100D9
:103CE000E78020DB3DA058410DEF97D5010093857B
:103CF000E5AB17C501001305253997B00100E78032
:103D000040D917D501001305E5CF97B00100E78032
:103D100040D82244B2402945410117B30100670051
:103D200023DCA1679386D7036313D70297D50100DD
:103D30009385C5A717C501001305053597B0010088
:103D4000E78020D517D501001305C5CC7DBFED0751
:103D500097D50100938585A517C501001305C532C8
:103D6000631BF70097B00100E780A0D217D50100D0
:103D7000130585CB59BF97B00100E78080D14C4037
:103D800017D50100130545CC91BF411197D501000E
:103D90009385459D17C501001305052F06C697B0ED
:103DA0000100E78000CFB2402945410117B301006F
:103DB000670003D3797122D426D24AD02E842A896F
:103DC0008145B2844800714606D697E0FFFFE78040
:103DD000003497F7FF1F9387275EDC4783D70700E0
:103DE000231421012313F10097500000E78040E5E0
:103DF0008547A305F1009307401F3EC6FD572305E5
:103E0000A100230AF10097500000E780A0F7268662
:103E1000A285480097500000E78060E5B250225428
:103E2000925402594561828097270020239307907E
:103E300097170020238C077EB7E70400BC47411189
:103E400006C641468145170500201305A52C82971B
:103E5000170700200347072E9307F00A6315F702A0
:103E60009307F0F88945170500201305A52C1707BF
:103E700000202301F72C97070020A38D072A9760C5
:103E80000000E780409E97600000E780A0C9814560
:103E9000370504009707002023AC0726970700206A
:103EA00023960726970700202383072697070020DD
:103EB0002392071E970700202390071C97070020D6
:103EC0002395072497070020239E0724973000009E
:103ED000E780402A014597600000E780C0A197D5A0
:103EE00001009385A58A17C501001305E51997B050
:103EF0000100E78000BA17D50100130525BB97B074
:103F00000100E78000B9B2402945410117B3010023
:103F1000670003BD4111814617F6FF1F13060647D0
:103F20008545170500200355E51406C697C0000017
:103F3000E780E02715C997D501009385E58517C56A
:103F400001001305651497B00100E78080B417D510
:103F500001001305A5A597B00100E78080B32945AE
:103F600097B00100E780C0B797D501009385C5825F
:103F700017C501001305451197B00100E78060B136
:103F800017D501001305C5A397B00100E78060B005
:103F9000294597B00100E780A0B497F7FF1F9387EA
:103FA000A741DC47054797C501009385E57E23902F
:103FB000E70017C501001305250D97B00100E78044
:103FC00040AD17D501001305E5A097B00100E780CB
:103FD00040ACB2402945410117B30100670043B02E
:103FE000411122C497C501009385857D2A8417C598
:103FF00001001305650906C697B00100E78060A9B6
:104000004C4017D501001305E59797B00100E780F4
:1040100040A8294597B00100E78080AC0347040021
:104020009307F00F631FF70297C501009385457949
:1040300017C501001305450597B00100E78060A58D
:104040004C4017D501001305E59497B00100E780B7
:1040500040A42244B2402945410117B30100670042
:1040600023A8B240224441018280411122C426C2C9
:104070002A84AE8417C501001305050197C5010008
:104080009385C56F06C697B00100E78080A017D55D
:104090000100130525A097B00100E780809F294506
:1040A00097B00100E780C0A397C501009385056D17
:1040B00097070020239087FC17C501001305C5FC56
:1040C000054497070020239597FA9707002023922D
:1040D00087FA97170020239E976497B00100E78026
:1040E000409B9715002083D5C56417D501001305A3
:1040F000E59A97B00100E780C099294597B0010083
:10410000E780009E971700202382875297F7FF1FB2
:104110009387872ADC4703D70700C167FD1763121F
:10412000F7022244B7E70400B240924403A3870594
:1041300017F5FF1F034505731306000A8545410166
:104140000283B2402244924441018280B1C14111B4
:1041500022C417C50100130525F32E8497C501005D
:104160009385056106C697B00100E7808092A2851D
:1041700017D501001305459197B00100E7806091C4
:104180002244B2402945410117B30100670043951D
:104190008280011122CC06CE26CA4AC84EC693F7A9
:1041A00015002E84B1CF97000000E780E0D693077A
:1041B00010F817070020230FF7F69707002083D782
:1041C00027EB17070020A307F7F6170500201305B4
:1041D00065F6A183914517070020230EF7F4970792
:1041E0000020A38A07F497500000E780C0671345BA
:1041F0001400F2406244D2444249B24905618280CF
:1042000093F705108DC7054597500000E780A06E15
:10421000171500200355E55197500000E780003A3C
:1042200097200000E780000B13450410D9B793F7DF
:104230002500E9CF17070020035747ED69C7AD6494
:10424000B71900409384A4AA23A0990097060020E0
:10425000938606EC944297D7010093872787170629
:1042600000200346C6EA814517050020130585EAAC
:1042700097700000E780600F23A0990097F7FF1F59
:104280002390A7042A8941C197C5010093858557CA
:1042900017C50100130545DF97A00100E780607F87
:1042A000CA8517C501001305E5F597A00100E78051
:1042B000407E294597B00100E78080829707002063
:1042C000239607E4930710F8170700202304F7E666
:1042D0009707002083D7C7D917070020A30CF7E45E
:1042E000A183170700202308F7E491458D471705A0
:1042F0000020130525E417070020A30EF7E29750CE
:104300000000E780405613452400E5B593F74500CB
:10431000D1C397C501009385E54E17C5010013056C
:10432000A5D697A00100E780C07617C50100130548
:1043300025EF97A00100E780C075294597A00100EF
:10434000E780007A930720F8170700202304F7DEA0
:104350009707002083D707D417070020A30CF7DCAA
:10436000A183170700202308F7DC854717070020E3
:10437000A303F7DC97500000E780C0A017050020DA
:10438000130545DB914597500000E780C04D13456C
:10439000440085B593F78500A9C797C501009385AB
:1043A000654617C50100130525CE97A00100E780DB
:1043B000406E17C501001305E5E797A00100E780EF
:1043C000406D294597A00100E78080719707002084
:1043D000239E07D297700000E780000913458400F0
:1043E00009BD93F70501D1C3854517050020035585
:1043F00065CA97600100E780C0BE97C5010093853C
:10440000654017C50100130525C897A00100E78086
:10441000406817C50100130525E397A00100E78058
:104420004067294597A00100E780806B930730F82B
:10443000170700202300F7D09707002083D787C5F0
:1044400017070020A308F7CE17050020130585CE17
:10445000A1838D4517070020230FF7CC975000004C
:10446000E78060401345040169B393F70502D1C7A3
:1044700097C501009385053917C501001305C5C00F
:1044800097A00100E780E06017C50100130505DE75
:1044900097A00100E780E05F294597A00100E78031
:1044A0002064930740F8170700202305F7C89707F3
:1044B000002083D767BC17070020A30DF7C6A18390
:1044C000170700202309F7C6854717070020A30414
:1044D000F7C697070020239107BA97500000E7809E
:1044E000608A170500201305E5C491459750000028
:1044F000E780603713450402EDB993F70504FDC367
:1045000097C501009385053017C501001305C5B790
:1045100097A00100E780E05717C50100130585D675
:1045200097A00100E780E056294597A00100E780A9
:10453000205B9707002083C7E7BF1307700A6386D5
:10454000E7061307800A638CE7081307600A639382
:10455000E704930760F817070020230DF7BC9707BF
:10456000002083D787BA17070020A305F7BCA183D3
:10457000170700202301F7BC854717070020A30079
:10458000F7BCB145170500201305C5BA97500000C8
:10459000E780602D97400000E780C07E134504044B
:1045A00097070020239307B6A9B1930770F8170760
:1045B00000202301F7B89707002083D707B5170716
:1045C0000020A309F7B6A183170700202305F7B63B
:1045D000854717070020A301F7B6994565B79307EC
:1045E00080F8F1B793F705080145E38407C097C544
:1045F00001009385252117C501001305E5A897A0A3
:104600000100E780004917C50100130525C997A0DF
:104610000100E7800048294597A00100E780404C51
:104620009307A0F8170700202306F7B0970700208C
:1046300083D747AF17070020A30EF7AEA183170754
:104640000020230AF7AE854717070020A305F7AE21
:1046500097070020239807AC97400000E7808072FE
:1046600017050020130505AD914597500000E78020
:10467000801F13450408B5BE011122CC37E40400A5
:104680005C5C06CE354697C501009385252517D578
:1046900001001305A5F3829711E917C50100130561
:1046A00065A497A00100E780A05601A097F7FF1F1F
:1046B0009387071C3EC4B7F507008567938707807B
:1046C000814617F6FF1F1306261AE10519453EC657
:1046D00097E0FF1FE780E0107C44194697F5FF1F25
:1046E00093858518170500201305059B82973400D4
:1046F00017F6FF1F1306461797C501009385856FB0
:1047000017C501001305857097700000E780E09AD7
:104710002A841DCD97C501009385C50D17C50100DD
:104720001305859697A00100E780A036A28517C5DE
:1047300001001305A51B97A00100E78080352945DE
:1047400097A00100E780C039F24062440561828091
:1047500097E00000E780E00017C501001305051091
:1047600097600000E780208F97A00000E780205529
:1047700097600100E780A0B917F5FF1F130545C03A
:1047800097600100E78040A217C501001305050EE0
:1047900097600100E78020BA2A8497600000E780D4
:1047A00060F597100100E780809197800100E78015
:1047B000A02A97700000E780405197600000E780D2
:1047C000606B97300100E780E05297C50100938548
:1047D000650217C501001305258B19C897A00100B4
:1047E000E780202BA28517C5010013056512A1B72C
:1047F00097A00100E780E02917C501001305851384
:1048000097A00100E780E028294597A00100E780F4
:10481000202D97300100E780C02E97F00000E78040
:10482000804D7DC185453705040097300000E78045
:10483000609497C501009385E5FB17C5010013053A
:10484000A58497A00100E780C02417C501001305C7
:10485000E50F97A00100E780C023294597A001003C
:10486000E780002897F7FF1F938787A483D7070067
:1048700017170020231FF7EA854717170020230783
:10488000F7DA97F7FF1F938727B3DC4703D70700B3
:10489000C167FD176316F70097F0FFFFE780C06759
:1048A00097700000E78080CC1305C5149770000056
:1048B000E78080CC97200000E78080B5972000003B
:1048C000E78040A1171500200355A5E6975000008A
:1048D000E780C0CE054597500000E780C00197C52E
:1048E0000100938525F117B501001305E57997A01F
:1048F0000100E780001A17C501001305650797A09E
:104900000100E780001925BD97C50100938585EE5C
:1049100017B501001305457797A00100E7806017E0
:1049200017C501001305851897A00100E7806016E0
:10493000294597A00100E780A01A014569BF4111F0
:1049400022C437E404008327041A06C682979750CE
:104950000000E78060CA83270408170500001305DC
:104960008583829797F7FF1F238EA7EE17F5FF1F0A
:10497000130585A497400000E78060732244B2408D
:10498000410117030000670063CFB7E70400FC474D
:104990001171A2DDCAD986DFA6DBCED72E8432897B
:1049A0002E86AA8517F5FF1F1305C578829717F77E
:1049B000FF1F13072778834707009306800293871A
:1049C000E70793F7F70FE3ECF610BA898A0717B7F2
:1049D00001001307A774BA979C43BA9782878D4743
:1049E00097C50100938545E317B501001305C56917
:1049F000630FF40097A00100E780A00917C501002C
:104A0000130545A097A00100E780A008BDA497A0CA
:104A10000100E780000817C50100130525A097A035
:104A20000100E7800007294597A00100E780400BBF
:104A3000930720F8114697F5FF1F9385A56F4A85C8
:104A400017F7FF1F2308F76E97F7FF1FA385076E61
:104A500097F0FFFFE78040362A841DC997C5010003
:104A6000938585DB17B501001305056297A001004A
:104A7000E7802002A28517C501001305E59D97A0D8
:104A80000100E7800001294597A00100E78040056B
:104A900097C50100938545D817B501001305C55E7C
:104AA00097A00100E780E0FE17C501001305059CF3
:104AB00097A00100E780E0FD294597A00100E7806D
:104AC00020024165930730FA054697F5FF1F93854D
:104AD00065667D1517F7FF1F230EF76497F0FFFF3C
:104AE000E780802D2A841DC997C501009385C5D212
:104AF00017B501001305455997A00100E78060F93B
:104B0000A28517C501001305259597A00100E78030
:104B100040F8294597A00100E78080FCB7E7040032
:104B2000BC4F0566130606C8A14517F5FF1F0345D0
:104B300065D38297FE506E54DE544E59BE591161B2
:104B4000828091476303F40297C501009385C5CC29
:104B500017B501001305455397A00100E78060F3E6
:104B600017C501001305C59371BDB7E70400FC4FDD
:104B7000914517F5FF1F0345E5CE829797C50100C4
:104B8000938585C917B501001305055097A001004D
:104B9000E78020F017C501001305459297A001009A
:104BA000E78020EF294597A00100E78060F3974058
:104BB0000000E780201D914535A485476303F4027A
:104BC00097C50100938545C517B501001305C54B71
:104BD00097A00100E780E0EB17C501001305858F62
:104BE00015B597F7FF1F2397274BB7E70400056616
:104BF000BC4F130606C8C1450DBF8D476303F402C1
:104C000097C50100938545C117B501001305C54738
:104C100097A00100E780E0E717C501001305458D67
:104C2000D5B3930740F8114697F5FF1F938585503C
:104C30004A8517F7FF1F230FF74E97F7FF1FA38C27
:104C4000074E97F0FFFFE78020172A84E30405EE64
:104C500097C50100938545BC17B501001305C542F2
:104C600097A00100E780E0E2A28517B501001305D7
:104C7000A57E97A00100E780C0E1294597A001002B
:104C8000E78000E645BD9147E31CF4F6B7E7040072
:104C9000FC4F9305000217F5FF1F0345A5BC829743
:104CA00097C50100938545B717B501001305C53DAC
:104CB00097A00100E780E0DD17C501001305C5845A
:104CC000F1BD894763E3870297C501009385C5B4A9
:104CD00017B501001305453B97A00100E78060DB95
:104CE00017C501001305858331BB97F4FF1F83C4EB
:104CF000844497F7FF1F83C7F74397C50100938547
:104D0000A5B1A20417B5010013050538DD8C97A0E5
:104D10000100E78000D8A28517C501001305458171
:104D200097A00100E780E0D6C204294597A00100C2
:104D3000E78000DBC1849305D4FF93960401C18210
:104D40004A8693F5F50F17F5FF1F1305D53E9720FB
:104D50000000E780E045E35F90DC930750F817F729
:104D6000FF1F2309F73C83C73900228697F5FF1FF1
:104D70009385453C85074A8517F7FF1FA30DF73A32
:104D800097F0FFFFE78040032A84E30505DA97C523
:104D90000100938565A817B501001305E52E97A0BE
:104DA0000100E78000CFA28517C501001305C5CC1F
:104DB000C9B5894763E3870297C501009385C5A5F7
:104DC00017B501001305452C97A00100E78060CCC2
:104DD00017B501001305857735B197400000E780CE
:104DE00060FAA28517F5FF1F1305C5349750000020
:104DF000E78060A781B38D476303F40297C5010084
:104E0000938585A117B501001305052897A001001A
:104E1000E78020C817B5010013050575E5B6B7662C
:104E200002000146B7750200054597E0FF1FE780C5
:104E3000409B930760F817F7FF1F230DF72E97F796
:104E4000FF1FA38A072E9307000617F7FF1F2305EE
:104E5000F72E894717F7FF1FA300F72E97F7FF1FBD
:104E6000238D072C97F7FF1FA389072CC14717F73E
:104E7000FF1F2305F72C930720F917F7FF1FA30F38
:104E8000F72A314697F7FF1FA38BA72A97F5FF1F35
:104E90009385452A4A8597F7FF1F2382072A97F0B3
:104EA000FFFFE78060F12A84E30605C897C501008B
:104EB0009385859617B501001305051D97A0010080
:104EC000E78020BDA28517B501001305656B55B3BA
:104ED000B1476303F40297C501009385E59317B5C5
:104EE00001001305651A97A00100E78080BA17B585
:104EF00001001305A56A39B6B7E70400FC4F930516
:104F0000000417F5FF1F0345E595829797400000C1
:104F1000E78040E7B145F9B5914763E3870297C55C
:104F200001009385658F17B501001305E51597A05E
:104F30000100E78000B617B501001305E567D9B495
:104F400097F4FF1F83C4441F97F7FF1F83C7B71E43
:104F5000A204DD8C8E04B77702006D14BE94228605
:104F6000A68517B501001305656697A00100E780C7
:104F700040B2B7E70400FC47228697F5FF1F9385F0
:104F8000B51B2800829793160401C1823000A685C4
:104F9000094597E0FF1FE780C0842A8409C917B537
:104FA00001001305656497A00100E78060C69307C0
:104FB00070F8194697F5FF1F9385C5174A8517F7AF
:104FC000FF1F2309F71697F7FF1FA387871697F090
:104FD000FFFFE78060DE2A84E30E05B497C5010079
:104FE0009385858317B501001305050A97A0010075
:104FF000E78020AAA28517B501001305E55F95B9E2
:105000009947630BF41297C501009385E58017B5A6
:1050100001001305650797A00100E78080A717B579
:1050200001001305E55EF9BA914763E3870297B57E
:1050300001009385657E17B501001305E50497A06F
:105040000100E78000A517B501001305E55D5DBA15
:1050500097F4FF1F83C4440E97F7FF1F83C7B70D54
:10506000A204DD8C8E04B77702006D14BE942286F4
:10507000A68517B501001305655C97A00100E780C0
:1050800040A1B7E70400FC47228697F5FF1F9385F0
:10509000B50A2800829793160401C1823000A685C4
:1050A0000D4597D0FF1FE780C0732A8409C917B543
:1050B00001001305655A97A00100E78060B59307CA
:1050C00080F8194697F5FF1F9385C5064A8517F79F
:1050D000FF1F2301F70697F7FF1FA38F870497F0A1
:1050E000FFFFE78060CD2A84E30605A497B50100A1
:1050F0009385857217B50100130505F997A0010086
:10510000E7802099A28517B501001305255695B6AD
:1051100099476303F40297B501009385E56F17B5CE
:105120000100130565F697A00100E780809617B58A
:10513000010013052555F9B0B7E70400FC4F9305AE
:10514000000417E5FF1F0345E571829797400000B3
:10515000E78040C3994579B18D476303F40297B561
:1051600001009385656B17B501001305E5F197A064
:105170000100E780009217B501001305255259B0D0
:1051800017B501001305855297A00100E78040A8DC
:105190001305C01297D0FF1FE780A01A014597E0C2
:1051A000FFFFE78060EF0D4597100000E780E09F6C
:1051B000294597D0FF1FE780C01897D0FF1FE780D1
:1051C00020098DBA99476303F40297B501009385CE
:1051D000A56417B50100130525EB97A00100E78032
:1051E000408B17B501001305254D29B817F7FF1F90
:1051F000034797F497F7FF1F83C707F422075D8FD4
:105200009166BA96C2061166C1821306F6EF8D4703
:105210006365D60297E7FF1F9387071A9C4B17F623
:10522000FF1F034656F19386C7002DC203D6070021
:1052300069CA8907E39CD7FE89471307A0F811467E
:1052400097F5FF1F938505EF4A8597F6FF1F238388
:10525000E6EE17F7FF1FA300F7EE97F0FFFFE780DA
:10526000A0B52A84E308058C97B501009385C55A3B
:1052700017B50100130545E197A00100E7806081A3
:10528000A28517B5010013056544E5B203D60700F2
:10529000630EE60A8907E39BF6FE8D4779BF9147C7
:1052A0006304F40297B501009385055717B5010013
:1052B000130585DD97900100E780A07D17B50100FB
:1052C000130545426FF00FF4B7E70400FC4F930558
:1052D000000817E5FF1F0345E5588297C9B897B541
:1052E00001009385655317B501001305E5D9979023
:1052F0000100E780007A17B50100130525406FF023
:105300006FF02390E70017E5FF1F1305E50A9730BC
:105310000100E78080A497B501009385E54F17B59C
:105320000100130565D697900100E780807617B5D8
:1053300001001305A53D97900100E7808075294580
:1053400097900100E780C0798147C5BD2390070091
:1053500017E5FF1F1305450697300100E780E09F22
:1053600097B501009385454B17B501001305C5D1CD
:1053700097900100E780E07117B501001305853AA9
:105380005DBF411122C406C6834705002A849DC71C
:1053900097B501009385054417B501001305C5CEE7
:1053A00097900100E780E06E4C4017B501001305AF
:1053B000E57297900100E780C06DE1A05841B70702
:1053C000CF009387777D631DF70697B5010093851E
:1053D000654017B50100130525CB97900100E780C4
:1053E000406B1C448356E4008355C40003C6070089
:1053F00017B501001305057097900100E7806069FB
:10540000294597900100E780A06D0357E4009707B6
:10541000002083D707326309F7008355C40008448E
:1054200097E0FFFFE780C0DB0356E4008355C4002C
:1054300008442244B240410117F3FFFF670023559F
:10544000B707CC009387777D6315F70497B5010004
:105450009385453817B50100130505C397900100E2
:10546000E78020631C448356E4008355C40003C6D0
:10547000070017B501001305E56797900100E78065
:1054800040612244B2402945410117930100670061
:105490002365B707CE009387777D6304F70297B53E
:1054A00001009385253317B501001305E5BD9790DD
:1054B0000100E780005E4C4017B501001305C55898
:1054C000CDBDB240224441018280B7E70400FC47D1
:1054D00041112E8606C622C426C24AC02E842A89BD
:1054E000AA8517F5FF1F1305E5C4829797B501003C
:1054F0009385453417B50100130505B99790010050
:10550000E780205997F5FF1F83C5C5C217B5010075
:10551000130545DA97900100E780A0572945979039
:105520000100E780E05B97F4FF1F9384A4C083C76A
:10553000040041479387070693F7F70F636EF75A06
:1055400017B701001307C7C78A07BA979C43BA97D2
:1055500082879D476307F40297B501009385852DE7
:1055600017B50100130545B297900100E78060521E
:1055700017B50100130585D497900100E7806051AD
:105580008DA497F7FF1F83C7F7BADDCB17F7FF1F6F
:10559000034777BA97F7FF1F83C7E7B922075D8FE5
:1055A00097F7FF1F83C747B9C2075D8F97F7FF1FA4
:1055B00083C797B8E207D98F17F7FF1F232AF7B4DD
:1055C00083C7640097B501009385C52617B5010010
:1055D000130585AB17F7FF1F230BF7B29790010058
:1055E000E780204B97F7FF1F938787B28C4317F60E
:1055F000FF1F0346C6B117B501001305E5CD97900F
:105600000100E7800049294597900100E780404D5F
:1056100097F7FF1FA38007B22244B2409244024989
:10562000930700F817F7FF1F2306F7B09D4517F5FE
:10563000FF1F130525B04101174300006700A32297
:1056400097600000E780C0F197F7FF1F2385A7AEA2
:105650009357850017F7FF1FA30FF7AC935705016A
:105660002A8417F7FF1F2309F7AC935785010145DB
:1056700017F7FF1FA302F7AC97600000E780A0F2C6
:1056800097F7FF1F238BA7AA97B501009385851A6B
:1056900017B501001305459F97900100E780603F13
:1056A00017F6FF1F034666A9A28517B5010013056B
:1056B00025C4B1B7CD476303F40297B501009385C4
:1056C000651717B501001305259C97900100E78029
:1056D000403C17B50100130525C379BD37E404002C
:1056E0007C44414697F5FF1F9385D5A417F5FF1F0E
:1056F000130545A2829797F7FF1F83C7C7A417F723
:10570000FF1F034737A4A20703238405D98F17F788
:10571000FF1F231DF79E1306000A89452244B2404D
:105720009244024917E5FF1F0345C5134101028357
:105730008D476303F40297B501009385A50F17B554
:1057400001001305659497900100E780803417B538
:105750000100130525CB0DB517F4FF1F0344A49DCD
:1057600097F7FF1F83C7179D97B501009385850C99
:10577000220417B50100130525915D8C9790010057
:10578000E7802031A28517B50100130565B9979010
:105790000100E7800030294597900100E780403400
:1057A0000D4697F5FF1F9385E598228597E0FFFF4B
:1057B000E7808060AA8421C197B5010093858507A1
:1057C00017B501001305458C97900100E780602C08
:1057D000A68517B501001305E5B597900100E78090
:1057E000402B2244B240924402492945410117937B
:1057F00001006700E32E97F7FF1F239D8788B7E717
:105800000400116603A38705130606E8914539B71E
:105810008D476303F40297B501009385A50117B581
:1058200001001305658697900100E780802617B573
:1058300001001305E5CB89B317F4FF1F0344A48FC0
:1058400097F7FF1F83C7178F97B50100938585FED4
:10585000220417B50100130525835D8C9790010084
:10586000E7802023A28517B501001305E5AD9790C9
:105870000100E7800022294597900100E78040263B
:105880000D4697F5FF1F9385E58A228597E0FFFF78
:10589000E7808052AA841DC197B50100938585F9E0
:1058A00017A501001305457E97900100E780601E53
:1058B000A68517B50100130565AA05B797E7FF1F71
:1058C000239C877AB7E70400116603A387051306B4
:1058D00006E89305000299B5894763E3870297B507
:1058E0000100938525F517A501001305E57997902B
:1058F0000100E780001A17B50100130525C2ADB9F4
:1059000097F4FF1F83C4248397F7FF1F83C79782F1
:1059100097B50100938505F2A20417A501001305B0
:10592000A576DD8C97900100E780A016A68517B5B7
:105930000100130525A497900100E78080152945F3
:1059400097900100E780C019228697E5FF1F938595
:10595000657E268597E0FFFFE78000462A84630E78
:10596000051A97B501009385E5EC17A5010013050D
:10597000A57197900100E780C011A28517B50100BD
:10598000130585A099BD854763F9871883451900DC
:105990002244B24092440249B335B00097E7FF1F5A
:1059A0002384B77017B501001305459F4101179374
:1059B00001006700030EA2852244B24092444A854A
:1059C00002494101170300006700632499476303FC
:1059D000F40297B501009385E5E517A501001305CD
:1059E000A56A97900100E780C00A17B5010013056A
:1059F000A5CC59B617E4FF1F0344E47397E7FF1FD4
:105A000083C7577397B501009385C5E2220417A594
:105A10000100130565675D8C97900100E7806007C2
:105A2000A28517B501001305E59897900100E7805E
:105A30004006294597900100E780800A194697E5BE
:105A4000FF1F9385256F228597E0FFFFE780C03613
:105A5000AA841DC197B501009385C5DD17A5010076
:105A60001305856297900100E780A002A68517B50F
:105A700001001305259595B397E7FF1F2394876AC7
:105A8000B7E70400116603A38705130606E893052C
:105A9000000869B1854797B501009385A5D917A579
:105AA00001001305655E630BF40097900100E78029
:105AB00040FE17B50100130525927DBC97900100AB
:105AC000E78020FD17B5010013058592979001002E
:105AD000E78020FC294597900100E7806000224480
:105AE000B2409244024997E7FF1F239107624101A8
:105AF000176300006700439797B50100938585D32E
:105B000017A501001305455897900100E78060F83C
:105B100017B50100130585BE85B4B24022449244F6
:105B2000024941018280411106C622C497E0FFFF6D
:105B3000E780802821CD97E7FF1F83D70757850788
:105B40002A8417E7FF1F2312F75697B501009385A4
:105B5000E5CF97E7FF1F239BA75417A50100130567
:105B6000A55297900100E780C0F2A28517B5010009
:105B7000130585F097900100E780A0F12244B24020
:105B80002945410117930100670083F597E7FF1F3F
:105B900083D7E751B2402244850717E7FF1F231838
:105BA000F75041018280411122C491462A8417E6B0
:105BB000FF1F130626669D652D4506C697D0FF1F5D
:105BC000E78020C2B7F7070003C70701A5476313A3
:105BD000F70001A09306001001469D65254597D06A
:105BE000FF1FE78000C097E7FF1F238587622244DD
:105BF000B240914617E6FF1F1306C6619D65294511
:105C0000410117D3FF1F6700C3BD1171CED7B7E99C
:105C1000040083A7C904CAD917E9FF1F13098951D2
:105C2000A2DD2E8686DFA6DB2E84AA854A85829792
:105C300097E7FF1F83C707501307700A6385E710B4
:105C4000636DF7001307600A6385E704FE506E5426
:105C5000DE544E59BE59116182801307800A638554
:105C6000E7161307900AE393E7FE8D476306F41CDB
:105C700097B50100938585F317A501001305C5406D
:105C800097900100E780E0E017B50100130545EFAC
:105C900025A08D47630CF40297B50100938505F1AB
:105CA00017A501001305453E97900100E78060DECF
:105CB00017B50100130505E697900100E78060DD48
:105CC000294597900100E780A0E149B7854717B5BE
:105CD00001001305E5E517E7FF1F2307F73C979041
:105CE0000100E780E0F2B7750200B76602000146E6
:105CF000054597D0FF1FE780C0AE930760F817E710
:105D0000FF1F2309F74297E7FF1FA3860742930768
:105D1000002617E7FF1F2321F742E5779387072126
:105D200017E7FF1F231CF740B14597E7FF1F2388A4
:105D3000074097E7FF1FA384A7404A85970000000C
:105D4000E780E01621B7914763E3870297B501002A
:105D50009385C5E517A5010013050533979001004C
:105D6000E78020D317B50100130585DEB1B797E4AE
:105D7000FF1F83C4643C97E7FF1F83C7D73BA20480
:105D8000DD8C83A7C9046D14228697E5FF1F9385D8
:105D9000B53A280082978E0493160401B775020065
:105DA000C1823000A695094597D0FF1FE78060A308
:105DB000930770F817E7FF1F230EF736994597E70B
:105DC000FF1FA38BA73695BF914763E3870297B563
:105DD00001009385A5DD17A501001305E52A97901D
:105DE0000100E78000CB17B501001305E5D7E9B541
:105DF00097E4FF1F83C4443497E7FF1F83C7B7337B
:105E0000A204DD8C83A7C9046D14228697E5FF1FC9
:105E100093859532280082978E0493160401B775F6
:105E20000200C1823000A6950D4597D0FF1FE78084
:105E3000409B930780F8BDBF17B50100130585D5BA
:105E400097900100E780C0DC930790F82304F100ED
:105E5000834719008D452800A304F10083472900DA
:105E60002305F10097000000E78060041305C012CD
:105E700097C0FF1FE780E04C014597D0FFFFE78008
:105E8000A0210D4597000000E78020D2294597C04A
:105E9000FF1FE780004B97C0FF1FE780603B7DB38B
:105EA00097E7FF1F23A0A738828097E7FF1F9387FC
:105EB000673703A30700630303000283174300004F
:105EC0006700639A41114AC09706002083D6668610
:105ED000328917D6FF1F0356465022C426C206C673
:105EE0002A84AE8497000000E780C05D35C12DC0D4
:105EF000994763FF97048347140003470400A207F0
:105F0000D98F13978700A183D98FC2073167C183C7
:105F10001307C755639EE70297D7FF1F83D7E74B49
:105F2000A301F400A1832302F4009707002083D784
:105F3000478091C7A302F400A1832303F400A68540
:105F400017B50100130585CA97900100E78060B47A
:105F500097F7FF1F83C7876DA5C797D5FF1F83D509
:105F6000C54717B50100130525CA97900100E780C2
:105F700040B22686A28517D5FF1F03550546970018
:105F80000000E78080BA6306090497F7FF1F83C704
:105F9000E769A1E397E7FF1F83C707299DCB95C852
:105FA00097E7FF1F83C747108DE722852244B24041
:105FB0000249A68592444101174300006700A38A65
:105FC00017B50100130545C597900100E78040C44F
:105FD0005DBFB2402244924402494101828083471E
:105FE00055008345450017B501001305E5BEA2071E
:105FF000DD8D179301006700C3A917B501001305D4
:10600000A5BC179301006700A3C08D4763FBB70AC7
:10601000011126CA06CE22CC0344350097E4FF1FA7
:1060200083C4942097B501009385C5BFB337800022
:1060300017E7FF1FA30AF71E09C497B50100938550
:1060400025BF17B50100130525BF97900100E78014
:1060500040A497E7FF1F83C7371D6386970097000B
:106060000000E780E02E97E7FF1F83C7F71B8DC76F
:1060700085472306F100B7E7040083A747177000A0
:10608000854513055030829717B501001305C5BB30
:1060900097900100E780C0B79967938757EE231662
:1060A000F100680085479145A30781002307F100AF
:1060B00097000000E780A0DFF2406244D24405610F
:1060C00082808280894763F7B708011122CC06CE0F
:1060D00026CA8344250085472A84639DF40491479A
:1060E00063F5B704034545008347340022055D8D01
:1060F00097D7FF1F2393A72E97000000E7806045E6
:106100009967938767EE2314F100834734002305D2
:106110009100A305F100834744009545280023061C
:10612000F10097000000E78080D8F2406244D2443A
:1061300005618280FDF89967938767EE2314F1006B
:1061400097D7FF1F83D76729A305F1002305010017
:10615000A183E1B782800111996722CCD51717F48A
:10616000FF1F1304A44C2314F1008347040026CA24
:1061700097F4FF1F9384E45B2305F10083D70400A9
:1061800028009545A305F100A18306CE2306F10062
:1061900097000000E780A0D103D6040083450400E7
:1061A00017B501001305C5AB97900100E780608E1D
:1061B000F2406244D244056182809D677971D917AB
:1061C0002316F10097F7FF1F83C7474606D623071C
:1061D000F100A9C3B7E70400FC47414697E5FF1F5C
:1061E000938545F31305F10082976800CD4597002C
:1061F0000000E780C0CB97F5FF1F83C5254317B587
:1062000001001305E5A897900100E7808088B2504F
:1062100045618280B7E70400BC47414681451305CC
:10622000F1008297D9B745C5411106C622C493072C
:1062300050FA2300F5009307A005A300F500894755
:106240002301F5009147A301F5009307A003A302E2
:10625000F50097F7FF1F9387673D83C70700230269
:1062600005002A842303F50097E7FF1F9387D7FBD8
:1062700083C70700414697E5FF1F9385A5E9A30360
:10628000F50097F7FF1F83D7C74A2304F500A183C2
:10629000A304F50097D7FF1F83D727142305F50024
:1062A000A183A305F500B7E70400FC4731058297F9
:1062B0002285F14597000000E780C01C230EA40052
:1062C0002181A30EA400B240224441018280828039
:1062D0005D710A8586C6A2C497000000E780E0F4DD
:1062E00037E404007C448A850810794682973C4450
:1062F0001305E103094681458297101093050002BA
:10630000014597D0FFFFE780603FB64026446161BA
:106310008280411122C426C24AC02A84AE843289B6
:10632000AA8585660146254506C697C0FF1FE780FA
:10633000404BA2852244B240CA8626860249924436
:106340002945410117C3FF1F6700A3490111B7C7C2
:10635000A55A22CC9387C73317E4FF1F1304D4EC4C
:106360003EC4834704002C002146196506CE3EC674
:1063700097000000E78020FA8345040017B501006C
:10638000130505A097800100E780A070F2406244E9
:10639000056182800111A146300099652D4522CC0E
:1063A00006CE97C0FF1FE780C043A24737C4A55A57
:1063B0001304C43363958702B24517B50100130572
:1063C000658FB335B00097E7FF1FA38FB7E49780C1
:1063D0000100E780006CF2406244056182809165B3
:1063E000A1463000938505F02D4597C0FF1FE7803B
:1063F000403FA247E38287FC97E7FF1FA38607E29F
:10640000814517B501001305258DD1B77971D146A6
:10641000700091652D4522D406D697C0FF1FE780F6
:10642000403CB24737C4A55A1304F4356398870239
:10643000B7E70400FC4717E5FF1F1305A5CD41464C
:106440000C08829717B501001305058F978001008E
:10645000E780007CB2502254456182809165D1462C
:106460007000938505E82D4597C0FF1FE7806037D2
:10647000B247E38F87FA17B501001305E58DF9B729
:10648000C16769768146FD170506139706014183AA
:106490006364B7003E8582803307D5000347070059
:1064A000B98F214713F81700858363050800B18F62
:1064B000C207C1837D171377F70F6DF78506F1B714
:1064C00041C5A547054763F2B70883471500034751
:1064D00005003168A207D98F13978700A183D98F50
:1064E000C207C1831308C8550547639007074111C8
:1064F00006C622C426C203442500914763F08704E0
:106500009307540063ECF502A301C5002182230226
:10651000C5009304340091C6A302D500A1822303D1
:10652000D5002A84A68597000000E780A0F5269470
:106530002300A4002181A300A4000147B24022440B
:1065400092443A854101828005473A858280011153
:10655000B7C7A55A22CC9387E7342A842AC6214696
:106560002C00156506CE3EC497000000E780A0DA37
:10657000A28517B501001305A58297800100E78069
:10658000405197000000E780E0D4F240624405618A
:1065900082800111A146300095652D4522CC06CEA2
:1065A00097C0FF1FE780E023A24737C4A55A130412
:1065B000E43463958702B24517A501001305C5733E
:1065C00097D7FF1F239BB7E0C205C18197800100C9
:1065D000E780204CF2406244056182809165A146CB
:1065E0003000938505EE2D4597C0FF1FE780601FA3
:1065F000A247E38287FCD14717D7FF1F231FF7DC91
:10660000D14517A5010013052571C9B721C1411155
:1066100026C206C622C4AE848DC52A849700000017
:10662000E780806697E7FF1F83C707C099CB228565
:106630002244B240A685924441011733000067000E
:106640008322B2402244924441018280828001111F
:106650004AC806CE22CC26CA4EC693F715002E890C
:106660009DCBAD67371700409387A7AA1CC3B7E738
:106670000400BC4F13060019854517D5FF1F0345BD
:10668000A5D5829713451900F2406244D24442498D
:10669000B2490561828093F72500638A071C17F7CA
:1066A000FF1F0357E708954763F9E70C014417F606
:1066B000FF1F1306E6F79306300513055004130871
:1066C00010049308B00413039005930764006374E7
:1066D000F7043A84FD5997F4FF1F83C464F597F7D4
:1066E000FF1F83C7F7F4A204DD8CAD679387B7550E
:1066F000638BF41463E3970AA9679387A755638EA6
:10670000F414A28517F5FF1F130585F2970000000A
:10671000E78000F031A2B307860083C50700639AC3
:10672000D50483C517006396A50483C5270063922B
:10673000050583C53700639ED50283C54700639A6C
:10674000150383C7570063966702A2890DE897F582
:10675000FF1F83D5E5FDB3853541C20517F5FF1F42
:10676000130505EDC1814E9597000000E78040EAD2
:10677000E1A005044204418089BF3A84FD59854760
:10678000E3EB87F45DC4854517F5FF1F130545EA64
:1067900097000000E780C0E769A8B1679387C755F5
:1067A0006380F404B5679387D755E39CF4F4A2851E
:1067B00017F5FF1F1305C5E797300000E780A00A13
:1067C0008947630FF4049305E4FFC205C18117F5FF
:1067D000FF1F130505E697000000E780E04A89A047
:1067E00097200000E780C0F797000000E78020496D
:1067F00011C9A28517F5FF1F130585E39700000057
:10680000E78080480546A28517F5FF1F130545E27E
:1068100097F0FFFFE780406B97200000E78040F48F
:10682000A68517A501001305655997800100E7802B
:106830004026FD57E39DF9F097F7FF1F239A07EED7
:106840001345290091B5A28517F5FF1F130545DEF5
:1068500097F0FFFFE780E078E1B7A28517F5FF1F0B
:10686000130505DD97F0FFFFE780607955BF93F7CB
:1068700045000145E38A07E017A5010013054555CA
:1068800097800100E780C03897300000E780402BF8
:1068900013454900D5BB411122C437E404005C5CB8
:1068A00006C6354697A501009385450317B5010037
:1068B0001305C5D1829711E917A5010013050552EB
:1068C00097800100E780C03401A08327041C8297D1
:1068D0002A84054597C00000E78000E89760010022
:1068E000E780206D97600100E780204297B00000AC
:1068F000E78080F92285B240224441018280411123
:10690000054506C622C426C297C0FFFFE780A062E5
:106910001305A00497B0FF1FE78060797575854562
:106920007D1597C0FFFFE780404C7D7585451305B9
:10693000F53697C0FFFFE780A05537140040832746
:10694000840A8D451305002093E707202324F40AC9
:1069500097C0FFFFE7806049B7E4040097D0FFFFCE
:10696000E780808EC85897800100E780602A17B5BD
:1069700001001305A5C597800100E78060298327E2
:10698000840C8545414593E707082324F40C97C000
:10699000FFFFE780E04F8D451305000897C0FFFF1C
:1069A000E780004F97C0FFFFE780E07B37A5070037
:1069B0001305051297C0FFFFE7808077014597C058
:1069C000FFFFE780A07D95450545894717F7FF1F25
:1069D0002302F7D697C0FFFFE780E07DB7E700E02E
:1069E00013070006238DE7403707000423A0E710B4
:1069F00097D0FFFFE78060FF97D0FFFFE78060112F
:106A000097000000E78060E997000000E780C098E9
:106A100097000000E78020B897E0FFFFE78060F272
:106A200097000000E780802797000000E780801033
:106A300083A70408170500001305A5C1829797D7FF
:106A4000FF1F238BA798BC4C1306006485458297D3
:106A500097C0FF1FE780C09901458280AD67371757
:106A600000409387A7AA1CC3B7E700E037074000A0
:106A700023A0E71801000100B7F7070003C70701CB
:106A8000A5476316F7009397450191C301A04111F3
:106A9000AE860146AA85254506C697C0FF1FE7803A
:106AA00040D4B240B7E700E03707400023A0E7102A
:106AB000410182804111B2862E86AA852D4506C6E7
:106AC00097C0FF1FE780E0D1B240014541018280BD
:106AD0009307000463ECC7041D71A2CC2A84080844
:106AE000A6CACAC886CE32C697800100E78000EFEA
:106AF000AD67371700409387A7AA1CC3B7E400E02F
:106B00003709400023A0241901000100B2461008F3
:106B1000A285294597C0FF1FE780A0CCF6406644B8
:106B200023A02411D64446492561828039558280AC
:106B300041110D658D4506C697C0FFFFE780E02A2D
:106B4000B71700408D6623A6D70A17F5FF1F130558
:106B5000A5BE1387C70A9387870A1CC15CC58566D3
:106B600089675CC958C114C518C9B7E70400B240A9
:106B700003A3871E410102838145B307B5008387C4
:106B8000070089E717230000670023C48505C205B5
:106B9000C181E5B797A701009387473E1357C5000A
:106BA0003E9703470700011106CE2304E100135767
:106BB00085003D8B3E970347070023060100A30491
:106BC000E100135745003D8B3D893E97AA97034747
:106BD000070083C7070028002305E100A305F10093
:106BE00097000000E78080F9F24005618280411142
:106BF00026C2E97797F4FF1F938484C422C4938745
:106C0000A7552E842381B4002E86AA8517F5FF1F71
:106C1000130545C306C62390F400A38104009780A2
:106C20000100E780A0DB93052400C205C18117F5B0
:106C3000FF1F130505C197000000E780A084B387FC
:106C400084002382A7002181A382A700930564000A
:106C50002244B24026859244C205C18141011723D6
:106C60000000670083B609C99307800263E6B70096
:106C7000170300006700E3F7828017F5FF1F034545
:106C800025AD828097F7FF1F83C747BB89E717238E
:106C90000000670083B3828097F7FF1F83C727BD7B
:106CA00099EF411106C697200000E780E0A9B240A5
:106CB000854717F7FF1F230CF7BA410182808280B6
:106CC0006307054A6385054A5D71CAC04EDE86C604
:106CD000A2C4A6C252DC56DA5AD85ED662D466D2B4
:106CE0006AD0B9472A89AE8963F9B706394697A5AC
:106CF00001009385651697800100E780C0CB31EDD8
:106D00008347E900130710036394E702854717F7E9
:106D1000FF1F2305F7B217A501001305E51497F728
:106D2000FF1F239C07B097000000E78020E571A0BB
:106D30001307000317A5010013050516E395E7FEE9
:106D400097F7FF1F238C07AE97F7FF1F239707AE18
:106D500017A501001305C512F9B797F7FF1F83C7E1
:106D6000E7AD63870722BD6AB96B938CFA55014A78
:106D700017FBFF1F130B0B9E138CEB65938AFA66B0
:106D800005A8B307490183C6070097F7FF1F83D7FC
:106D9000C7AAB1E39307A005639BF600854717F7E1
:106DA000FF1F231CF7A897F7FF1F2385D79A050A13
:106DB00093170A01C183E3E637FDB64026449644A3
:106DC0000649F259625AD25A425BB25B225C925C2B
:106DD000025D61618280054D639BA7039307500AA2
:106DE000639EF600894717F7FF1F2318F7A4930740
:106DF00050FA17F7FF1FA30FF79455BF9307A0058D
:106E0000E387F6FA97F7FF1F239907A24DB7138779
:106E100017004207DA9741832380D70017F6FF1F38
:106E2000231DE6A08D47E3F4E7F817F4FF1F0344A2
:106E3000949297F7FF1F83C7079222045D8C9307F4
:106E4000F4FFC207C1839306F00DE3EDF6FA930752
:106E50006400C207C183E31CF7F493052400C20554
:106E6000C18117F5FF1F1305058F97F0FFFFE7801E
:106E7000606133078B008347570003474700A20731
:106E8000D98F17F7FF1F231A079A6318F50E81444D
:106E9000630CA40197F4FF1F83C4048CA20497F72A
:106EA000FF1F83C7778BDD8C170500001305E5DB1B
:106EB00097F0FFFFE78000FF63878407636D9C0204
:106EC0009387EB556382F40497F7FF1F83C7C78846
:106ED00005476389E70681CB1387A7051377F70F6B
:106EE0008D4663F2E6081307F0072300E100A300D4
:106EF000F10089459DA063829405E39754FD97F0C6
:106F0000FFFFE780C02B11A8A28517F5FF1F13050F
:106F1000A58497F0FFFFE780800F014597F0FFFF02
:106F2000E78040F869B5A28517F5FF1F1305C582F4
:106F300097F0FFFFE7804019CDB797F0FFFFE7809C
:106F4000C021E1BF930710F8130511002300F100E1
:106F500097F0FFFFE780602DFD450A859700000050
:106F6000E78020C95DBFA28517E5FF1F1305C57E19
:106F700097F0FFFFE780A0C94DB79307F007894559
:106F80000A852310F10097000000E78080C605B550
:106F9000BD4763F83717414697A50100938505F271
:106FA0004A8597800100E78000A1631C051417A59E
:106FB00001001305E5F197000000E78020BC17E50C
:106FC000FF1F0355057797000000E780E0BC97E7B7
:106FD000FF1F83C7A76517A501001305E5E689E72D
:106FE00017A501001305C5E697000000E78000B96A
:106FF00017A50100130545EF97000000E78000B8D2
:1070000017C5FF1F0355053B97000000E780C0B878
:1070100017A50100130585ED97000000E78000B675
:1070200017C5FF1F0355653B97000000E780C0B6FA
:1070300017A50100130505EC97000000E78000B4D8
:1070400017D5FF1F0355A50697000000E780C0B4C1
:1070500017A50100130585EA97000000E78000B23C
:1070600017D5FF1F0355650497000000E780C0B2E5
:1070700017A50100130505E997000000E78000B09F
:1070800017D5FF1F0355850297000000E780C0B0A9
:1070900017A50100130545E797000000E78000AE43
:1070A00017C5FF1F0355C52197000000E780C0AE3C
:1070B00017A501001305C5E597000000E78000ACA7
:1070C00097D7FF1F83C70705A20717D5FF1F0345E3
:1070D00075045D8D97000000E78000AC97D7FF1F17
:1070E00083C76703A20717D5FF1F0345D5025D8D30
:1070F00097000000E78040AA179501001305855509
:107100001DB1C14763FE3705414697A50100938530
:1071100065E04A8597800100E780E08931E1834797
:10712000090113071003639CE700854717E7FF1F5A
:107130002300F76217A50100130505DFEDB613075D
:10714000000317A50100130525E1E39EE7BC97E7BF
:10715000FF1F238F075E17A50100130565DEE1B64B
:10716000CE854A8597C0FFFFE7808007B9B182804E
:10717000411126C2AE848D4522C406C62A8497C01A
:10718000FFFFE780E0D0B717004099C803A5C70C00
:10719000418D23A6A70CB240224492444101828033
:1071A00003A5870C418D23A4A70CF5B783470500E1
:1071B00003471500A207D98FC2076177C18713075C
:1071C0002720639AE700834525003705040017034D
:1071D0000000670023FA828017E6FF1F1306866906
:1071E0008147B2861303F00FA9483308F60003481D
:1071F000080013F7F70F6307A80C630668008507FC
:10720000E39517FF2947B387E6002380A70097E798
:10721000FF1F9387E7665DA8411113D765001347E9
:10722000170006C693F63500058B954791CA0546AB
:1072300099476387C60009469D476383C600A147F7
:1072400013F645003336C00093F68503050685C264
:10725000A145638BB604E145638AB60493058002B9
:107260006388B604930580036393B600914697F54F
:10727000FF1F238CF58697F5FF1F2387C58697F59B
:10728000FF1FA383D586BE8517A50100130505D36F
:1072900097700100E780E07FB240854717F7FF1F36
:1072A000A305F784410182808546D1B78946C1B7DD
:1072B0008D4675BF17A501001305C5D217730100D0
:1072C0006700237D17E7FF1F1307875BBA972380AB
:1072D000B700E147E302F5F493077002E30CF5FC15
:1072E00082802A8723800500814717E5FF1F130549
:1072F00065581308F00F2946B306F50083C606004B
:107300006396E60297E6FF1F93868657B69783C774
:10731000070005452380F5009947636EF7029D47F6
:1073200063FDE700E147630DF70082806385060196
:107330008507E393C7FC0145C5B72380050082801C
:10734000B737004003C7370083C7050093F707042A
:10735000D98F2380F50082805D7152DC56DA5ED6CB
:10736000716A97FBFF1F938B6B898D6AA6C24EDEF5
:1073700062D486C6A2C4CAC05AD866D26AD06ECEBB
:10738000C1495E8C97E4FF1F93844450130A0A207E
:10739000938A7ADC17F9FF1F03494989B3872B01C8
:1073A00083C7070093F7F70FC9EFB787004003C7FC
:1073B0006700058BE310077C03C76700118BE30DA3
:1073C000077E83C75700918B99E36F10200317F74F
:1073D000FF1F0347C78585476304F7006F1040010F
:1073E00097E7FF1FA383E77097E7FF1F23800756E8
:1073F00097E7FF1F238E076097E7FF1F238C076C1B
:1074000097E7FF1F2389076C97E7FF1FA3800754A7
:1074100097E7FF1FA38E075E97E7FF1FA38C076AFE
:1074200097E7FF1FA389076A97E7FF1FA380076CF1
:1074300097E7FF1FA38D077EB787004011476F00B6
:1074400070779307190093F7F70F3D476364F706CA
:1074500017E7FF1F230CF77C97E7FF1F9387077C35
:10746000CA9783C707001307100293F7F703638EC9
:10747000E71E6366F70405446385871CE38C076297
:107480000947638EE71013070002E384E74EB7E76E
:1074900000E03707400023A0E718010001006299CF
:1074A00023000900FD1923A0E71093F9F90FE393D6
:1074B00009EEE5BD97E7FF1F238A077671BF130723
:1074C00030026388E70C63E8E71613074002638C19
:1074D000E70A13070003E39CE7FA97E7FF1F938788
:1074E000E772CA9703C70700A1471377F70FE31B9B
:1074F000F71483C7640097E6FF1F238FF65C97E7B6
:10750000FF1F83C7173991C7FD5797E6FF1F2385D4
:10751000F65C97E5FF1F83C5753797E7FF1FA38DBF
:10752000B75A97E7FF1F83C7673613FB0708930611
:10753000000493F70706639FD74C9307A009638D58
:10754000F51663EAB7129307F0056386F54A9307C9
:1075500050096384F52A014497E7FF1F83C7D75773
:107560001547E392E736B7E700E03707400023A06E
:10757000E71801000100B786004023808602130649
:1075800080FC6F00500EFD5717E7FF1F2305F754CF
:10759000FDBDFD5717E7FF1F230EF752CDBD17A501
:1075A00001001305A5B597700100E780606697E7B5
:1075B000FF1F9387A765CA9703C40700014B97EC89
:1075C000FF1F938C2C451374F40F17AD0100130D9E
:1075D0006DB363478B04294597700100E7804050E5
:1075E000854717E7FF1FA305F74217E7FF1F230291
:1075F000874217E7FF1F230BF74E37E700E0B70678
:1076000040002320D718010001003786004083473F
:10761000A60293F7370F2305F6022320D71085BD66
:10762000B3876C0183C507006A85050B977001005D
:10763000E780204679BF854717E7FF1F230AF73CFD
:10764000B9B517E7FF1F1307675C4A9703470700A1
:1076500097E6FF1FA38CF62E97E6FF1F2389E62EE1
:1076600017E7FF1F2304F7481DB5854717E7FF1FDE
:10767000230EF72C29BD9307400A6389F53493073D
:10768000200B6384F5369307100AE396F5EC8387A5
:1076900024000144E3D207EC97E7FF1F83C7371F9D
:1076A00093F63700638A061A0546638AC62209469E
:1076B0006395C61A1D4755A217E5FF1F0345251DF3
:1076C000C94797ECFF1F83CC9C1C97E5FF1F83C520
:1076D000251C17E4FF1F0344B41B6315F510CD47A9
:1076E0006392FC1093077008639CF5021307300F38
:1076F000B7170E006308E4001307900DB7B7040036
:107700006314E40817E7FF1F232EF73CBE8517A577
:1077100001001305A59F97700100E780803725BD04
:1077200093078008639DF500B307804013F4F70FBB
:10773000B7774600938787CDB3D78702E1B7930722
:107740009008639AF500B307804013F4F70F916730
:107750009387C766D5B79307A008639BF500B30767
:10776000804013F4F70FB7173D0093870790E9B7F0
:107770009307B008639AF500B307804013F4F70F3E
:107780009167938797D04DBF93F5F5078D47639B1E
:10779000F500B307804013F4F70FB7975B009387AA
:1077A00007D859BF8947639BF500B307804013F49E
:1077B000F70FB7770B009387071BBDBF8547639A09
:1077C000F500B307804013F4F70FDD67938767E395
:1077D000A5B7D28785F9B307804093F7F70FB3D7E2
:1077E000FA020DB797000000E780409FA2856685EA
:1077F00097000000E780809EB9BB9305610017E504
:10780000FF1F0345C50817E4FF1F034454089700F2
:107810000000E78040AD93057100228597000000CD
:10782000E78060AC3C0017E7FF1F2327F73C834746
:1078300061002304F10083477100A304F10089472C
:1078400017E7FF1F230AF7288357810017E7FF1F59
:10785000231EF702094409B3154793F64700B336D0
:10786000D00093F78703850685C32146638BC7063F
:107870006146638AC706130680026388C70613063B
:1078800080036393C700914717E6FF1F230ED6249A
:1078900097E6FF1FA38AF62497E7FF1F2387E724B5
:1078A00017E7FF1F0347C7FE9376070497E7FF1FFD
:1078B00083C717FE8DEE1377770C93067008630C61
:1078C000D7021377F7078D466312D70CB307F04042
:1078D000B7955B0093F7F70F938505D849A819472B
:1078E000ADBF854755B7894745B78D4771BF9306EB
:1078F00070086311D7021307300FB7150E006389A4
:10790000E7021307900DB7B504006383E70213077E
:10791000700845BF9306800C6311D702B307F0408F
:10792000B775460013F7F70F938785CDB3D5E702F8
:1079300097E7FF1F23A8B71AD9BB9306900C631CC7
:10794000D700B307F04093F5F70F91679387C766A9
:10795000B3D5B702F1BF9306A00C631DD700B307E0
:10796000F040B7153D0093F7F70F93850590B3D519
:10797000F5027DBF9306B00CE315D7F4B307F040D2
:1079800093F5F70F9167938797D0D9B78946631B13
:10799000D700B307F040B7750B0093F7F70F938547
:1079A000051BF1B78546631AD700B307F040DD65C4
:1079B00093F7F70F938565E35DBFD28535FBB3057C
:1079C000F04093F5F50FB3D5BA029DB783C72400F5
:1079D000C18B99C7854717E7FF1F2302F710A5BE84
:1079E00097E7FF1F238D070EBDB6854717E7FF1FDB
:1079F000A30DF70E8DB63C0017E7FF1F232EF71ED1
:107A00000947930700032314F10097E6FF1F23851E
:107A1000E60C2DBD63940756A94763E5B742179757
:107A200001001307E7568A05BA959C41BA978287E9
:107A300017E4FF1F0344B4E5894C6306940D63E625
:107A40008C0685476303F4089307F00F17E7FF1FC1
:107A50000347870863F6E70017E7FF1F230EF706C3
:107A600097ECFF1F83CC4C079307000413F4FC0F23
:107A700063F497011304000497E7FF1F9387C71768
:107A800003AD070022862685EA85B38C8C40229DB3
:107A900097700100E78080F497E7FF1F238E97031C
:107AA00097E7FF1F23AAA71545BC8D47630CF40A6F
:107AB0009947E31BF4F8979701009387E75317E77B
:107AC000FF1F232BF712A94751B717E7FF1F0347E3
:107AD000071697E7FF1F93872702494697950100EE
:107AE0009385855A63068700979501009385C55550
:107AF0003E8597700100E78060EE17E7FF1F232D9A
:107B0000A70EC947A1B797E6FF1F83C646120547D0
:107B100097E7FF1F938747FE6394E6023E851306AF
:107B20007002979501009385A55397700100E78037
:107B3000E0EA17E7FF1F2321A70C9307700239B76C
:107B40003E8513063004979501009385A54B9770E9
:107B50000100E780A0E817E7FF1F232FA70893077E
:107B60003004EDB597E5FF1F83C565D21795010079
:107B70001305055B97700100E780A0F1054D97EDB7
:107B8000FF1F83CDCD0A97E5FF1F83C545D017950D
:107B900001001305E5586398AD0B97700100E7806D
:107BA00040EF97E7FF1F83C787CEB5CBE36EF4E8BE
:107BB0001794010013048451638CB70117940100DA
:107BC000130444516386970117940100130404526F
:107BD000228597700100E780E0041375F50F930785
:107BE0001500860717E7FF1F2308F7F08D4717E7F3
:107BF000FF1FA303F7F097E7FF1F9387E7EF014706
:107C0000BE861376F70F89076365A60297E7FF1F05
:107C100023A4D7FE97E7FF1F83C707EE05BD9797FD
:107C200001009387A74317E7FF1F2327F7FC91471E
:107C300031BD3306E40003460600A38007000507B4
:107C40002380C7007DBF97700100E78080E497E73D
:107C5000FF1F83C7C7C3E1D7E368F4DE17940100B1
:107C60001304C443638CA7011794010013048443D5
:107C7000638697011794010013044444228597708A
:107C80000100E78020FA1375F50F930715008607AA
:107C900017E7FF1F2302F7E68D4717E7FF1FA30D26
:107CA000F7E497E7FF1F938727E50147BE86137622
:107CB000F70F8907E37CA6F43306E40003460600C9
:107CC000A380070005072380C700D5B797E5FF1FEE
:107CD00083C5E5BB17950100130545459770010065
:107CE000E78020DB97E7FF1F83C7D7E093E74700D4
:107CF00017E7FF1FA300F7E083C7240017E7FF1F64
:107D0000A308F7DE89B8179501001305654397703E
:107D10000100E780E0EF97E7FF1F938767DD83C7E8
:107D2000070017E7FF1F2303F7B617E4FF1F0344FD
:107D3000A4DA333480000DB0179501001305854196
:107D400097700100E780C0EC97E7FF1F83C797DAC1
:107D500093E7070117E7FF1FA30EF7D883C7240097
:107D600017E7FF1F2306F7D86FF0EFFE1795010006
:107D70001305853F97700100E78080E903C7040081
:107D80007D8B51EFB787004003C767021377C70B9E
:107D9000136727002383E70203C7A7021377C70BE4
:107DA000136727002385E70203C7E7021377C70B92
:107DB000136727002387E70203C727031377C70B3F
:107DC000136727002389E702854717E7FF1F230F63
:107DD000F7B617E7FF1F230DF7C217E7FF1F230BA7
:107DE000F7CE17E7FF1F2308F7CE97E7FF1FA38FF4
:107DF00007B497E7FF1FA38D07C097E7FF1FA38B6B
:107E000007CC97E7FF1FA38807CC97E7FF1FA38F37
:107E100007CC97E7FF1FA38C07E06FF0CFF38947EC
:107E20006312F70297E7FF1F83C787A69146638C0B
:107E3000D70863E0F604638EE70C6369F70A054729
:107E40006380E70EFD5717E7FF1FA307F7C8370743
:107E50004000B7E700E023A0E71801000100B78663
:107E600000401306F0FC2381C60223A0E7106FF048
:107E70000FE2130720086382E7086362F702130723
:107E80001008E391E7FC378700408347670293F7C8
:107E9000C70B93E727002303F7026FF0CFEB13071D
:107EA00030086389E70213074008E39DE7F8378746
:107EB00000408347270393F7C70B93E72700230965
:107EC000F7026FF04FE9378700408347270393F7A6
:107ED0003707F5B7378700408347E70293F7C70BAB
:107EE00093E727002307F7026FF0EFE6378700409C
:107EF0008347E70293F73707F5B737870040834793
:107F0000A70293F7C70B93E727002305F7026FF04B
:107F10008FE4378700408347A70293F73707F5B709
:107F2000378700408347670293F73707ADB7179548
:107F300001001305652497700100E78060CD97E785
:107F4000FF1F23850794D5B3179501001305C5239B
:107F500097700100E780C0CB97E7FF1F2398079237
:107F600097E7FF1F938747B703C40700894763F369
:107F7000870009441374F40F6FF00FDE130700023B
:107F8000E392E7EC631B0B0A638FF5009307200273
:107F90006383F5081795010013058522977001008A
:107FA000E78020AF45B5179501001305A51E977012
:107FB0000100E780E0C50144179D0100130DCD1EAF
:107FC000A14CB387840083C507006A8505049770B8
:107FD0000100E78000ACE31694FF1785010013054C
:107FE000656D97700100E780A0C217E4FF1F03448E
:107FF000248A01E897E7FF1F238C0786014B6FF067
:10800000AFD58947E310F4E4854717E7FF1F230145
:10801000F7866FF04FD417E6FF1F0346568797E5A4
:10802000FF1F83C5C5861795010013056518977056
:108030000100E78000A66FF00FD26380F50693077A
:108040001002E399F5F497E5FF1F83C56584179542
:1080500001001305E51797700100E78080A397E7FB
:10806000FF1F23AB97B897E7FF1F9387A7A79443FA
:1080700083D7470017E7FF1F034727A717E6FF1F10
:108080002326D6801D4497E6FF1F2393F68097E7AB
:10809000FF1F2380E7806FF02FCC97D5FF1F83C58C
:1080A000257F179501001305251497700100E780BF
:1080B000409E97D7FF1F238D077A97D7FF1F2397DF
:1080C000077C6FF02FF92547638FE7C899463787FC
:1080D00000406394D70223008702B7E700E0B706A9
:1080E000400023A0D71801000100130600FC230163
:1080F000C70223A0D7106FF08FB99306100A639FB1
:10810000D70023008702B7E700E0B706400023A0AE
:10811000D71801000100130680FCD1BF9306A00907
:10812000E381D7FE9306400AE38DD7FC9306200235
:10813000639DD700B7E700E0B706400023A0D7183B
:108140000100010023008702F9B78546E384D7FECA
:1081500093070008E300FBFEB7E700E0B706400026
:1081600023A0D71801000100130620FC230087027A
:10817000BDBF17E7FF1F034737966302F71E63E78C
:10818000E70295476300F7109947630AF704B7863B
:10819000004023800602B7E700E03707400023A035
:1081A000E718010001001306A0FC75B99307F0055C
:1081B000630AF700930750096306F700930710025C
:1081C000E317F7FCB7E700E03707400023A0E71804
:1081D00001000100B7860040130620FC69B117EBCF
:1081E000FF1F034B6B8F930700045A8D63F46701E5
:1081F000130D000497E7FF1F938707A083AC0700C8
:108200001374FD0F2286E685268597600100E780BE
:10821000E07CB3078B40669417E7FF1F230EF78AB5
:1082200097E7FF1F23AA879CB7870040630C0B02C8
:108230002380A703B7E600E03706400023A0C61856
:108240000100010003C72702134707042381E70247
:1082500003C727021377C70F2381E70223A0C610A5
:108260006FF0EFA22380070237E700E0B706400077
:108270002320D71801000100130620FC2381C70228
:108280006FF0AFB9378700408347370097E6FF1F8D
:1082900083C6168693F70708D58FA301F700B706A4
:1082A0004000B7E700E023A0D71801000100130643
:1082B000A0FC35BD97E7FF1F93874795CA9783C7F3
:1082C000070093F7F70FC1CF97E7FF1F83C72796E4
:1082D000D9E717E7FF1F03473780930700026310B2
:1082E000F70883AD040017DDFF1F034D6D5A97DCBF
:1082F000FF1F83CCFC5917DBFF1F034B8B59E6870D
:108300006A87DA866E8697D5FF1F83C565561795EF
:1083100001001305E5EE97600100E780807797D7AD
:10832000FF1F23A1B77D97D7FF1F238FA77B97D769
:10833000FF1FA38B977B97D7FF1F2388677B97D758
:10834000FF1FA3868752B7E700E03707400023A04E
:10835000E71801000100B78600406FF04FA2B7E7B1
:1083600000E03707400023A0E71801000100B786AE
:10837000004015BD97E6FF1F83C6668B0547639CCB
:10838000E60429472381E70209472383E70223857F
:10839000E70297D7FF1FA38B077497E7FF1FA388F8
:1083A0000788B7870040A381070017D7FF1FA301E5
:1083B000077405472383E700B640264496440649E0
:1083C000F259625AD25A425BB25B225C925C025D05
:1083D000F24D6161828029472381E70209472383A7
:1083E000E7022385E7022387E7022389E70255B7DF
:1083F00017D7FF1FA30DF7466FE01FFF854717D75D
:10840000FF1F2305F75417D7FF1F2303F76017D764
:10841000FF1F2301F76C17D7FF1F230EF76A6FE0CA
:10842000BFFE854717D7FF1F2302F75217D7FF1F3D
:108430002300F75E17D7FF1F230EF76817D7FF1F1C
:10844000230BF76817D7FF1FA302075017D7FF1F8B
:10845000A300075C17D7FF1FA30E076697D7FF1F60
:10846000A38B07668280411106C697000000E78053
:1084700080FBB787004023800700130740FC23865A
:10848000E7001307C004A386E70017D7FF1F1307F1
:10849000E73F2398E70017D7FF1F13072743239AC7
:1084A000E70017D7FF1F1307A74E239CE70017D736
:1084B000FF1F1307275A239EE70029472381E7025E
:1084C00009472383E7022385E7022387E7022389FD
:1084D000E702A3810700930600F8A380D700930664
:1084E00090022380D700FD562383D7002381E70025
:1084F0009306000537E700E0230BD740B70640009E
:108500002320D71003C7170013671700A380E700C5
:10851000B24097D7FF1F239D075C41018280411124
:1085200006C697000000E78000F0B7870040238070
:108530000700130700FC2386E7003147A386E70006
:1085400017D7FF1F130787342398E70017D7FF1F9C
:108550001307C737239AE70017D7FF1F13074743AF
:10856000239CE70029472381E70209472383E70289
:108570002385E702A3810700930600F8A380D700B4
:10858000930690022380D700FD562383D7002381D2
:10859000E7009306000537E700E0230BD740B70656
:1085A00040002320D71003C7170013671700A380CC
:1085B000E700B24097D7FF1F239C075241018280FA
:1085C000F1679387072017D7FF1F232DF7508547A3
:1085D00017D7FF1F231AF750A14717D7FF1F2306EE
:1085E000F75097D7FF1FA382075097D7FF1F238FFE
:1085F000074E97D7FF1F238D072697D7FF1FA38806
:108600000726814717D5FF1F1305C526FD5517D629
:10861000FF1F1306E6262947B306F5002380B600A0
:10862000B306F600238006008507E397E7FE97D799
:10863000FF1FA384074A97D7FF1FA382074A97D734
:10864000FF1F238D074897D7FF1F2388074897D719
:10865000FF1F2387074897D7FF1FA381074897D796
:10866000FF1F238E0746814717D6FF1F13060659A3
:108670004147B306F600238006008507E39BE7FE2B
:10868000828017D7FF1F0347875A85476316F70075
:10869000170300006700E3E8170300006700E3DC4E
:1086A000411122C406C617D7FF1F03474758854705
:1086B0002E8613F4F50FAA856317F70417D5FF1F4D
:1086C0001305053197600100E780403197D7FF1F00
:1086D00023800734B787004023848702B7E600E091
:1086E0003706400023A0C6180100010003C7A702F7
:1086F0001377C70F2385E702B240224423A0C61098
:1087000001454101828017D5FF1F13052520976081
:108710000100E780A02C97D7FF1F23890722B78786
:10872000004023828702B7E600E03706400023A01E
:10873000C6180100010003C767021377C70F238320
:10874000E7025DBF411106C697000000E78080E7A1
:10875000B2404101170300006700E3F2411106C671
:1087600097F0FFFFE78080BF97D7FF1F83C7171ED3
:10877000A1CB97D5FF1F83C5851D89C917D5FF1FBD
:108780001305051D97E0FFFFE780C05397D7FF1F34
:10879000A38E071A97D7FF1F238A073437E700E015
:1087A000B70640002320D71801000100378600409B
:1087B0008347660293F7370F2303F6022320D7106F
:1087C000B2404101828041C9D9C597D7FF1F83C7F5
:1087D0002732D1C3011122CC4AC84EC656C25AC054
:1087E00006CE26CA52C42E89AA890144930A0004DF
:1087F000371B030063772403B3078940C207C18393
:10880000BE8463F4FA0093040004C204C180130A16
:108810001BD497D7FF1F83C767139DE37D1A631C83
:108820000A00F2406244D2444249B249224A924A82
:10883000024B0561828097F0FFFFE78020B2D1BF35
:10884000338589002694A685420497000000E780BE
:1088500060E5418045B7828097D7FF1F9387C74067
:1088600018429C4383D645000345070083C5C700D3
:10887000035646006396A50083D5E700638DD502B5
:10888000011106CE2386A7002397D700B705CF0096
:10889000DC4B9385757D05077D162EC223000100F4
:1088A0003AC42316C1002317D10099C30A858297C1
:1088B000F240056182808280DC4DDC4B81CFB7E7DE
:1088C0000400904503A38705914517D5FF1F034575
:1088D000E539028382806D713C083EC6B707E5002A
:1088E000232291103EC8AA843C0832852326111009
:1088F0003ECA23248110232021112E8997300000A5
:10890000E78080632A84979501009385E592177527
:1089100001001305657797600100E7808017A28545
:10892000179501001305C5A197600100E780601647
:10893000294597600100E780A01AB705CB00938511
:10894000757D680097100000E7800069A2856800C7
:1089500097300000E780A050014781467000CA852B
:10896000268597200000E780808C05CD2A84979586
:1089700001009385658C177501001305E5709760FC
:108980000100E7800011A285179501001305059CE1
:1089900097600100E780E00F294597600100E780BC
:1089A00020148320C1100324811083244110032943
:1089B00001105161828097D7FF1F9387E72A1842E1
:1089C0009C43797122D406D60348070083C8070167
:1089D0002A8483D64500035546006396080183D850
:1089E0002701638DD8022388070105072399D70043
:1089F0003708CC00DC4B1308787D3ACC1307F5FF21
:108A000042CA23080100231EE100231FD10099C799
:108A1000080832C62EC482973246A24522859700A6
:108A20000000E78080EBB2502254456182806D7176
:108A30003C083EC0B707E5003EC23C083EC42326C2
:108A400011102324811023229110231701002318D1
:108A5000010023190100231A0100231B010097B70D
:108A6000FF1F83D7E79999E3C167FD172316F1002C
:108A700097B7FF1F83D7E79891EB97D7FF1F93878F
:108A8000A71E9C439C43DC4783D7070017B4FF1FF6
:108A900013040497584C2317F10083574400484BA4
:108AA0002318F10031E1978501009385E57F177563
:108AB00001001305655D97600100E78080FD178563
:108AC00001001305A57F97600100E78080FC294520
:108AD00097600100E780C0008320C110032481104B
:108AE000832441105161828097B7FF1F83C7B791DC
:108AF00089EBB7E70400BC5782975C4C23AA0700B8
:108B0000E1BFFD1797B6FF1FA38FF68E035607012F
:108B1000834704014C470A85230BF100973000007E
:108B2000E780003197D7FF1F938707149C430147C5
:108B3000814688430A866C0097100000E780206F0A
:108B4000AA8429C1978501009385057617750100D0
:108B50001305855397600100E780A0F3A68517856C
:108B600001001305657697600100E78080F22945D2
:108B700097600100E780C0F6584CB7E70400BC5787
:108B8000484B9DBF97B7FF1F83C7F787F5D7B7E758
:108B90000400BC4F1044854517D5FF1F0345050D44
:108BA00082971DBF5C4EDC4BB9CFB1CD411122C4C1
:108BB000177501001305454D2E8497850100938597
:108BC000E56C06C697600100E780A0ECA2851785DA
:108BD00001001305257297600100E78080EB2945AD
:108BE00097600100E780C0EFB7E704002244B2407D
:108BF00003A3870517D5FF1F034545071306400646
:108C00009145410102838280411122C417A4FF1FB4
:108C10001304C47C1C4C06C689C7DC4399C34C486A
:108C20008297584CB7E70400BC57484B82975C4C7E
:108C3000B240224423AA07004101828017A7FF1FE8
:108C40001307C77B834707009306F00B850793F74D
:108C5000F70F63E9F60097A6FF1F2381F67A034515
:108C600007008280930700F8FDB7835745006386AD
:108C7000071001114AC817A9FF1F1309697852C4C8
:108C8000032AC90106CE22CC03274A0126CA4EC6B2
:108C900056C2F15735E31307D00DFD57636EC70475
:108CA000B7E9040083A709072A8413058600420553
:108CB0004181B284AE8A8297232AAA000325C90182
:108CC0005C49A9E7978501009385455A177501000E
:108CD0001305853B97600100E780A0DB1785010045
:108CE0001305856997600100E780A0DA2945976040
:108CF0000100E780E0DEDD57F2406244D2444249A1
:108D0000B249224A924A3E85056182809387440097
:108D1000B705CF002319F5009385757D31059710B0
:108D20000000E780602B0325C901834564003105FD
:108D300097300000E780A0120325C9012686D6855A
:108D4000310597300000E780A00E7146A2854A8564
:108D500097600100E78080C8504419CA83A789053D
:108D6000854517D5FF1F034565F08297814769B791
:108D700097000000E780E0CBD5BFFD573E8582809D
:108D8000411126C297A4FF1F93848467D84C22C444
:108D900037E404003C54484B06C68297DC4C03235E
:108DA000C4052244B240924423AA070017D5FF1FEE
:108DB0000345C5EB854541010283411126C297D485
:108DC000FF1F938464EA9C4006C622C44AC0D5C3F0
:108DD000DC43C5C35CC12300B5002A84978501002C
:108DE00093850544177501001305052A9760010056
:108DF000E78020CA294597600100E78060CE9C404B
:108E000023A4070023A2070097A7FF1F9387075DEE
:108E1000DC4FDC4B91C7295597000000E78000DF4D
:108E200097A7FF1F9387C75DDC4FDC4B89C797006F
:108E30000000E78020F537E904008327C90589454C
:108E400017D5FF1F034585E282978327C905914502
:108E500017D5FF1F034585E182979C4003A3470177
:108E60006309030022852244B24092440249410131
:108E70000283B2402244924402494101828001119E
:108E8000328506CE22CC26CA2E8497300000E78099
:108E9000A00AAA84978501009385C53B1775010038
:108EA0001305851E97600100E780A0BE03078400BC
:108EB0000356640083554400A686178501001305F8
:108EC000654597600100E780C0BC294597600100B7
:108ED000E78000C197A7FF1F83C7A750639D970036
:108EE000014597000000E78060D281450A85970020
:108EF0000000E780C0ECF2406244D2440561828009
:108F00006D7123248110232611102322911093F7D1
:108F100045002E84638707143C083EC0B707E50070
:108F20003EC23C083EC42317010023180100231948
:108F30000100231A0100231B010097A7FF1F83D7FD
:108F4000E74999E3C167FD172316F10097A7FF1FB3
:108F500083D7E74891EB97D7FF1F9387E7D09C43D0
:108F60009C43DC4783D7070017A7FF1F130707475A
:108F70002317F100544F835747002318F100DC4AB0
:108F8000A1E7978501009385253117750100130529
:108F9000A50F97600100E780C0AF1785010013059A
:108FA000E53197600100E780C0AE29459760010078
:108FB000E78000B3134544008320C11003248110CF
:108FC000832441105161828097A7FF1F83C7774197
:108FD0002555D9C3FD1717A6FF1FA304F64003D6D6
:108FE000060183470701CC460A85230BF100973021
:108FF0000000E780E0E397D7FF1F9387E7C69C4315
:1090000017A7FF1F1307873D978601009386062E3B
:1090100088430A866C0097100000E7804021AA84EC
:1090200051D99785010093852527177501001305F0
:10903000A50597600100E780C0A5A68517850100FA
:109040001305852897600100E780A0A42945976053
:109050000100E780E0A8268597000000E78000BBBC
:1090600091BF93F725009DC7B7E70400BC47414671
:10907000814528088297255597000000E78000B9B0
:1090800028089305F00F97000000E78040D31345B0
:1090900024001DB793F71500014599DF97000000E4
:1090A000E78020991345140001BF5C4D411106C6AD
:1090B00088C317D7FF1F2329F7BAB7E7040083A790
:1090C0000708170500001305E5E38297B24097D71C
:1090D000FF1F238DA7B8014541018280011133355F
:1090E000A000A307A100B7E7040083A7471706CE97
:1090F0001306F1008545130550308297F240056153
:1091000082808280411122C406C697D7FF1F83C781
:1091100067B7014489EF97B7FF1F83C7F71005446E
:1091200099E717B4FF1F0344241013441400228549
:1091300097000000E780C0FA178501001305C52ECF
:1091400009E4178501001305252F2244B24041018F
:10915000176301006700E393797122D4A30F010024
:1091600037E404008327841726D24AD006D6AA847F
:109170002E89130550309305F10132C6829732468D
:109180008347F10193150601C18185CB01452EC6A8
:1091900097000000E780C0F483274417B2454A8651
:1091A00026858297054597000000E78060F3B2505E
:1091B00022549254025945618280832744174A867B
:1091C00026858297EDB741119397050122C406C603
:1091D00026C2C1872E8463D40702B7E40400FC547E
:1091E00017A5FF1F0345C524829719C1BC54829758
:1091F0002165218DB240224492444101828093F73F
:1092000015008DC7B7E7040083A7471A17A6FF1FED
:109210001306062197D5FF1F938505A617A5FF1FE7
:1092200003450521829713451400E9B793F72500FC
:1092300099CFB7E70400BC4F13060064894517A512
:10924000FF1F0345E51E82971345240065B793F77A
:10925000850085CF97D7FF1F83C787A385E7B7E72B
:10926000040003A8871A1307401F97A7FF1F83C78F
:10927000271C814613064006994517D5FF1F035545
:10928000A5A0029813458400B5B793F745000145A2
:10929000B5D3B7E4040083A7041817D5FF1F0355FF
:1092A000A59E8297BC4C13060064914517A5FF1F2D
:1092B000034505188297134544002DBF97D7FF1F1C
:1092C00083D7879C6398A70217D7FF1F231FB79ADE
:1092D00017D7FF1F231CC79A17D7FF1F2319D79A29
:1092E0002E86178501001305A51BBE8517530100A7
:1092F0006700237A178501001305051C1763010019
:10930000670003910357450097D7FF1F83D7C7977F
:10931000631EF704C1674111F91722C417D7FF1F55
:109320002324F79637E4040097D7FF1F23A007965E
:1093300097D7FF1FA388079497D7FF1F238A079407
:109340007C4C06C6894517A5FF1F0345650E82970D
:109350007C4C914517A5FF1F0345850D829722443C
:10936000B240410117030000670003DA17850100CE
:109370001305851417630100670083897D159547E0
:1093800063E2A71C17870100130787080A053A95AF
:109390001C41011122CC06CEBA972E8482871785F4
:1093A00001001305E51197600100E7806086A1A226
:1093B00003C7250099476311F7022E859700000027
:1093C000E78080F48345640017850100130545108C
:1093D00097500100E780E06B97B7FF1F238607E4F3
:1093E00017850100130585107DBF03C7250095472C
:1093F0006319F702C16717D7FF1F0357E788F917EB
:1094000003D5A5006309F702B7E7040083A7C717D0
:109410008297178501001305650E97500100E780BC
:10942000207F854717B7FF1F2300F7E0178501004E
:109430001305450F8DBF97D7FF1F2397A78483D7A9
:10944000E50097D6FF1F2392F68483D7050197D6B0
:10945000FF1F239DF68283D7250197D6FF1F2398F0
:10946000F68297D7FF1FA38F0780631BE502B7E73C
:109470000400BC4F096613060690A14517A5FF1FFF
:10948000034505FB82970356E4008355A400178526
:1094900001001305E50797500100E780805F51B791
:1094A0009307700F2316F100B7E7040083A7870D19
:1094B00017A6FF1F0346C6F76C0082974DF9854734
:1094C00017C7FF1FA300F77C5DB7178501001305C1
:1094D0002506D1BD83C5250091476392F502178506
:1094E00001001305650697500100E7806072970040
:1094F0000000E78060C1F2406244056182809947C4
:109500006392F502228597000000E780E0DF834543
:109510006400178501001305A5FB97500100E78043
:109520004057D1BF9547639AF50083471400E1F394
:109530001785010013058503BDB5178501001305C7
:109540006503E1BF82803757315F97A7FF1F93877D
:1095500067EF130777D598C39356C50017870100A7
:109560001307C7F0BA9683C5060093568500BD8AD7
:10957000BA9603C6060093564500BD8A3D89BA9641
:109580002A9783C606000347070023840700238326
:10959000D700A383E7002382B700A382C70097A761
:1095A000FF1F938727EB2383B700A383C700238480
:1095B000D700A384E7008280411106C6970000000F
:1095C000E780A0F8B7E7040083A7871417A6FF1F5A
:1095D000130646E7D54501458297B2404D4697A50B
:1095E000FF1F938525E71305703041011703000025
:1095F0006700C3B661712324811A37E4040083270E
:1096000004082326111A2322911A2320211B232E1A
:10961000311917050000130545BB829717A9FF1FD5
:10962000130909E1994785442300A900231CF1008F
:1096300097850100938585E2930740061775010021
:10964000130585A4231CF1082308910097C9FF1F67
:109650009389290E97500100E780A04383D5090024
:1096600017850100130585DE97500100E7806042F1
:10967000294597500100E780A04603D50900896974
:1096800097000000E78060EC8327441710088545A9
:109690001305503082978327441717A6FF1F130620
:1096A00066DBCD451305703082978327441717A6D4
:1096B000FF1F130626D8B545130560308297832710
:1096C00044173008894513051031829783274417C2
:1096D00030098945130520318297832744159385E6
:1096E00009900D458297832744159385099011456C
:1096F0008297A30591002306910002CD2308010063
:10970000230C01008327841630099145130570400E
:109710008297832784161306B10085451305004000
:109720008297832784167000854513051040829721
:1097300083278416300885451305204082978327A8
:109740008416100885451305504082978327041519
:109750007D558297832744137D5582977D5597A029
:10976000FFFFE78080F28327440C829797A0FFFFDA
:10977000E780E0CD8327841417A6FF1F130686CC4D
:10978000D5450145829789471306700F8145280901
:109790002306F1009790FFFFE78060978D4713063F
:1097A000000881452808230CF1089790FFFFE78007
:1097B00000969147230CF100976701009387477E3D
:1097C000984383C747003AC8230AF10097D0FFFFA8
:1097D000E78040B070008545054597A0FFFFE78012
:1097E000E0F130099305700F094597A0FFFFE7806E
:1097F000E0F03008930500080D4597A0FFFFE780D3
:10980000E0EF10089545114597A0FFFFE78000EFB6
:10981000C16717C7FF1F13072747F9171CC3232268
:10982000070017A5FF1F130565C097A0FFFFE7807E
:10983000C0EB8327C41D17C5FF1F1305654382971F
:109840003C4803450900854582978320C11A0324BB
:10985000811A8324411A0329011A8329C1195D61E0
:109860008280C16717C8FF1F03580842F9176301B8
:10987000F8083DCDB5CD011126CAB7E4040083A791
:10988000841222CC2E862315B10006CE2A840147ED
:109890008146ED45428582972AC611ED1785010064
:1098A000130505BE97500100E7808036F240624400
:1098B000D24405618280FC440356A100A2858297B0
:1098C0002C0017C5FF1F0355253C97A0FFFFE7801D
:1098D00080EE69DD178501001305C5BB97500100B7
:1098E000E780003383A7C412ED45280082977DBF2F
:1098F00082800DC5854717A7FF1FA302F7B497A75E
:10990000FF1F238F07B2354697A5FF1F938585B2AA
:1099100013056030170300006700438497A7FF1FFB
:10992000A38F07B0E9BF97C7FF1F83C76736A9EFAB
:10993000C16717C7FF1F03572735F9176306F704D9
:109940004111854722C417C7FF1F2303F73437E4AB
:1099500004007C4C06C6A14517A5FF1F034545AD75
:1099600082970323841A2244B24097A7FF1F83C71C
:1099700027AC17C5FF1F035525311307401F81462C
:10998000314699454101028382806D712324811003
:109990002326111023229110328401CD8947630AB6
:1099A000F5028320C11003248110832441105161EA
:1099B0008280178501001305A5BCAE849750010075
:1099C000E7800025A285268597C0FFFFE78020B0AD
:1099D000C9BFB7E70400FC4728008297178501003C
:1099E0001305C5BA97500100E780802283478100A4
:1099F00039C41307000B6380E7021387A7051377A9
:109A0000F70F8D4663EDE602A285280097C0FFFFA1
:109A1000E780E01F79B78547E3F587F88345910034
:109A20001775010013058597B335B00097A7FF1F81
:109A3000238CB76697500100E780A0059DB70347C8
:109A40009100A207D98F35671307D7556385E708BB
:109A50006368F7022D671307B7556387E706316719
:109A60001307C755638AE70429671307A75563944B
:109A7000E702A285280097C0FFFFE780405815B78E
:109A800039679306E7656381D70863E9F600130732
:109A9000E7556384E706A28528003DB73D67930636
:109AA000F755638AD7061307F766E396E7FE97C074
:109AB000FFFFE780C070F5B50146A285280097C07A
:109AC000FFFFE7806040F1BDA285280097C0FFFF3F
:109AD000E7802051F9B58947E3F587EC970000004E
:109AE000E780A0E49305E4FFC205C1811305A1004E
:109AF0009790FFFFE780C06E6DB5A285280097C0E4
:109B0000FFFFE780C05071BDA285280097C0FFFF0E
:109B1000E780805B79B597C0FFFFE780006451B5AF
:109B2000C16717C5FF1F03552516F9176307F50011
:109B3000B7E7040003A3C71702838280854717C7CE
:109B4000FF1F2301F714014517F3FFFF6700435977
:109B50001783FFFFE70203572A8408452E89B2893D
:109B600019C900C1971500009385A5866105973036
:109B70000100E780200581447D5A97100000E780AE
:109B8000E03963C7A404814497100000E780003ADD
:109B900063C8A40497C7FF1F9387C70F9C43DC4784
:109BA000B307F94091872302F400638309048327F4
:109BB000C900B307F4409587A302F4001C4C89C781
:109BC0009C4799C3228582971783FFFF6700C35282
:109BD0005C44139714008504BA972390470171BF22
:109BE0001C48139714008504BA972390070069BF97
:109BF000832789000547B307F4409587A302F40043
:109C000083570400638EE7028DC309476384E7042A
:109C10000D47E395E7FA978701009387E7E91CCCA6
:109C200097870100938747EA11A8978701009387D8
:109C300027B01CCC97870100938787B05CC8BDBF55
:109C4000978701009387C79B1CCC97870100938758
:109C5000279CEDB7978701009387C7EA1CCC9787AD
:109C60000100938727EBD9BF95E51783FFFFE70234
:109C70000347004618448347940075839D8B631700
:109C8000F70097100000E78060B448C41783FFFF17
:109C90006700234782801783FFFFE702A3421389EF
:109CA0003500C16442094111AA890144F1141359D4
:109CB0000901054A2EC697100000E7802026B2450C
:109CC0006348A400014541011783FFFF6700C342B9
:109CD00083A7090013171400BA9783D70700638876
:109CE000B7006394970063742A010504E1B7054542
:109CF000D9BF1783FFFFE702033CAA892E89328B65
:109D0000B6843A8ABE8A97A00000E780C0FE71C977
:109D1000268597200000E780C00C8D4763E7A700E9
:109D20007D551783FFFF6700833C83DB440097105A
:109D30000000E780A0242A8497100000E7804025D7
:109D40009307740031443305850263CDA702971051
:109D50000000E780A02297100000E78020222A84DC
:109D600097100000E780C022930774003144330548
:109D7000850263C3A70497100000E78020209307A3
:109D8000450029A897100000E78080203305850250
:109D90001307F0179307C017E35FA7FA2D55E3C227
:109DA00077F963040B02D6865286A6854A859720EA
:109DB0000100E780C0BDB5B797100000E780401DE7
:109DC000330585029307C5FFD1BF8327490013855B
:109DD000C90083D5270097000000E78000EC61F5FB
:109DE00081B769553DBF97C7FF1F2397A7EA97C75C
:109DF000FF1F938727EA904381470C463307F500FE
:109E0000420741836393B70082805446139847000A
:109E10008507C2962390E600D5B797C7FF1F9387A3
:109E200067E79C4303C58700828017C5FF1F035562
:109E3000A5E682801783FFFFE702632AC1671387C5
:109E4000D7FF630BE502636AA700F1176300F50211
:109E500001451783FFFF6700C32A1387E7FF6302EB
:109E6000E502FD171D8D13351500E5B7975000006D
:109E7000E780602A7D15C5BF97500000E780E0FEAF
:109E8000D5BF97500000E78000FDEDB71783FFFFB7
:109E9000E702E3244111AA8401442EC69710000072
:109EA000E780C008B2456348A4000145410117831B
:109EB000FFFF670003259C48131514003E95835748
:109EC0000500E385B7FE0504C9BF03485500814678
:109ED00093F7F60F63E5070181473E858280584579
:109EE00093975600BA9703D727006316B70003D796
:109EF0000700E304C7FE8506E1BF8346450001472E
:109F00009377F70F63E4D700814711A81C45131618
:109F100057000507B29703D60700E313B6FE3E8548
:109F200082801783FFFFE702E31993170501C187BA
:109F300097CAFF1F938A0AD6635BF00883A70A00BB
:109F4000C0479C4703570400198D4205418163684F
:109F5000F500014422851783FFFF6700E31912050E
:109F60002A94CDBFDC4713944900014A3E948347AD
:109F700044006341FA02014A834754006349FA02EC
:109F80008509C20993D9090183A70A009847E3EB21
:109F9000E9FCC1B71C4413195A00A6853E994A85AD
:109FA00097000000E780C0EE05E1050AC9B75C44F0
:109FB00013195A00A6853E994A8597000000E7804C
:109FC00020ED19E1050A4DBFE30C09FA61B7AA8437
:109FD00081495DBF1783FFFFE70263101C452A8498
:109FE00081E79307C5001CC51C44231204001CC054
:109FF0009307F00F63EDB70093F5F50F22859720D7
:10A000000000E780C0E51783FFFF6700830F93948C
:10A010000501C167C18063F9F500A68522859720F7
:10A020000000E780E0E8C5B7C18193F5F50F228510
:10A0300097200000E780A0E2A685228597200000F7
:10A04000E780E0E3C9B797C7FF1F9387A7C488439A
:10A0500082801C4599C797C7FF1F23ADA7C2014542
:10A0600082807D55828097C7FF1F9387A7C2984340
:10A0700083474500484792073E9582801783FFFF3C
:10A08000E702E305617100451C183EC6B707800171
:10A090003EC81C183ECA8357440002CE02D002CCF0
:10A0A000231EF100834784002A8902D22301F10292
:10A0B0003C083ED402D697000000E78000FB83579F
:10A0C00005002316F10297500000E78000C823071F
:10A0D000A1025C4003556400F18313F71700834726
:10A0E000F10252055181F99BD98FA307F102971014
:10A0F0000100E780207939CDAA840355050097A097
:10A100000000E78020C083D704002AD26800231C07
:10A11000F10083D72400231DF1001C4803D647001B
:10A120008C4397200000E780A0D08347B400CA8604
:10A1300017760100130646468117A305F4006C004C
:10A14000481097200100E78080845D611783FFFF3E
:10A15000670023FB2155D5BF1C45B1CF03C5A70020
:10A16000894613576500630BD7028D46630ED702ED
:10A1700085466300D702130740063305E50203C78F
:10A18000B700418B15CB83C7B700BD8B3355F54066
:10A1900082801375F5031307803EC5B709671375F1
:10A1A000F50313070771D1BF372709001375F503AE
:10A1B0001307077CD9B7014582801783FFFFE702A9
:10A1C00003F203A98500630C09048347B900AE8438
:10A1D00093F7070E85C303459900930520030D816E
:10A1E0000505B305B5028844610597300100E78095
:10A1F00080AD35A02E8597000000E78020F62A84E8
:10A2000019CD97000000E780605C8325C900B30783
:10A21000B54063FA87002E94B305A440E9F517838F
:10A22000FFFF670003EE85457DBF1783FFFFE70251
:10A2300003EB2A8403D50500011132C636C43AC2A5
:10A240002EC002CA02CC02CE97A00000E78080ABED
:10A2500082452ACA22852ECC97000000E780E0E0E4
:10A2600003570500231EE10097500000E780E0AD92
:10A27000A24632469247230FA10036874C08B28689
:10A280002285014697000000E780E0A6056117835C
:10A29000FFFF670003E71783FFFFE70243E46171F5
:10A2A0001C183EC6B70780013EC81C183ECA3C08B1
:10A2B00000453ED4AA8402CC02CE02D002D202D6FD
:10A2C00097000000E78060DA8357050035592316B0
:10A2D000F10297500000E78040A72307A10209C4BC
:10A2E0008357440081EB21594A855D611783FFFF45
:10A2F000670023E103556400520551819710010066
:10A30000E78040582A8965D18347B40093F7070E48
:10A3100099C71305840197300100E780009D83579A
:10A320004400231EF100834784002301F1025C40B6
:10A3300003550900D98313F7070883471102231C2B
:10A34000A10093F7F707D98FA300F10283572900E3
:10A35000231DF1005C40F18313F717008347F102DE
:10A36000F99BD98FA307F10297A00000E78080999D
:10A370002AD235D983479400680013975700834742
:10A38000B400FD8BD98FA305F4001C4803D6470009
:10A390008C4397200000E780A0A9A68717770100CB
:10A3A0001307871F740005464C1026859700000090
:10A3B000E78060942A890DD98347B400A685FD8B78
:10A3C000A305F40097000000E78060DF31BF17832A
:10A3D000FFFFE702C3D0832485FE2A84411126852E
:10A3E00097000000E78080D7834734FF93F7070E7C
:10A3F0008DCB2AC6268597000000E78060C809CD6E
:10A40000834734FFB245FD8BA309F4FE91C5228535
:10A4100097300100E780208B41011783FFFF670021
:10A4200043CE7DD98327C4FF2685829775F5834760
:10A4300034FF93F7070E91C7228597300100E7801C
:10A44000C08A032584FE97000000E78000E5E9B795
:10A450001783FFFFE702A3C59C4141112A8903C767
:10A46000070089472E84935667006380F6040D46E3
:10A470006388C6049307F0076304F7022E859720CC
:10A480000000E78060ABAA848149C16B130C4900CE
:10A4900097C7FF1F938707809C43984763E4E904AD
:10A4A00041011783FFFF670043C403D74500854779
:10A4B000E3F8E7FE2E8597200000E78040ADE1B786
:10A4C00003D74500E3FEE7FC2E8597200000E780D8
:10A4D000A0A6AA84228597200000E78000A8C204D5
:10A4E000C98C5DB7DC470355A900139A49003E9A11
:10A4F00093170501C187635DF00083570A006397D6
:10A50000A70263E774038327CA00034D5A002DA0F6
:10A51000A1672167A98F1307F7EFE374F7FE63972D
:10A52000090097000000E780209161FD85098DB743
:10A5300083278A00034D4A00835DA9000357690001
:10A54000216A138BC7003AC6814A33CA4D01631E84
:10A550005D0197B7FF1F938767749C43E1DBA28679
:10A560006286814526858297D1B7A1679387F7EFE9
:10A57000930C4BFF63F24703B2455A8597F0FFFFF8
:10A58000E780A0710DC103278B00104709CE10434F
:10A590006382C4023107D5BFEE856685970000004F
:10A5A000E780008F71F993861A0093FAF60F130B68
:10A5B0000B0271BF835644005C43E3E9F6F6228543
:10A5C0003AC697200000E7802081A1679387D704CF
:10A5D0002A8A035D4400324763E897008347D90025
:10A5E00093E707F8A306F9001C4766852286E285F3
:10A5F0008297C1670844FD17337AFA00529508C064
:10A600002312A40125B797B7FF1F9387A768984324
:10A61000814715C31447814763FFD50093974500D1
:10A620004C47BE9519C903C7550081476375E600BD
:10A63000DC451606B2973E85828003C745008147F8
:10A64000E37BE6FE16069C45F5B71783FFFFE7029E
:10A6500063A7AA892E8A814497BAFF1F938A8A63C7
:10A6600083A70A00984763E6E4001783FFFF6700AB
:10A67000A3A8DC471394440001493E9413BB140083
:10A6800083474400634BF900014913BB140083471F
:10A690005400634FF9008504E1B70844931759004B
:10A6A0005287DA860146A2853E9582990509C9BF7F
:10A6B0004844931759005287DA860546A2853E958D
:10A6C00082990509E9B71783FFFFE70243A1814596
:10A6D00017F5FFFF1305054897B7FF1F239E075A7D
:10A6E00097000000E780A0F61783FFFF670063A1D3
:10A6F00097B7FF1F9387075A9C4395C31783FFFFA4
:10A70000E702E39D814517F5FFFF1305A544970078
:10A710000000E780C0F31783FFFF6700839E8280FD
:10A720001783FFFFE702039A37E4040083278412AC
:10A7300041112315E100AE893289368A3A86814675
:10A740000147ED45AA8482972AC621C90356A10074
:10A75000D28597400100E78060288327C413CE8507
:10A7600026858297058905C98327440D2314210175
:10A7700001462C00268582972A8401C9B7E7040088
:10A7800083A7C712ED4528008297228541011783D0
:10A79000FFFF670063964944D5B76554FDB75C4138
:10A7A000FD175CC182801783FFFFE7024393B7E781
:10A7B0000400FC5F829795473305F50281450D81C2
:10A7C0001783FFFF6700E3931783FFFFE7022391DF
:10A7D000B7E70400FC5F829795473305F5020D81CA
:10A7E0001783FFFF6700E3911783FFFFE702238FC3
:10A7F000B7E7040083A7870B0355050082971783EB
:10A80000FFFF670003901783FFFFE702438D0355A7
:10A8100005003287AE861796FF1F0356C6C997B547
:10A82000FF1F9385E54797000000E780A0EF17839F
:10A83000FFFF6700038D1783FFFFE702438AB7E737
:10A84000040083A7C71782971783FFFF6700638BF6
:10A850001783FFFFE702A388B7E7040083A78713E6
:10A8600097B5FF1F9385C543829701451783FFFF67
:10A87000670023891783FFFFE7026386B7E70400B9
:10A8800083A7C71F81451795FF1F0355C5BE829734
:10A890001783FFFF6700E3861783FFFFE702238428
:10A8A000B7E7040083A7871397B5FF1F938545403B
:10A8B000829701451783FFFF6700A3841783FFFF7B
:10A8C000E702E381B7E7040083A7C71F8145179517
:10A8D000FF1F035545C082971783FFFF6700638200
:10A8E0001773FFFFE702A37F2E8597800000E780A4
:10A8F00080B397800000E78080F01783FFFF670038
:10A9000043801773FFFFE702837D97800000E78095
:10A9100080FA1773FFFF6700C37E5C49E1175CC9CB
:10A920005CC583572501A1072319F500835705014D
:10A93000A1072318F5008280F1473305F50297B788
:10A94000FF1F9387E7389C433E9582808D476315B0
:10A95000F60803D74600854763F0E7081773FFFF43
:10A96000E702E377368536842E8997100000E7806A
:10A97000A05C29C98357440093140501C18063E397
:10A980009704228597100000E780005BFD142312D6
:10A9900094009307A0026300F5029307B0026307D7
:10A9A000F50293079002631FF500228597000100CE
:10A9B000E780608901A80146CA85228597A000002A
:10A9C000E78000B41773FFFF6700A3732285971019
:10A9D0000000E7806007FDB7828097B6FF1F93866F
:10A9E000662F9C42014599CF9843D44217B6FF1F6A
:10A9F0002322E62E6396D70097B6FF1F23AEE62CE0
:10AA00001385C7FE82801773FFFFE702436D97002F
:10AA10000000E780A04B7144330585029145979073
:10AA20000000E780C0EC11E565551773FFFF670074
:10AA3000436D97B7FF1F23ABA72897000000E7805F
:10AA4000E04833058502914597900000E78020EAB1
:10AA500061DD97B7FF1F23ADA72697000000E780B1
:10AA6000E04697B7FF1F239DA72497000000E780CB
:10AA7000E04597B7FF1F2396A72497770100938798
:10AA8000E7B617B7FF1F2321F72497070000938726
:10AA900007E917B7FF1F2327F722014579B7177377
:10AAA000FFFFE702C363AA8517B5FF1F1305452102
:10AAB00097100000E780605F1773FFFF6700636413
:10AAC0001773FFFFE702A36197000000E78060FDB6
:10AAD00097100000E780E05E97B7FF1F9387871FFE
:10AAE0009C4391CF1387C7FE19CB83D5C7FF17B5FA
:10AAF000FF1F1305A51E97200100E780C01C1773D8
:10AB0000FFFF670003601773FFFFE702435D9700D5
:10AB10000000E780C0EC09CD834785002A8493F7C5
:10AB2000070499EB0355E50097000000E78080F9E2
:10AB30001773FFFF6700E35C8347C500930445017B
:10AB400017B9FF1F1309091985E3832709005CC999
:10AB500097B7FF1F23A0971883274900F1FB97B7EA
:10AB6000FF1F23AB9716E9B7FD172306F500610514
:10AB700097800000E78060DA8307840063CB0704D6
:10AB80008347840093E707F82304F400B7E7040041
:10AB90009C5F82974205A94741813375F50283473F
:10ABA000840093F707FCC98F2304F4008347D40083
:10ABB0003E951C402318A40089CF984319CB8347A6
:10ABC000C4005040814585073305F50242054181A7
:10ABD0000297832709005CC897B7FF1F23AC970E25
:10ABE0008327490089E797B7FF1F23A7970E83475D
:10ABF000C4009DDF8355040117B5FF1F1305050E23
:10AC000097200100E780200C25B71773FFFFE702AC
:10AC1000034D97B7FF1F9387A7319C470144858356
:10AC2000858B85E3AE84B2853A8697100000E78075
:10AC3000204F2A8419C597100000E7806045829450
:10AC400008CC22851773FFFF6700A34B1773FFFF24
:10AC5000E702434741112E8932C6AA8997000000B6
:10AC6000E780C031324713060502CA869705000007
:10AC70009385C5CC17B5FF1F130585049700000009
:10AC8000E780E0F82A8425C99304C50097000000F6
:10AC9000E780E0411946AA85268597100000E780E5
:10ACA00020198545268597100000E7800015177547
:10ACB0000100130565914E95834505002685971083
:10ACC0000000E780C0195C4831468145A1075CC897
:10ACD0005CC483572401E1172319F400835704014E
:10ACE000E1172318F4001C4C3E859770FFFFE780A6
:10ACF0000042A3042501228541011773FFFF67006D
:10AD0000A33F1773FFFFE702833D4111AA842EC6BC
:10AD100032C497100000E780003A004DB245224649
:10AD2000834784000CC050C093F7F70393E70704F0
:10AD30002304F40023180400268597100000E78000
:10AD4000203583479400A9462317A40013D7370062
:10AD500005073307D7029D8B85072306F400A3065A
:10AD6000E40083C70401D8488507230FF7FE17B70F
:10AD7000FF1F130727F65843232A040093074401B3
:10AD800029E317B7FF1F2329F7F417B7FF1F232362
:10AD9000F7F417B4FF1F130464F422859720010011
:10ADA000E780A0E41C44858B5D8D19E581452285F3
:10ADB00097200100E78020F141011773FFFF670032
:10ADC00043341CC317B7FF1F2328F7F0D9B71773F5
:10ADD000FFFFE702C33097050000938565B7014583
:10ADE00097000000E78000B001451773FFFF670080
:10ADF00043311773FFFFE702832E97000000E780BF
:10AE000080B01773FFFF6700C32F8347C500A5E31A
:10AE10001773FFFFE702A32C2A840355E500970070
:10AE20000000E78000C821C18347840093F7F7FB47
:10AE30002304F4001C4091C7DC4381C74C4001450A
:10AE4000829797000000E78080B917B5FF1F1305B0
:10AE5000E5E897200100E78040E90355E40097000A
:10AE60000000E78020C61773FFFF670083298280F8
:10AE70001773FFFFE702A32697B7FF1F938787E5A6
:10AE800097050000938565C817B5FF1F130505E5F5
:10AE900023A0070023A2070097200100E78080D2AB
:10AEA0001773FFFF6700E3251C4D91CFDC4381CF73
:10AEB0001773FFFFE702A3228345070082971773EA
:10AEC000FFFF67000324828097B7FF1F938747E344
:10AED0009C4303C50700828097B7FF1F938747E213
:10AEE0009C4303C51700828097B7FF1F938747E1F4
:10AEF0009C4303C52700828097B7FF1F938747E0D5
:10AF00009C4303C54700828097B7FF1F938747DFA5
:10AF10009C4303C53700828097B7FF1F938747DEA6
:10AF20009C4303C55700828097B7FF1F938747DD77
:10AF30009C4303C56700828097B7FF1F938747DC58
:10AF40009C4303C57700828097B7FF1F938747DB39
:10AF50009C4303C58700828097B7FF1F938747DA1A
:10AF60009C4303C59700828097B7FF1F938747D9FB
:10AF70009C4303C5A700828097B7FF1F938747D8DC
:10AF80009C4303C5B70011E11D45828097B7FF1FA1
:10AF9000938707D79C4303C5C700828097B7FF1FDD
:10AFA000938707D69C4303C5D700828097B7FF1FBE
:10AFB000938707D59C4303C5E700828097B7FF1F9F
:10AFC000938707D49C4303D50701828097B7FF1F5F
:10AFD000938707D39C4303C52701828097B7FF1F40
:10AFE000938707D29C4303D54701828097B7FF1F01
:10AFF000938707D19C4303D56701828097B7FF1FD2
:10B00000938707D09C4303D58701828097B7FF1FA2
:10B01000938707CF9C4303C5A701828097B7FF1F83
:10B02000938707CE9C4303C5B701828097B7FF1F64
:10B03000938707CD9C4303C5C701828097B7FF1F45
:10B04000938707CC9C4303C5D701828097B7FF1F26
:10B05000938707CB9C438857828097B7FF1F9387BE
:10B0600027CA9C4303D5C702828097B7FF1F9387E7
:10B0700027C99C4303D5E70219E11305800C8280A0
:10B0800097B7FF1F9387C7C79C4303C507038280F9
:10B0900097B7FF1F9387C7C69C43C85B828097B74B
:10B0A000FF1F938767C58843828097B7FF1F9387E9
:10B0B000E7C48843828019E17D558280F5DE98429D
:10B0C00065DFFDD917B7FF1F130787E61847AA8763
:10B0D0007155058B631D072403C507001547E37DE4
:10B0E000A7FC03C737001305F0057D171377F70F8B
:10B0F000E364E5FC03C35700E30003FC83C8670077
:10B10000E38C08FA03C77700494579171377F70FDF
:10B11000E364E5FA03C7A70011481305F7FF1375A9
:10B12000F50FE36BA8F803CE97000D481305FEFF5B
:10B130001375F50FE362A8F803C8B70063090800A8
:10B1400065181378F80F1305600DE36705F703C55D
:10B15000C700794879151375F50FE36FA8F403C894
:10B16000D7000D457D181378F80FE36705F503D870
:10B170000701930E40175118420813580801E3EDD8
:10B180000EF303C8E7007D181378F80FE36605F3A4
:10B1900003C827017D181378F80FE36F05F103C882
:10B1A0008700C54E75181378F80FE3E70EF103D842
:10B1B0006701856E938EBEE06D1842081358080132
:10B1C000E3EC0EEF03D847016D184208135808014D
:10B1D000E3E40EEF03D887017918420813580801F9
:10B1E000E36C05ED03C8A7017D181378F80FE3653C
:10B1F00005ED03C5B7011D487D151375F50FE36D0A
:10B20000A8EA03C5D701714879151375F50FE365F1
:10B21000A8EA03D5E7011308E00F7D154205418137
:10B22000E36CA8E803C50702494879151375F50FC3
:10B23000E364A8E8C85301C937C834005915130896
:10B2400058BFE36BA8E603A8870237C5340013058F
:10B2500055BF5918E36205E717B5FF1F2320C5AA9C
:10B2600003C6050117B5FF1F232CF5A80545E37597
:10B27000C5E403D82501D04933760603E31E06E270
:10B2800003C61501E30A06E217B6FF1F2326B6A67A
:10B2900083C5270001466387A50003C61700F14553
:10B2A0003306B60283C707039305C00272971A07D5
:10B2B0001307C70516031A9796084697B387B70270
:10B2C00041553E973297420741836362E806177300
:10B2D000FFFFE702C3E0368597800000E780406CFF
:10B2E00097000100E780C04B2A8497A00000E78008
:10B2F000205E2A9497F00000E780002A2A94979015
:10B300000000E78040852A9497F0FFFFE780E06F18
:10B310002A9497400000E78000972A9497700000D5
:10B32000E78040A022951773FFFF670083DD8280CE
:10B330001773FFFFE702A3DA4111A307A10097A04B
:10B340000000E78040C99305F100170500001305D0
:10B35000E5B597F0FFFFE780802F014541011773A6
:10B36000FFFF670003DA1773FFFFE702C3D417B4C8
:10B37000FF1F1304E4BB0328840079599368180065
:10B3800097B4FF1F23AA14BB137818006310080298
:10B39000BA84BE89368B328A2E89AA8A97F0FFFF3B
:10B3A000E780E0A77D15269519E531594A85177381
:10B3B000FFFF6700C3D397F0FFFFE78040A67D152E
:10B3C0002695A167E353F5FE97B7FF1F938707ED17
:10B3D00098433E8C814B01CB014597F00000E780FC
:10B3E000C047933B15004A85DA865686D2859790EA
:10B3F0000000E78060512A8911CD1C44F99B17B7E2
:10B40000FF1F232BF7B283270C00CDD3E3800BFA69
:10B41000829769BF268597B7FF1F23AD07B097F0C6
:10B42000FFFFE780809C4146CE8517B5FF1F1305BF
:10B43000A5B997300100E780605A97D00000E780F7
:10B44000E09C0325040B97D00000E780A0A00545F1
:10B4500097D00000E780A0A7054597000000E7808F
:10B4600060EDA9B797B7FF1F938787AC9C47858B83
:10B47000EDC71773FFFFE70283C617B5FF1F13055C
:10B48000E5B297B7FF1F23A507AA97B7FF1F23A30E
:10B4900007AA97B7FF1F23A107AA97200100E780FB
:10B4A000C08497500000E78080F997100100E78082
:10B4B000405097100100E780405697B7FF1F9387D1
:10B4C000A7A59C4391C7054597800000E780E0232E
:10B4D00097B7FF1F9387078E9C4399C741657D15DA
:10B4E00097700000E780E0A597F00000E7808041BA
:10B4F00097D00000E780209397B7FF1F938707B886
:10B500009C43139717016356070097F00000E780EC
:10B51000A0B097B7FF1F23A907AA97B7FF1F23A7BC
:10B5200007AA97B7FF1F23A507AA97B7FF1F23A353
:10B5300007AA97000000E780008C97000000E780D2
:10B54000A07597F0FFFFE780401897F00000E780B4
:10B55000E0D91773FFFF6700C3BA828097B7FF1F58
:10B560009387079D8843828097B7FF1F9387479CE7
:10B57000C8438280B7E7B0009387075063E1A70212
:10B5800097B7FF1F9387C79AD843FD576367E500B6
:10B5900097B7FF1F23A0A79A81473E858280B9579E
:10B5A000EDBF1773FFFFE70283B397800000E780CA
:10B5B000607597800000E780C0771773FFFF670012
:10B5C00043B41773FFFFE702E3AF2A849304140226
:10B5D00001112E85B289A685214636C63A89973053
:10B5E0000100E780403D0DE9B24638082686CE8549
:10B5F0001305940497500000E780604121462C0811
:10B600004A8597300100E780003B1335150005613E
:10B610001773FFFF670043AE0145D5BF1773FFFFE8
:10B62000E702E3AB9305450617A5FF1F1305856DDC
:10B6300097100100E78020691773FFFF670063AC74
:10B640001773FFFFE702A3A941112EC697F0FFFF72
:10B65000E780C017B24588C141011773FFFF67003B
:10B6600043AA1773FFFFE702E3A5AA842E849780FD
:10B670000000E780006CAA898545228597000000BC
:10B68000E780E07D83C7E4011389940899E3138977
:10B690000403CE85228597000000E780407C214688
:10B6A00093051902228597000000E780607897B71C
:10B6B000FF1F9387E7878C43228597100000E78060
:10B6C000C082214693858402228597000000E7808E
:10B6D00020761773FFFF670023A21773FFFFE702AF
:10B6E000839D397197F00000E780E0B49305400630
:10B6F00061E997800000E78000606302051497A766
:10B70000FF1F83C7E76113B7170097A6FF1F2389A1
:10B71000E660014499CFC16417B9FF1F130949813D
:10B720009309400EFD1497000000E78020836342D8
:10B73000A40A97F0FFFFE78060094169B729090073
:10B74000096AFD7A2A8B81447D199389F97B130A52
:10B750000A71938A8AC797000000E780208063D728
:10B76000A4041304400EB387840217A7FF1F130716
:10B77000277C0324070B3E948357C4016382270B65
:10B7800018403307EB4063EAE9008347440085072C
:10B79000B3874703D6976365F70801468145094596
:10B7A00097F0FFFFE780C04AAA8B29E59740000089
:10B7B000E780808385476317F50689659385057162
:10B7C00017A5FF1F1305055497100100E780A04F30
:10B7D00095A0B30734030327090BBA9703D7C70112
:10B7E0006308970003C75700A38207002382E7007E
:10B7F000050415BF9305C500228597000000E7806A
:10B8000080E65E85228697650100938525DD97F0A9
:10B81000FFFFE780404F5E8597100000E780608A59
:10B82000850415BF97A7FF1F938787709C478D835B
:10B83000858BC1F721611773FFFF6700438B0146BA
:10B840008545094502D002D202D402D697F0FFFF07
:10B85000E7800040AA8479DD97F00000E780E09C53
:10B860001389C4002A8481454A8597000000E78037
:10B87000005F0C4041464A8597000000E780405B2E
:10B88000832944006385090C4E8502D802DA02DC64
:10B8900002DE97300100E780E0382ACE141005461A
:10B8A0002C0808184ECC97500000E780E00A13756A
:10B8B000F50F51ED8355840093E525004A859700E7
:10B8C0000000E780E05E11460C104A8597000000FA
:10B8D000E78000560146976501009385A5D026852F
:10B8E00097F0FFFFE7802042268597000000E78061
:10B8F000407D5C40A1D3014685450D4597F0FFFF93
:10B90000E7800035AA841DD548401389C4009730CC
:10B910000100E78020312AC64A8597000000E780B1
:10B92000404C3246636FC5004C404A85970000008A
:10B93000E780005001468145268597F0FFFFE780AC
:10B94000803C268597000000E780A077E5B5835509
:10B950008400ADB71763FFFFE702637897A7FF1F67
:10B960009387075D9C471DC193E7870017A5FF1FBD
:10B970001305453917A7FF1F2320F75C9710010017
:10B98000E78040321763FFFF6700A377DD9B17A7AF
:10B99000FF1F2323F75A97300000E780E0647DF112
:10B9A00017A5FF1F1305053697100100E780E03348
:10B9B000D1BF1763FFFFE70203704169AA892E8A8E
:10B9C000B28A368BBA8B814417ACFF1F130C4C56CE
:10B9D000930C400E7D1997F0FFFFE780205863C459
:10B9E000A40001443DA03384940383270C0B3E94B0
:10B9F0008357C401638627055A87D6865286CE852B
:10BA00001305040397000000E780E0BB01C9238011
:10BA10000B0022851763FFFF6700636D8347F40106
:10BA200085C35A87D6865286CE851305940897001B
:10BA30000000E78040B909C585472380FB00D1BFDE
:10BA4000850451BF835745006380071E1763FFFFBE
:10BA5000E702436701112A8497000000E780C04D88
:10BA600009C985476309F50605611763FFFF67008C
:10BA7000A36897E00000E780007C7DF583574400D1
:10BA80004947ED9BE392E7FEC14522859700000000
:10BA9000E7804033AA84228597000000E780204F8A
:10BAA0000357440002CE91472A89631AF700228582
:10BAB00097000000E780A0513C082ACC3ECE97E0DA
:10BAC0000000E78080765C55C5D374084A86A68559
:10BAD0000545829751BF03574400D147E3F6E7F885
:10BAE000032A0400C169014997AAFF1F938A4A44A7
:10BAF000130B400EFD1997F0FFFFE7802046634FC0
:10BB0000A90E2285032A040097000000E780C042A6
:10BB1000A1452A89228597000000E780A02AAA84EF
:10BB2000228597000000E780804A14402A86AA896F
:10BB300078082685CA8597000000E780C0E7AA84B8
:10BB400005D503C7F40189476315F7008347C10191
:10BB500081DF5546D2851385640097300100E78068
:10BB6000E0E7014597800000E780C01901C583D751
:10BB7000C401A5E797A7FF1F9387873B9C47935571
:10BB80001900858913D73700058B01CF8983858BF1
:10BB90006399B70001452EC697000000E780C0DB1F
:10BBA000B2454E8597800000E780601F0346C101C3
:10BBB0002A8493751900268597900000E780E03964
:10BBC00035C1268597800000E780E018268511C0E2
:10BBD000014597800000E780004C97300000E78027
:10BBE000A0408547E312F5E883C754001307F00F20
:10BBF000E38CE7E68507A382F400BDB5B3046903CF
:10BC000083A70A0BBE9483D7C401638B37015546C3
:10BC1000D2851385640097300100E780C0D955DDD7
:10BC20000509D1BD5DD86DB782801763FFFFE702BC
:10BC3000634997800000E780000C05C1C16401449E
:10BC400017A9FF1F1309C92E9309400EFD1497F081
:10BC5000FFFFE780A030634EA40017A5FF1F130568
:10BC6000650A97100100E780E0031763FFFF670094
:10BC7000A348330534038327090B3E958357C50139
:10BC8000638897002312050097800000E780A00CCE
:10BC9000050475BF97A7FF1F938787299C478D834E
:10BCA000858B8DE31763FFFFE702634317A5FF1F33
:10BCB0001305450597100100E78020031763FFFF78
:10BCC0006700234482801763FFFFE7024341970523
:10BCD00000009385C5A017A5FF1F1305A5029710A7
:10BCE0000100E78020EE1763FFFF670083411763C1
:10BCF000FFFFE702C33E8841B7E70400BC5B0505D0
:10BD000042054181829709C585472300F500050555
:10BD10001763FFFF6700E33E83C7F5FF2E858507A6
:10BD2000A38FF5FE828083C7F5FFFD1793F7F70F0A
:10BD3000A38FF5FE99EF1763FFFFE702433AB7E7DA
:10BD40000400BC571385F5FF82971763FFFF670058
:10BD5000433B82801C41035745008D8FBA951CC11F
:10BD60002312B5003E85828093D78500A205144139
:10BD7000DD8D835745001387E6FF18C1890723121D
:10BD8000F50013D685004111238FB6FEA38FC6FEA2
:10BD90004101828018419307F7FF1CC1835745007A
:10BDA00085072312F500A30FB7FE82808357450055
:10BDB0008D8F2312F5001C41BE950CC12E8582800B
:10BDC000AA8703D7470008410D8FAA952392E70061
:10BDD0008CC38280184108453305A7408280835771
:10BDE0004500035765001D8F1C4108453385A7405A
:10BDF0003305A74082801763FFFFE702432E4111FE
:10BE00002EC62A8497000000E780A0FDB245637328
:10BE1000B50001A0835744000840BE952312B4002A
:10BE20003E9541011763FFFF6700A32D1763FFFFD6
:10BE3000E702E32A41112E84B28532C69700000042
:10BE4000E780A0FB3246A28597300100E78000B969
:10BE500041011763FFFF6700C32A1763FFFFE70273
:10BE600003282E84854597000000E78000F9230011
:10BE700085001763FFFF6700C3281763FFFFE70212
:10BE8000032641112317B100894597000000E78080
:10BE9000C0F68347E1002300F5008347F100A300CB
:10BEA000F50041011763FFFF6700A3251763FFFF3C
:10BEB000E702E32293D78500A2054111DD8D231708
:10BEC000B100894597000000E78020F38347E10037
:10BED0002300F5008347F100A300F500410117633B
:10BEE000FFFF670003221763FFFFE702431F13975B
:10BEF000850193D78501C166938606F0D98F13D744
:10BF00008500758FD98FA2053707FF00F98D411184
:10BF1000DD8D2EC6914597000000E78000EE6C0095
:10BF2000114697300100E78060AB41011763FFFFC6
:10BF30006700231D1763FFFFE702631A1C41854555
:10BF400003C4070097000000E78080E6228517639E
:10BF5000FFFF6700031B1763FFFFE70243181C4145
:10BF60004111894503C7070083C717002307E10074
:10BF7000A307F10097000000E78080E30355E1008C
:10BF800041011763FFFF6700C3171763FFFFE70255
:10BF900003151C414111894503C7070083C71700DA
:10BFA0002307E100A307F10097000000E78040E0CD
:10BFB0008357E100410113D58700A2075D8D42053B
:10BFC00041811763FFFF6700C3131763FFFFE70299
:10BFD00003110C4141112A84114668009730010079
:10BFE000E780C09F9145228597000000E78040DCF4
:10BFF000B247C166938606F01397870113D5870170
:10C00000598D13D78700758F598DA2073707FF0009
:10C01000F98F5D8D41011763FFFF6700830E1C459B
:10C02000BE950CC18280AE87944391E6584101EFE2
:10C030000CC15CC1828003C7570013671700A3823D
:10C04000E700B687D5B70CC3EDB7AA87084119CD6D
:10C050001841D44398C36313D500D8C32A87034635
:10C0600057009376160081E62320070082809443D0
:10C0700081CA8C4203A847008CC363930601CCC3DA
:10C08000799A14C3A302C7003687D1BF1C45DC4789
:10C090001D8DB777DBB6938777DB09853305F5020E
:10C0A000420541818280F147B385F50248452E95CE
:10C0B00082808347450085072302F500828017634D
:10C0C000FFFFE702C3012A8409E41763FFFF67004B
:10C0D000430383474400F5DBFD1793F7F70F230273
:10C0E000F400E5F71C4403D7270005072391E70078
:10C0F000DC4399C3228582974C4889CD83475400FD
:10C10000898B99E71C4422859C479C439C478297D6
:10C11000232A04000040232004007DB71763FFFF9B
:10C12000E702E3FB8357250041112EC681EB014452
:10C13000228541011763FFFF6700A3FC0357050039
:10C140008147F146E305F7FEB385D70240458507F1
:10C150002E948345440008C4F5F5B247AA8481E7CC
:10C16000232A040009A81C456C0022859C439C439B
:10C17000829748C84DDD85472312F400B24723203B
:10C180000400231804002319F4005C485CC483D71E
:10C190002400FD172391F40061BF1763FFFFE7023E
:10C1A00003F497A7FF1F9387E7B78843232605006B
:10C1B00023240500410597100100E78000B31763B1
:10C1C000FFFF670003F41763FFFFE70243F117A4C3
:10C1D000FF1F130424B51C40411199CF9C47230035
:10C1E000B5002AC65CC197000000E78040FB1C40F8
:10C1F000DC4399C33245829741011763FFFF670013
:10C2000043F00347450029E3584DAA877D551DCFCC
:10C210001763FFFFE702A3EC1CC3DC4797A6FF1FD1
:10C2200023A2E6B0F156130507012390D700970526
:10C2300000009385050297100100E780A098014552
:10C240001763FFFF6700E3EB7D55828082801763F1
:10C25000FFFFE702C3E801116146814528009760AE
:10C26000FFFFE780C0EA97A7FF1F9387A7AB9C4318
:10C2700028009305F00FDC473EC697000000E780DA
:10C28000C0F405611763FFFF6700A3E797A7FF1FCF
:10C29000938747A99C43D847A1679387C702631E2A
:10C2A000F70A397106DE22DC26DA80004AD84ED63B
:10C2B00052D456D23285B28497000000E780C0C7BE
:10C2C000AA89268597000000E78020C92318A4FCCE
:10C2D000268597000000E78040C82319A4FC268526
:10C2E00097000000E78060C783D744000A8A231ABA
:10C2F000A4FC858393F7F70F230EF4FC8607BD0794
:10C3000093F7073F3301F1408A8A01498347C4FD0F
:10C310006367F902CE85130584FC232C54FD970036
:10C320000000E78080EA5281130104FCF25062545D
:10C33000D2544259B259225A925A2161828026859A
:10C3400097000000E78060C193171900D697050990
:10C350002390A7001379F90F55BF828097A7FF1F7D
:10C360009387479C9C43D847A1679387A702631A8A
:10C37000F70A397106DE22DC26DA80004AD84ED66A
:10C3800052D456D23285B28497000000E780C0BAFA
:10C39000AA89268597000000E78020BCFD57231856
:10C3A000A4FC26852319F4FC97000000E780E0BA7E
:10C3B00083D744000A8A231AA4FC858393F7F70FD6
:10C3C000230EF4FC8607BD0793F7073F3301F140C6
:10C3D0008A8A01498347C4FD6367F902CE85130544
:10C3E00084FC232C54FD97000000E78000DE52817E
:10C3F000130104FCF2506254D2544259B259225AE9
:10C40000925A21618280268597000000E780E0B47F
:10C4100093171900D69705092390A7001379F90FF0
:10C4200055BF828097A7FF1F9387C78F9C43D8472C
:10C43000A16789076310F70A397106DE22DC26DA64
:10C4400080004AD84ED652D456D2328532899700CF
:10C450000000E78060AEAA894A8597000000E78067
:10C46000C0AF835749000A8A2318A4FC858393F739
:10C47000F70F230CF4FC8607BD0793F7073F330142
:10C48000F1408A8A8144834784FD63E7F402CE85C4
:10C49000130584FC232A54FD97000000E780E0D2B6
:10C4A0005281130104FCF2506254D2544259B259E1
:10C4B000225A925A216182804A8597000000E780C3
:10C4C000C0A993971400D69785042390A70093F4EE
:10C4D000F40F55BF828097A7FF1F9387A7849C43C3
:10C4E000D847A1679387E704631EF70A397106DE10
:10C4F00022DC26DA80004AD84ED652D456D2328573
:10C50000B28497000000E78020A3AA8926859700BF
:10C510000000E78080A42318A4FC26859700000073
:10C52000E780A0A3231AA4FC268597000000E780DB
:10C53000C0A283D744000A8A2319A4FC858393F7F9
:10C54000F70F230EF4FC8607BD0793F7073F33016F
:10C55000F1408A8A01498347C4FD6367F902CE85A9
:10C56000130584FC232C54FD97000000E780E0C5F0
:10C570005281130104FCF2506254D2544259B25910
:10C58000225A925A21618280268597000000E78016
:10C59000C09C93171900D69705092390A70013791B
:10C5A000F90F55BF82809797FF1F9387A7779C430A
:10C5B000D847A1679387C704631AF70A397106DE63
:10C5C00022DC26DA80004AD84ED652D456D23285A2
:10C5D000B28497000000E7802096AA8926859700FC
:10C5E0000000E7808097FD572318A4FC2685231AB6
:10C5F000F4FC97000000E780409683D744000A8A45
:10C600002319A4FC858393F7F70F230EF4FC860708
:10C61000BD0793F7073F3301F1408A8A01498347F9
:10C62000C4FD6367F902CE85130584FC232C54FDF9
:10C6300097000000E78060B95281130104FCF250BA
:10C640006254D2544259B259225A925A216182807C
:10C65000268597000000E780409093171900D69731
:10C6600005092390A7001379F90F55BF828097978A
:10C67000FF1F9387276B9C43D847A167DD0763178C
:10C68000F7041763FFFFE70283A5797132853284CF
:10C6900097000000E780408A2AC6228597000000A4
:10C6A000E780A08B2311A102228597000000E7807C
:10C6B000A088B2452300A102280897000000E78067
:10C6C000C0B045611763FFFF6700A3A382809797FF
:10C6D000FF1F938727659C43D847A16793878704EB
:10C6E0006317F7041763FFFFE702639F79713285D1
:10C6F000328497000000E78020842AC622859700B4
:10C700000000E78080852311A102228597000000A8
:10C71000E7808082B2452300A1022808970000002C
:10C72000E780A0AA45611763FFFF6700839D8280B1
:10C730009797FF1F9387075F9C43D847A16793870D
:10C74000A7046312F7021763FFFFE7024399011181
:10C750002800814597000000E78020A70561176346
:10C76000FFFF6700039A82809797FF1F9387875B7D
:10C770009C43D847A167938757026319F702176351
:10C78000FFFFE702C3950111328597F0FFFFE780B5
:10C79000A07A2308A1008145280097000000E780C7
:10C7A000C0A205611763FFFF6700A395828097977A
:10C7B000FF1F938727579C43D847A1679387E702BA
:10C7C000631BF7041763FFFFE702639101113285D2
:10C7D000328497F0FFFFE7804078AA84228597F0A3
:10C7E000FFFFE7808077854709E9228597F0FFFF03
:10C7F000E78080744205B337A000280081452318E4
:10C8000091003ECA97000000E780209C05611763F5
:10C81000FFFF6700038F82809797FF1F93878750E2
:10C820009C43D84799476313F7081763FFFFE70254
:10C83000038B79713285328497F0FFFFE780C06FF8
:10C840002AC6228597F0FFFFE78020712310A102FE
:10C85000228597F0FFFFE780206E2301A102228549
:10C8600097F0FFFFE780406DA301A102228597F0BA
:10C87000FFFFE780606C2302A102228597F0FFFF93
:10C88000E780806B2313A102228597F0FFFFE780EA
:10C89000A06AB2452314A102280897000000E7808F
:10C8A000C09245611763FFFF6700A3858280979759
:10C8B000FF1F938727479C43D847A1679387C703E8
:10C8C0006313F7081763FFFFE7026381797132850D
:10C8D000328497F0FFFFE78020662AC6228597F012
:10C8E000FFFFE78080672310A102228597F0FFFFFA
:10C8F000E780A0662311A102228597F0FFFFE78061
:10C90000A0632302A102228597F0FFFFE780C062A7
:10C91000A302A102228597F0FFFFE780E0612303D5
:10C92000A102228597F0FFFFE7800061B245A303D3
:10C93000A102280897000000E7802089456117536D
:10C94000FFFF6700037C82801753FFFFE702237914
:10C9500001112A8497F0FFFFE780005EAA842285F8
:10C9600097F0FFFFE780605F228597F0FFFFE78089
:10C97000C05E035744008D4763F7E700228597F0B8
:10C98000FFFFE780805D228597F0FFFFE780E05C96
:10C990002800A68597000000E780208305611753D3
:10C9A000FFFF670003769797FF1F9387A7379C4386
:10C9B000D847A167FD07631FF7001753FFFFE70282
:10C9C0000372328597000000E78040F81753FFFF9D
:10C9D0006700237382809797FF1F9387A7349C4338
:10C9E000D847A167E5076315F7081753FFFFE7026C
:10C9F000036F79713285328497F0FFFFE780C0536F
:10CA00002AC6228597F0FFFFE7802055228597F000
:10CA1000FFFFE78080542310A102228597F0FFFFDB
:10CA2000E780A053520551812311A10222852302E0
:10CA3000010297F0FFFFE7802050A302A1022285A8
:10CA400097F0FFFFE780404F2303A102228597F074
:10CA5000FFFFE780604EB245A303A102280897F0CC
:10CA6000FFFFE780807645611753FFFF670063692A
:10CA700082809797FF1F9387E72A9C43D847A16737
:10CA80009387E703631FF7001753FFFFE702236550
:10CA9000328597000000E78060EB1753FFFF6700C7
:10CAA000436682809797FF1F9387C7279C43D84789
:10CAB000A16793874704631EF7021753FFFFE7023E
:10CAC000036279713285328497F0FFFFE780C046B8
:10CAD0002AC6228597F0FFFFE7802048B245280844
:10CAE00097F0FFFFE780606E45611753FFFF670017
:10CAF000436182809797FF1F9387C7229C43D84743
:10CB0000A167938787026310F7041753FFFFE702BB
:10CB1000035D79713285328497F0FFFFE780C04171
:10CB20002AC6228597F0FFFFE7800041B245230027
:10CB3000A102280897F0FFFFE7802069456117539D
:10CB4000FFFF6700035C82801753FFFFE702235952
:10CB5000011197F0FFFFE780203EAA85280097F09B
:10CB6000FFFFE780806605611753FFFF6700635989
:10CB70009797FF1F9387071B9C43D847A167D1074F
:10CB8000631FF7001753FFFFE702635532859700D5
:10CB90000000E780A0FB1753FFFF670083568280E9
:10CBA0009797FF1F938707189C43D847A167C5072E
:10CBB000631FF7001753FFFFE702635232859700A8
:10CBC0000000E780A0F81753FFFF670083538280BF
:10CBD0009797FF1F938707159C43D847A167B9070D
:10CBE000631FF7001753FFFFE702634F328597007B
:10CBF0000000E780A0F51753FFFF67008350828095
:10CC00009797FF1F938707129C43D847A167AD07EB
:10CC1000631FF7001753FFFFE702634C328597004D
:10CC20000000E780A0F21753FFFF6700834D82806A
:10CC30009797FF1F9387070F9C43D847894763182F
:10CC4000F7021753FFFFE70283490111328532C80B
:10CC500097F0FFFFE780402EAA85280097F0FFFF9E
:10CC6000E780A05605611753FFFF67008349828064
:10CC70009797FF1F9387070B9C43D847A1678D07A2
:10CC80006311F7041753FFFFE70263450111328573
:10CC9000328497F0FFFFE780202A13066100AA8400
:10CCA0004C00228597300000E780C0232800A6852D
:10CCB00097F0FFFFE780605105611753FFFF6700A2
:10CCC000434482809797FF1F938707069C4381CF39
:10CCD000DC4391CB1753FFFFE70263408297175362
:10CCE000FFFF6700034282801753FFFFE702233FE5
:10CCF00079713C08AE843ED2A165B7070A002A8448
:10CD00003ED448103C08DD053ED636C432C63AC291
:10CD100097D0FFFFE780402C12474810BA8597F064
:10CD2000FFFFE780C01332464810B28597F0FFFF3F
:10CD3000E780E014A2464810B68597F0FFFFE78031
:10CD40000012501001478146A685228597D0FFFF2B
:10CD5000E780E04D45611753FFFF6700833A1753A3
:10CD6000FFFFE702C33701117C000329C501AE8430
:10CD70003ECAA165B70707002A843ECC48087C005C
:10CD8000C5053ECE97D0FFFFE78000258345D9003B
:10CD9000480897F0FFFFE780800C50080147814664
:10CDA000A685228597D0FFFFE7806048056117536D
:10CDB000FFFF670003351753FFFFE702433283C7C6
:10CDC000950093F7F707A384F50097000000E7802C
:10CDD00040F91753FFFF6700C3321753FFFFE70205
:10CDE000033079713C08AE843ED2A165B7070900D3
:10CDF0002A843ED448103C08938545043ED632C66A
:10CE000036C497D0FFFFE780201DA2464810B685A4
:10CE100097F0FFFFE780A00432464810B28597F0F4
:10CE2000FFFFE780C005501001478146A685228597
:10CE300097D0FFFFE780A03F45611753FFFF6700D2
:10CE4000432C1753FFFFE702832983C79500411145
:10CE50002A8493F7F707A384F50032852EC697F04E
:10CE6000FFFFE780800F85672AC46370F502977023
:10CE70000000E78020E92246B24509ED11478146CE
:10CE8000228597000000E78060E641011753FFFF0D
:10CE90006700232701478346F501DDB71753FFFFDE
:10CEA000E702432201113C003ECAB7070A003ECC0C
:10CEB0003C003ECE83C79500AA89328593F7F707D9
:10CEC000A384F5002E8497F0FFFFE78000098567B3
:10CED000637DF504A165AA8493858504480897D0ED
:10CEE000FFFFE780600F268597700000E78080E1F4
:10CEF0002A8929E19145480897F0FFFFE78020F64D
:10CF0000A685480897F0FFFFE78060F7CA854808C4
:10CF100097F0FFFFE780A0F4014781465008A28503
:10CF20004E8597D0FFFFE780803005611753FFFFE4
:10CF30006700831C8145480897F0FFFFE78020F2D7
:10CF40000349090275BF1753FFFFE702A317797161
:10CF50001C103ECAB7070F003ECC404D1C10AA84DF
:10CF6000AE894808994532C636893ECE97D0FFFF34
:10CF7000E780800632464808B28597F0FFFFE780D9
:10CF800000EE630C0902A545480897F0FFFFE78013
:10CF9000C0E62546CA8597200100E78020A45008F6
:10CFA00001478146CE85268597D0FFFFE780202860
:10CFB00045611753FFFF670023148355C4024808D7
:10CFC00097F0FFFFE780A0EB0355E402814505C51C
:10CFD000854785456301F502C167FD179305F00F8D
:10CFE000630BF5007D1597700000E780208E930598
:10CFF000150093F5F50F480897F0FFFFE78020E64E
:10D0000083450403480897F0FFFFE78040E5834528
:10D010001403480897F0FFFFE78060E4835524037A
:10D02000480897F0FFFFE78080E5835544034808F0
:10D0300097F0FFFFE780A0E49DB71753FFFFE702DB
:10D04000030A83C795008146014693F7F707A38437
:10D05000F50097000000E78040EF1753FFFF6700DF
:10D06000430A1753FFFFE702830779713E841C10C0
:10D070003ECA2E89B7070F00A1653ECCFD051C10E6
:10D08000AA84480842C03AC23ECE36C432C697D0BF
:10D09000FFFFE78060F432464808B28597F0FFFF53
:10D0A000E780E0DBA2464808B68597F0FFFFE780FF
:10D0B00000DD12474808BA8597F0FFFFE78020DCC3
:10D0C0000248630C08029145480897F0FFFFE7808B
:10D0D000C0D21146A28597200100E7802090500819
:10D0E00001478146CA85268597D0FFFFE780201437
:10D0F00045611753FFFF6700C3008945480897F053
:10D10000FFFFE78080CF834704002300F5008347BB
:10D110001400A300F500E1B71753FFFFE70283FAFD
:10D1200083C7950001112A8A93F7F707A384F500B6
:10D130003285AE8432C697F0FFFFE78000E23246C8
:10D140002A89328597F0FFFFE78000DF85676373E8
:10D15000F902AA894A8597700000E780A0BA2A845C
:10D1600019ED114781464A86A68552859700000031
:10D17000E780C0B705611753FFFF6700E3F79387A8
:10D18000E9FF93F7F70F0547E366F7FE8347F501DD
:10D1900095EB8947E380F9FE8346F4015285014708
:10D1A0004A86A68597000000E78040B4A167D907AA
:10D1B00048083ECC230A010002CE97000000E78019
:10D1C000A0B04DBF639EE7008947639EF9009307B7
:10D1D0001020231FF50097700000E780C0B76DBFD7
:10D1E0000947E39BE7FA8D47E398F9FA22859770A0
:10D1F0000000E78080DF9797FF1F9387E7D19C436C
:10D2000099E79797FF1F9387E7BA9C4399C703D580
:10D21000040097800000E780A0CE231F0400228531
:10D220005DBF1753FFFFE70283EB01113C003ECACD
:10D23000B7070B003ECC3C003ECE83C795002A8941
:10D24000328593F7F707A384F500AE8497F0FFFFCC
:10D25000E780A0D093170501C187635AF006A16546
:10D260002A849385E502480897D0FFFFE780C0D65F
:10D27000A285480897F0FFFFE78060C09797FF1FDF
:10D28000938747B39C43A9EB01449375F40F480877
:10D2900097F0FFFFE780A0BC9355844093F5F50F0E
:10D2A000480897F0FFFFE78080BB9355044193F552
:10D2B000F50F480897F0FFFFE78060BA0147814605
:10D2C0005008A6854A8597D0FFFFE78040F60561A4
:10D2D0001753FFFF6700E3E2416585460546A285D7
:10D2E0007D1597500000E78060BD59DD510597001E
:10D2F0000100E780808F130440063344850271B734
:10D300001753FFFFE702A3DD0111B70706003EC672
:10D3100083C7950021642A8993F7F707A384F50052
:10D32000AE8428009305A4040AC40AC897D0FFFF5E
:10D33000E78080CA300001478146A6854A8597D09C
:10D34000FFFFE780C0EE97E0FFFFE780E0111304E6
:10D350009404480822CC230A010002CE9700000062
:10D36000E780809605611753FFFF670083D9175345
:10D37000FFFFE70223D5C1642A8901449799FF1F63
:10D38000938909BB130A8002FD1497E0FFFFE78031
:10D39000E0BD6347A40001451753FFFF6700C3D5F5
:10D3A000B307440303A7C90ABA9703D70700630664
:10D3B000970083D72700638427010504F9B7054543
:10D3C000E1BF1753FFFFE702E3CF2A8A2E8999C1F5
:10D3D00023A0050081498144979AFF1F938A0A95EB
:10D3E000614B97E0FFFFE780A0BE63C7A4004E85B6
:10D3F0001753FFFF670043D03384640383A70A00F9
:10D400003E948357040099E76304090023208900B0
:10D410008504C1BF4146D285130544009710010021
:10D42000E780605975F5A289E5B71753FFFFE7025A
:10D4300063C939717C083ED4B7070A003ED67C0820
:10D440003ED883C795002A8A328593F7F707A384CD
:10D45000F5002E8932C697F0FFFFE78000B08567A0
:10D460006373F5083246AA84328597F0FFFFE780A0
:10D47000A0AC8547AA8963E8A706A16593858504C2
:10D48000281097D0FFFFE78020B526859770000011
:10D49000E78040872A8429ED9145281097F0FFFF07
:10D4A000E780E09BA685281097F0FFFFE780209D8E
:10D4B000CE85281097F0FFFFE780609A01478146EC
:10D4C0003010CA85528597D0FFFFE78040D6A1670C
:10D4D0009387770448183EDC230A010202DE97F0A6
:10D4E000FFFFE780607E21611753FFFF6700C3C025
:10D4F0008145281097F0FFFFE7806096A6852810E9
:10D5000097F0FFFFE780A0979797FF1F9387C7D8F3
:10D510009C4381CB22856389090097D00000E78076
:10D5200040248345040271B797D00000E780C022F1
:10D53000CDBF1753FFFFE702E3B883C79500411142
:10D54000AA8993F7F707A384F5003285AE84328A5F
:10D5500097F0FFFFE78060A08567637FF5022A8967
:10D5600097600000E780007A2A84914631C583479E
:10D57000F50105476387E70291C70D476366F70426
:10D58000AD461DA89305050303250A0041469710E3
:10D590000100E78040420DE941011753FFFF67009A
:10D5A000A3B59305950803250A004146971001008D
:10D5B000E7806040814669F54A86A6854E859700DA
:10D5C0000000E780C081C9BF83250A0013059408C5
:10D5D00097700000E780A02919C1C146F1BF979755
:10D5E000FF1F938767939C4399E79787FF1F938754
:10D5F000677C9C4399C7228597800000E780208A3A
:10D6000069FD8547A30FF400228597B00000E780ED
:10D610006084228597600000E780E0734E85814634
:10D620004A86A68597F0FFFFE780607BA167938716
:10D63000570448003EC42302010002C697F0FFFFD2
:10D64000E780806891BF1753FFFFE702C3A683C737
:10D6500095004111AA8993F7F707A384F500328555
:10D660002E89B28A97F0FFFFE780208F8567637469
:10D67000F50EAA8497600000E780C0682A840DED4B
:10D68000416B014A979BFF1F938B8B8A130C400EB3
:10D690007D1B19A833048A0383A70B0B3E94835781
:10D6A000C40163836705050A97E0FFFFE780008BED
:10D6B000E342AAFE95460DA08357C50163969702E3
:10D6C0009305050303A50A00414697100100E78072
:10D6D000802E994611E181462686CA854E8597F0AF
:10D6E000FFFFE780C06F85A883A50A001305040328
:10D6F00097700000E780A017C14679FD2285231EA0
:10D70000940097A00000E780E074228597600000F5
:10D71000E78060649797FF1F938707B89C43A9C36E
:10D7200023000402228597D00000E78040F04E8558
:10D7300081462686CA8597F0FFFFE780406AA16789
:10D740009387070448003EC42302010002C697F0F5
:10D75000FFFFE780605741011753FFFF67002399E0
:10D7600089472300F402E1B7397106DE22DC4AD88A
:10D77000800052D456D25AD026DA4ED65ECE2E8AA9
:10D7800032892A8B97D0FFFFE780407A0605710522
:10D7900041998A8A3301A140232224FC231404FCEA
:10D7A00097D0FFFFE780807883479A00060535050C
:10D7B00093F7F7072315A4FCA304FA004A85232650
:10D7C00024FC97E0FFFFE780407993170501C187AC
:10D7D0006340F0025681130104FCF2506254D254AB
:10D7E0004259B259225A925A025BF24B216182800D
:10D7F000AA844A8597E0FFFFE7802076AA894A85B8
:10D8000097E0FFFFE7806075A1659385C5022A89CF
:10D81000130544FC97C0FFFFE780007C268597C076
:10D82000FFFFE7804070854511C94A86CE8597C0C5
:10D83000FFFFE780C069AA8B21E98945130544FCF5
:10D8400097E0FFFFE780A061A685130544FC97E001
:10D85000FFFFE780C062CE85130544FC97E0FFFF21
:10D86000E780E061CA85130544FC97E0FFFFE7808D
:10D87000006101478146130644FCD2855A8597D042
:10D88000FFFFE780C09AB9B78145130544FC97E0D4
:10D89000FFFFE780C05CA685130544FC97E0FFFF0F
:10D8A000E780E05DCE85130544FC97E0FFFFE7804D
:10D8B000005DCA85130544FC97E0FFFFE780205C0C
:10D8C000814497D0FFFFE7806066E3D4A4FA83A782
:10D8D0000B0113971400BA9783D5070099C5130558
:10D8E00044FC97E0FFFFE78080598504D9BF797138
:10D8F00006D622D44AD000184ECE52CC56CA26D2D2
:10D900005AC8AE893289AA8A97D0FFFFE7800062A1
:10D910000605690541990A8A3301A140232A24FC9E
:10D92000231C04FC97D0FFFFE780406083C7990069
:10D9300006052D0593F7F707231DA4FCA384F90022
:10D940004A85232E24FC97E0FFFFE78000619317B0
:10D950000501C187634FF0005281130104FDB250ED
:10D96000225492540259F249624AD24A424B4561CA
:10D970008280AA844A8597E0FFFFE780005EA16568
:10D980009385A5022A89130544FD97C0FFFFE78010
:10D99000A064268597C0FFFFE780E058854509C948
:10D9A000CA8597C0FFFFE78080552A8B29E189450A
:10D9B000130544FD97E0FFFFE780604AA685130545
:10D9C00044FD97E0FFFFE780804BCA85130544FDC7
:10D9D00097E0FFFFE780A04A01478146130644FD18
:10D9E000CE85568597D0FFFFE7806084B5B7814527
:10D9F000130544FD97E0FFFFE7806046A685130509
:10DA000044FD97E0FFFFE7808047CA85130544FD8A
:10DA100097E0FFFFE780A046814497D0FFFFE780B3
:10DA2000E050E3DBA4FA83270B0113971400BA97A5
:10DA300083D5070099C5130544FD97E0FFFFE780F4
:10DA400000448504D9BF1743FFFFE70243698347BA
:10DA50004500404DD5EFFD575DC48346940009470E
:10DA60006363D70A0346B400854663EEC60883069F
:10DA7000E40063CA06085C45F9562390D7009787EF
:10DA8000FF1F83C7E72A99E3A304E4009787FF1FDA
:10DA9000938747329C4381E78947A306F400978721
:10DAA000FF1F9387677F9C4381E789472306F40024
:10DAB0009705000093854506AA841305040197F095
:10DAC0000000E7802010FD57231AF40281471CDC78
:10DAD00001489787FF1F23A987249787FF1F9387F4
:10DAE000E724232E040304C0804397D0FFFFE78080
:10DAF000204E61463306C502814522859740FFFFCF
:10DB0000E780E06081473E851743FFFF6700635F62
:10DB1000FD57D5BF1743FFFFE702635C2A84035517
:10DB2000450297600000E780E01D19E5231E040010
:10DB30001743FFFF6700E35C8357E401F5DB9305C0
:10DB400004FF174501001305A5E397E00000E780F7
:10DB5000E014F9BF1743FFFFE70263582E89A16560
:10DB600041119385E5032A8436C432C6BE843AC285
:10DB700097C0FFFFE780404612472285BA8597E0AD
:10DB8000FFFFE780C02D32462285B28597E0FFFF78
:10DB9000E780E02EA2462285B68597E0FFFFE7806A
:10DBA000002E630309029145228597E0FFFFE7807D
:10DBB000C0241146A68597100100E78020E24101AC
:10DBC0001743FFFF6700E3538945228597E0FFFF76
:10DBD000E780A02283C704002300F50083C7140058
:10DBE000A300F500E9BF1743FFFFE702434F83C7D8
:10DBF0009500444D054793F7F707A384F5001C42B1
:10DC0000411183C707006367F7062E842A89B1C0D4
:10DC100003C7D400630FF7021787FF1F1307871985
:10DC2000184305C3A386F40097A00000E780404A8C
:10DC300083C7D40099E741657D1597400000E780D0
:10DC4000403083D72403918B89C797E00000E78099
:10DC5000C0134A85A28597F0FFFFE7808010A16777
:10DC6000C10748003EC42302010002C697F0FFFF2F
:10DC7000E780800541011743FFFF67008348174392
:10DC8000FFFFE702C34503D745008D47AA84411132
:10DC90002E8432892E8563E3E70297E0FFFFE78059
:10DCA000C02BAA8523000900268597C0FFFFE780C7
:10DCB000002541011743FFFF6700A34497E0FFFFE2
:10DCC000E780A0292AC6228597E0FFFFE780E028A9
:10DCD000B24585472A862300F900268597C0FFFFB5
:10DCE000E780E01EF9B7397106DE22DC26DA800013
:10DCF0004ED652D456D24AD85AD05ECEAE89B284CD
:10DD0000AA8A97D0FFFFE780602106051305250248
:10DD100041990A8A3301A140232224FC231404FCE4
:10DD200097D0FFFFE780801F83C7990006054D0548
:10DD300093F7F7072315A4FCA384F900268523266F
:10DD400024FC97E0FFFFE780402193170501C1877E
:10DD50006340F0025281130104FCF2506254D25429
:10DD60004259B259225A925A025BF24B2161828087
:10DD7000AA8B03AB040097C0FFFFE780C01A51E5F0
:10DD800083D7440001498544F11793B71700A301D5
:10DD9000F4FC834734FCA165C9C79385E5041305EA
:10DDA00044FC97C0FFFFE7802023A685130544FCB1
:10DDB00097E0FFFFE780A00ADE85130544FC97E0AB
:10DDC000FFFFE780C00B834734FC114691E309460F
:10DDD000DA85130544FC97E0FFFFE7806005814486
:10DDE000630A0900416B7D1B97D0FFFFE78000139A
:10DDF00063CCA40201478146130644FCCE855685B8
:10DE000097C0FFFFE780A042B1B7A685130634FC98
:10DE100097000000E780E0E6933415002A89860425
:10DE20008DBF9385C504A5BF8327C9001397140030
:10DE3000BA9783D5070063886501130544FC97E012
:10DE4000FFFFE780C003850445B71743FFFFE702E4
:10DE5000832679711C103EC4B7070F003EC61C1004
:10DE60003EC883C79500AA8A328593F7F707A38433
:10DE7000F500AE89328497E0FFFFE780000E93172C
:10DE80000501C187635AF0062A8A228597E0FFFFC1
:10DE9000E780A00C2A895285032B040097C0FFFF5E
:10DEA000E780600839ED8357440081440544F11749
:10DEB00093B71700A303F10083457100DA87228727
:10DEC000CA865286280097000000E780E0C8014714
:10DED00081463000CE85568597C0FFFFE78020350C
:10DEE000A1679387D70348083ECC230A810026CE3A
:10DEF00097F0FFFFE78040DD45611743FFFF6700B4
:10DF0000031FA2851306710097000000E78060D709
:10DF1000AA84094455D13544E30055FB4A8597F05E
:10DF2000FFFFE78000450D4441D9014497D0FFFF32
:10DF3000E780C0FE634DA400C16B0144FD1B97D078
:10DF4000FFFFE780A0FD634EA4001544B5B7DC4495
:10DF500013171400BA9783D70700638327030504B8
:10DF6000F1B7D84493171400BA9703D70700631B7F
:10DF7000770123902701268597A00000E78080DBAA
:10DF800001441DBF050465BF1743FFFFE70283136C
:10DF900083C7950041112A8A93F7F707A384F500F8
:10DFA00032852E89328497E0FFFFE78000FB9317CC
:10DFB0000501C1876353F006AA89228597E0FFFF18
:10DFC000E780A0F92311A1004E85832A040097C0A1
:10DFD000FFFFE78040F539E583574400854401445D
:10DFE000F11793B71700A300F1000348110003577E
:10DFF0002100D6875285CE862686CA8597F0FFFFF8
:10E00000E7806006A167F10748003EC42302910043
:10E0100022C697F0FFFFE78020CB41011743FFFFA7
:10E020006700830DA2851306110097000000E780AA
:10E0300040C52A84894455D98357210011678544F6
:10E04000BA97C2071167C1831307F7EFE36FF7F8B9
:10E050009787FF1F938747EC9C4381CB854513052A
:10E06000210097500000E78020758355210022850C
:10E07000814497C0FFFFE780A0E125D92310050068
:10E08000228597A00000E78040CD85B71743FFFFAA
:10E09000E702630283C7950041112A8B93F7F707C4
:10E0A000A384F50032852E8A328497E0FFFFE78053
:10E0B000C0EA93170501C1876351F006AA8A228539
:10E0C00097E0FFFFE78060E92A895685832B0400EB
:10E0D00097C0FFFFE78020E531E583574400814486
:10E0E0000544F11793B71700A301F100034831006D
:10E0F000DE875A854A87D6862286D28597F0FFFF2B
:10E10000E78060F6A167ED0748003EC42302810066
:10E1100026C697F0FFFFE78020BB41011743FFFFB2
:10E120006700E3FCA2851306310097000000E7803A
:10E1300040B5AA8409445DD99167CA97C20711679F
:10E14000C1831307F7EF0544E362F7FACA8597C066
:10E15000FFFFE780E0D3014451F9814997D0FFFFE9
:10E16000E780C0DC63DBA900984893971900BA9751
:10E1700003D7070005EF2390270197D0FFFFE78023
:10E18000E0DA1544E384A9F6268597A00000E7802D
:10E19000C0BC9787FF1F938727D89C430144B9D7FA
:10E1A0004A8597500000E780C05889B785097DB738
:10E1B0001743FFFFE70203F179713E847C083EC8F4
:10E1C0002E8AB7071400A1653ECAE5057C08AA8916
:10E1D000080836C4428932C6BA8AC6843ECC97C083
:10E1E000FFFFE78060DFCA85080897E0FFFFE78050
:10E1F00000C732460808B28597E0FFFFE78020C8D5
:10E20000A246630A09049D45080897E0FFFFE780DE
:10E21000C0BE1D4681459740FFFFE78040EF638900
:10E220000A089145080897E0FFFFE78000BD114606
:10E23000A68597000100E780607A100801478146B3
:10E24000D2854E8597C0FFFFE78060FE456117438A
:10E25000FFFF670063EAB685080897E0FFFFE780E5
:10E2600000C21C400808D8439355C701858912078E
:10E270005183B205D98D97E0FFFFE78040C01C4075
:10E28000080883C5870097E0FFFFE78040BD1C407A
:10E29000080883C5A70097E0FFFFE78040BC1C404B
:10E2A000080883C5970097E0FFFFE78040BB85BF64
:10E2B0008945080897E0FFFFE78020B483C7040082
:10E2C0002300F50083C71400A300F500BDB7174372
:10E2D000FFFFE70223DF83C795004111AA8993F767
:10E2E000F707A384F5003285AE84328497E0FFFF00
:10E2F000E780A0C693170501C187635DF0042A89F2
:10E30000032A040097C0FFFFE780E0C119E98357A3
:10E3100044000548F11793B71700A307F1008146A1
:10E3200031A81306F100A28597000000E7806095F0
:10E330001DC51C459DC783D6470001480347F10012
:10E3400093078500D2884A86A6854E8597000000EF
:10E35000E78040E641011743FFFF6700E3D9094822
:10E360007DBF1D486DBF1743FFFFE702A3D5657151
:10E370005C083EC4B7077B013EC65C083EC883C745
:10E3800095002A8A328593F7F707A384F500AE89B2
:10E3900097E0FFFFE78040BA8357E100E1C7894576
:10E3A000280097C0FFFFE78020C38145280097E041
:10E3B000FFFFE780C0AA97C0FFFFE78000C99787EB
:10E3C000FF1F938767ED9C431784FF1F0344449608
:10E3D000AA843334800099C3136424009787FF1FF5
:10E3E0009387479D9C4399C3136444009787FF1FFD
:10E3F000938787B29C4399C31364840083D5040038
:10E400002800014997E0FFFFE78060A783D524003B
:10E41000280097E0FFFFE78080A683D5440028000E
:10E4200097E0FFFFE780A0A597D0FFFFE78000AB54
:10E4300093150501C181280097E0FFFFE78020A424
:10E44000A285280097E0FFFFE78060A39C446360FB
:10E45000F902014781463000CE85528597C0FFFF03
:10E46000E780E0DC59611743FFFF6700E3C8DC4445
:10E470001314490028003E9497E0FFFFE780609660
:10E48000834744000347540089070607BA97860765
:10E49000E36AF5FC835524002800814A97E0FFFFDA
:10E4A000E780E09D83454400280097E0FFFFE78078
:10E4B000009B83455400280097E0FFFFE780209AE7
:10E4C0008347440063C9FA00814A8347540063C10B
:10E4D000FA020509A5BF1C4413975A002800BA97F1
:10E4E00083D50700850A97E0FFFFE7804099C9BF01
:10E4F000032BC40093975A0028003E9B83552B00A2
:10E50000850A97E0FFFFE780809783550B0028007E
:10E5100097E0FFFFE780A0964DBF1743FFFFE7029C
:10E5200003BC5C4993E717005CC997A00000E78033
:10E5300020B61743FFFF6700C3BC1743FFFFE70286
:10E5400003BA2E84814597F0FFFFE780C0E705C539
:10E5500083570500FD172310F50009C483572500D4
:10E560002310F40097000000E78060FB014517438B
:10E57000FFFF670003B931457DD823100400C5BFF4
:10E580001743FFFFE70203B483C7950041112A8AAE
:10E5900093F7F707A384F50032852E89328497E03C
:10E5A000FFFFE780809B93170501C1876356F00644
:10E5B000AA89C145228597E0FFFFE780A0802A8BCA
:10E5C0004E85832A040097C0FFFFE780C09531E99C
:10E5D00083574400231101000544F11793B7170036
:10E5E000A300F10081440348110003572100D6879E
:10E5F0005285CE862286CA8597F0FFFFE780A0A6C7
:10E60000A1679387170248003EC42302810026C6F3
:10E6100097E0FFFFE780406B41011743FFFF670072
:10E62000A3AD13061100A28597F0FFFFE780606598
:10E63000AA8409E523110100094475B79305210057
:10E640005A8597000000E78080EF835721002A84D5
:10E65000D9DB9787FF1F9387278C9C4381CB854508
:10E660001305210097500000E78000158355210015
:10E670002685314497C0FFFFE78080812DD5231088
:10E680000500268597900000E780206D0144A1BF1A
:10E690001743FFFFE702A3A441112E896C00AA844F
:10E6A00002C697F0FFFFE78000D20DC103570500B7
:10E6B00005072310E50097000000E78040E681474A
:10E6C0003E8541011743FFFF6700A3A332479547EB
:10E6D00065DBCA85268597300000E780400DC1477D
:10E6E000E34005FE3244854741462310F40083573A
:10E6F0000900A685130544002311F40097000100CA
:10E70000E780C02D228545BF1743FFFFE702839BAB
:10E7100083C795004111AA8A93F7F707A384F500F0
:10E720003285AE89328497E0FFFFE780008393173C
:10E730000501C1876356F0062A8AC145228597D014
:10E74000FFFFE7802068AA845285032B040097B05E
:10E75000FFFFE780407D31E983574400231101002A
:10E760008544F11793B71700A300F1000144034853
:10E77000110003572100DA875685D2862686CE857A
:10E7800097F0FFFFE780208EA1679387070248007C
:10E790003EC42302910022C697E0FFFFE780C052EB
:10E7A00041011743FFFF67002395A285130611005F
:10E7B00097F0FFFFE780E04C2A8409E52311010070
:10E7C000894475B726859305210097000000E780EE
:10E7D00060ECAA8449FD83552100228597B0FFFF94
:10E7E000E780006B49F5014997C0FFFFE78000749F
:10E7F000635DA900184893171900BA9703D707005B
:10E800000DEF035721002390E70097C0FFFFE7803B
:10E81000E071630625039777FF1F9387E76F9C439B
:10E8200099C70355210097500000E78080F02285AA
:10E8300097900000E78060521DBF050975B79544A9
:10E840003DB705C19307F00F630FF500C547630C93
:10E85000F5009307F5FF05453315F50042054181A5
:10E8600082800145828041657D158280B9E9174328
:10E87000FFFFE702C38603450603328497000000CA
:10E88000E78060FC9305803EB305B502C205C181F7
:10E8900081CD0357E402854763F8E70013050401BF
:10E8A00097E00000E78020428357E40241677D172C
:10E8B0006385E700FD172317F4021743FFFF670086
:10E8C000438482801733FFFFE702E37E004283C761
:10E8D0009500444D0349140093F7F707A384F5000E
:10E8E00083470400220911673369F900A167B34720
:10E8F000F90041112A8BAE8A63ECE70E83472400AE
:10E900001307C00EB91793F7F70F6373F710034798
:10E910003400C14763EEE70E834744001307E00766
:10E9200093C707086371F70C834984008347740019
:10E93000A209B3E9F900856763F7F90A034A64009D
:10E94000834754004E85220A336AFA00975000002C
:10E95000E780403B61C123962403834B3400137A44
:10E96000FA00239A34032388740323994403938978
:10E970000401631C090023A60402239804024E85A7
:10E9800097E00000E78060363DA0034924004A85F7
:10E9900097000000E78020EB2397A4028347440000
:10E9A0004E85A388F402E38D0BFCE30B09FC97E092
:10E9B0000000E780202F97900000E78000738146D9
:10E9C0000146D6855A8597E0FFFFE7800058A1678A
:10E9D000938797033EC423020100480002C697E0D4
:10E9E000FFFFE780602E41011733FFFF67002370B0
:10E9F0008544A2862686D6855A8597E0FFFFE78064
:10EA0000C054A167938797033EC423029100F1B7D6
:10EA1000BD44C5B79144F1BF1733FFFFE702836AD6
:10EA200001111C08404D3EC2B7070F003EC41C0830
:10EA30003EC62A89AE8997C0FFFFE78000D7585CA1
:10EA40001C5C6346B70E6394E50063E2A70E338552
:10EA5000A740B3B7A700B305B7401306803E814671
:10EA60009D8D97000100E78080B793140501C18058
:10EA7000A1659385C503480097B0FFFFE780C055A7
:10EA80008145480097D0FFFFE780603D835504042F
:10EA9000480097D0FFFFE780803E8355240448005C
:10EAA00097D0FFFFE780A03D814589CCC167FD1766
:10EAB0009305F00F6388F400268597500000E780E7
:10EAC000E0E0AA85480097D0FFFFE7804039035572
:10EAD0004404814501CDC167FD179305F00F63071D
:10EAE000F50097500000E78060DEAA85480097D0C7
:10EAF000FFFFE780C03683456404480097D0FFFFDE
:10EB0000E780E03583457404480097D0FFFFE78035
:10EB10000035500001478146CE854A8597B0FFFFFA
:10EB2000E780E07005611733FFFF6700E35C814415
:10EB300081B71733FFFFE702835A83C7950093F726
:10EB4000F707A384F50097000000E78020ED173356
:10EB5000FFFF6700035B1733FFFFE702A35683C77E
:10EB600095004111404D93F7F707A384F5002A8AD9
:10EB70003285B284AE8997D0FFFFE780003E2A8BB2
:10EB8000268597D0FFFFE780403D2A89268597D0CC
:10EB9000FFFFE780603A93170B0163CA0702E17732
:10EBA000CA97C207C183116763E3E702930709109D
:10EBB000C207C1831307B00F637BF70093170901E6
:10EBC000C187AA8A634AF000C54763FE5701410125
:10EBD0001733FFFF6700435297B0FFFFE780202500
:10EBE000E31725FFD5B763080B02630609028144CA
:10EBF00063890A02B7077F002310640523112405E7
:10EC00007CC0568597000000E780E0C39304803EF7
:10EC1000B304950239A0B7077F00232004047CC009
:10EC200081440355240497E00000E780A0A3A1C419
:10EC300097C0FFFFE78060B7269593D7F44133373D
:10EC40009500AE97BA9708DC5CDCCE8552859700BC
:10EC50000000E780A0DC99E023220404A1679387E9
:10EC6000B70348003EC42302010002C697E0FFFF3D
:10EC7000E7808005A9BF814701481CDC232E0403DF
:10EC8000E9B71733FFFFE702834597C0FFFFE7802F
:10EC90002034E1473305F502914597500000E780A5
:10ECA00000C5E55711C59777FF1F23A1A708814726
:10ECB0003E851733FFFF6700C34485471777FF1F63
:10ECC0002308F70682801733FFFFE7024341977757
:10ECD000FF1F9387670580433DC0835704046390FB
:10ECE000A70683572404639CB7043689B28497C06F
:10ECF000FFFFE78080AB5C5C63C3B7046395B7003C
:10ED00001C5C63EEA7028347640463F3F400A687E8
:10ED10002303F4048347740463F39700A687A303D3
:10ED2000F4048357440441677D176385E700850732
:10ED30002312F4043C4481C7CA8526858297173381
:10ED4000FFFF6700033C9777FF1F9387E7FD9C4316
:10ED5000014599C303C5870082801733FFFFE7028F
:10ED600003380111B70707003EC683C79500584D09
:10ED70000AC493F7F7070AC8A384F5002A89AE846A
:10ED800011CB1C4283C707002304F70097900000B3
:10ED9000E7800034216493055402280097B0FFFFF8
:10EDA000E780802397000000E78020FAAA852800EA
:10EDB00097D0FFFFE780A00A300001478146A68573
:10EDC0004A8597B0FFFFE780804613044402480855
:10EDD00022CC230A010002CE97E0FFFFE780C0EEBD
:10EDE00005611733FFFF6700C3311733FFFFE702E9
:10EDF000032F01117C003ECAB70707003ECC7C0000
:10EE00003ECE83C795002E84AA8493F7F707A38488
:10EE1000F500A16593855502480897B0FFFFE7808C
:10EE2000A01B97000000E78040F2AA85480897D011
:10EE3000FFFFE780C002500801478146A285268572
:10EE400097B0FFFFE780A03E05611733FFFF670023
:10EE5000432B9777FF1F938727ED9C43094599C361
:10EE600003C5970082809777FF1F9387E7EB9C434A
:10EE7000094599C303C5D70082809777FF1F938701
:10EE8000A7EA9C43014599C303C5A70082801733B5
:10EE9000FFFFE70223230111B70708003EC683C71F
:10EEA0009500404D0AC493F7F7070AC8A384F500FC
:10EEB0002A89AE8429C41442854703C7060063E04B
:10EEC000E70A83479400094681496380C702B30774
:10EED000F740A304E400B339F00083C7160023050C
:10EEE000F40097900000E780A01E03572403058BD1
:10EEF00019C76386090097D00000E78000E9216404
:10EF000093058402280097B0FFFFE780E00C97008C
:10EF10000000E78040F4AA85280097D0FFFFE78033
:10EF200000F497000000E78080F5AA85280097D0BC
:10EF3000FFFFE780C0F2014781463000A6854A8581
:10EF400097B0FFFFE780A02E13047402480822CC7C
:10EF5000230A010002CE97E0FFFFE780E0D60561BB
:10EF60001733FFFF670043191733FFFFE70223172B
:10EF700001117C003ECAB70708003ECC7C003ECEA3
:10EF800083C795002E84AA8493F7F707A384F5001E
:10EF9000A16593858502480897B0FFFFE780C0030D
:10EFA00097000000E78020EBAA85480897D0FFFF74
:10EFB000E780E0EA97000000E78060ECAA85480857
:10EFC00097D0FFFFE780A0E9500801478146A2855E
:10EFD000268597B0FFFFE780802505611733FFFF87
:10EFE000670023129777FF1F938707D49C4301453F
:10EFF00099C303C5B70082801733FFFFE702230ED2
:10F000000111B70707003EC683C79500404D0AC4EB
:10F0100093F7F7070AC8A384F5002A89AE8405C8C8
:10F020001C42054783C707006368F7060347B4001F
:10F03000630FF700A305F40097900000E7804009F4
:10F040008347B400B9CF97D0FFFFE78040BE21646B
:10F050009305B400280097B0FFFFE780E0F7970022
:10F060000000E78060F8AA85280097D0FFFFE780BE
:10F0700000DF014781463000A6854A8597B0FFFF33
:10F08000E780E01A2904480822CC230A010002CEB6
:10F0900097E0FFFFE78040C305611733FFFF67007C
:10F0A000430697D0FFFFE78020BF55B71733FFFF18
:10F0B000E702E30201117C003ECAB70707003ECC1D
:10F0C0007C003ECE83C795002E84AA8493F7F70771
:10F0D000A384F500A165AD05480897B0FFFFE78060
:10F0E000A0EF97000000E78020F0AA85480897D09D
:10F0F000FFFFE780C0D6500801478146A2852685DC
:10F1000097B0FFFFE780A01205611733FFFF67008C
:10F1100043FF9777FF1F938727C19C43094599C3F6
:10F1200003C5C70082801733FFFFE70243FB0111CD
:10F130007C00AE843ECAA165B70707002A843ECC96
:10F14000D1057C0048083ECE97B0FFFFE780C0E8BD
:10F1500097000000E78020FCAA85480897D0FFFFB1
:10F16000E780E0CF500801478146A685228597B009
:10F17000FFFFE780C00B05611733FFFF670063F8EF
:10F180001733FFFFE702A3F583C7950093F7F7074F
:10F19000A384F50097000000E78020F91733FFFFF4
:10F1A000670023F61733FFFFE702C3F183C795001B
:10F1B0000329C501411193F7F707A384F5001C4209
:10F1C00083C90700854763E637079777FF1F938753
:10F1D000A70C9C432E84AA8485CF97000000E7806B
:10F1E00080F389476306F502630409028347C90077
:10F1F000638037032306390197900000E78040EDD4
:10F2000083572903898B89C797D00000E780E0B72F
:10F210002685A28597000000E78020F1A167CD0731
:10F2200048003EC42302010002C697E0FFFFE780CA
:10F23000A0A941011733FFFF670003EC9777FF1F79
:10F24000938787AE9C431D4599C303C5E700828021
:10F250001733FFFFE702A3E80111B70707003EC617
:10F2600083C79500584D0AC493F7F7070AC8A384CB
:10F27000F5002A89AE8415C71C4283C70700939600
:10F280008701E18663C4060685466381D706834607
:10F29000E7006388F6002307F70097900000E780F7
:10F2A00020E321649305E400280097B0FFFFE78086
:10F2B000A0D297000000E780A0F8AA85280097D088
:10F2C000FFFFE780C0B9014781463000A6854A8527
:10F2D00097B0FFFFE780A0F53504480822CC230A49
:10F2E000010002CE97E0FFFFE780009E0561173323
:10F2F000FFFF670003E11733FFFFE70243DE011161
:10F300007C003ECAB70707003ECC7C003ECE83C7D8
:10F3100095002E84AA8493F7F707A384F500A165CE
:10F32000B905480897B0FFFFE78000CB97000000C1
:10F33000E78000F1AA85480897D0FFFFE78020B258
:10F34000500801478146A285268597B0FFFFE780D8
:10F3500000EE05611733FFFF6700A3DA1733FFFFE5
:10F36000E70243D6AA8401441779FF1F1309099CB9
:10F37000E14997C0FFFFE780A0C56344A4000145B1
:10F3800019A833053403832709003E9583572500C8
:10F390006397970011051733FFFF6700E3D5050456
:10F3A000C9BF032E8500630A0E121773FF1F1303D4
:10F3B000A3B60323030063150300294363900612D9
:10F3C00003234E01631503001D4363990710173390
:10F3D000FFFFE70243CEC689428A3E89BA8AB684D5
:10F3E000328BAE8B2A84B5E103554E0019E50143FB
:10F3F0001A851733FFFF670083CFA167A98F1167B5
:10F4000063FBE70097000000E78080F5814597F0F7
:10F41000FFFFE780C0120844B70700E05841F98FAA
:10F4200018455CC1B707001FF98F1CC55C4991C71F
:10F43000610597E00000E780408BE38A09FA2285A6
:10F4400097900000E78060C65DB7328597C00000E6
:10F45000E78040430D4349DD1C44116703D5470055
:10F46000A167A98F63FBE70097000000E78040EFEA
:10F47000814597F0FFFFE780800C032384009316FB
:10F480004B01D1828347B300035663008588FD8B0F
:10F49000A305F300FD777D8E558EFD76FD16B20433
:10F4A000F18E83274301C58E231273012313D300EA
:10F4B0002304530123052301A3044301BDDF228557
:10F4C00097B0FFFFE78080C9AA850844B5D16105E0
:10F4D00097D00000E780207F8DB71D431A8582807A
:10F4E0001733FFFFE70203BE0569AA84AE89328A9B
:10F4F0000144FD5A7D1997C0FFFFE78020A26347B2
:10F50000A40001451733FFFF670003BFD8449317DA
:10F510001400BA9703D70700631F370323905701DE
:10F5200063070A00268597900000E780A0809C442E
:10F530009DC383D76700B3F72701639E3701D28845
:10F54000014881470147814601468145268597004C
:10F550000000E78040E5050479BF1733FFFFE702AD
:10F5600063B679711C103EC4B7070F003EC61C106D
:10F570003EC883C79500AA8A328593F7F707A3840C
:10F58000F5002E89328497D0FFFFE780009D931706
:10F590000501C187635AF006AA89228597D0FFFF2B
:10F5A000E780A09B2A8A4E85032B040097B0FFFFBB
:10F5B000E780609739ED8357440081440544F11793
:10F5C00093B71700A303F10083457100DA87228700
:10F5D000D2864E86280097E0FFFFE780E05701477C
:10F5E00081463000CA85568597B0FFFFE78020C46A
:10F5F000A1679387F70348083ECC230A810026CEF3
:10F6000097D0FFFFE780406C45611733FFFF67002D
:10F61000A3AEA2851306710097E0FFFFE780606646
:10F62000AA84094455D1528597E0FFFFE78060D452
:10F630000D4459D90546D285268597000000E780FC
:10F6400060EA2A8451B71733FFFFE70243A98355C5
:10F6500007000346270041112A842E8532C62EC496
:10F6600097E0FFFFE780E0D001C93246A24522853E
:10F6700097000000E78000E741011733FFFF6700B4
:10F6800043A81733FFFFE70203A383C79500411187
:10F69000AA8A93F7F707A384F5003285AE893284EE
:10F6A00097D0FFFFE780608B93170501C1876357F1
:10F6B000F00AC1452A8A228597C0FFFFE780807043
:10F6C0002A8D228597D0FFFFE78020892A8922850D
:10F6D00097D0FFFFE7804086930705F893F7F70F71
:10F6E0001307E007AA8B637BF706228597D0FFFFFD
:10F6F000E78080842A8C228597D0FFFFE780C08333
:10F70000AA8C5285032B040097B0FFFFE780A081ED
:10F7100039E983574400231101008144F11793B75D
:10F720001700A300F1000544034711008356210090
:10F73000938784005685DA8822885286CE8597F092
:10F74000FFFFE78020A7A167E90748003EC4230226
:10F75000810026C697D0FFFFE7800057410117338D
:10F76000FFFF6700C39813061100A28597E0FFFF13
:10F77000E7802051AA8409E52311010009446DB7EF
:10F78000930521006A8597F0FFFFE780A0F02A84A7
:10F7900041FD835521009356C90013164901854840
:10F7A0006688E2875E87858A5182268597000000F9
:10F7B000E78060BF2A848DBF1733FFFFE702A38F66
:10F7C00083C7950041112A8B93F7F707A384F500AF
:10F7D0003285AE89328497C0FFFFE78000789317A7
:10F7E0000501C1876352F00A2A8A228597C0FFFF6C
:10F7F000E780A076AA8A228597C0FFFFE780E075A0
:10F800002A89228597C0FFFFE7800073930705F8D8
:10F8100093F7F70F1307E0072A8C6377F706228523
:10F8200097C0FFFFE7804071AA8C228597C0FFFF39
:10F83000E78080702A8D5285832B040097A0FFFFFC
:10F84000E780606E39E58357440085440144F11731
:10F8500093B71700A301F100034731009307840019
:10F860005A85DE882688D6865286CE8597F0FFFF99
:10F87000E78040948D4748003EC42302910022C691
:10F8800097D0FFFFE780404441011733FFFF670037
:10F890000386A2851306310097E0FFFFE780603EF4
:10F8A0002A84894455D99356C900131649018548BD
:10F8B0006A88E6876287858A5182D685970000002C
:10F8C000E78060AEAA8449BF1723FFFFE702837F6A
:10F8D0002A8981440144617A916A176BFF1F130BD7
:10F8E000AB6397B0FFFFE780606463C7A400228525
:10F8F0001733FFFF670043808327090093991400A3
:10F90000CE9703D50700330745014207418363645F
:10F91000570305C103270B0019C785453E8597404E
:10F920000000E78060E9832709000504CE97239053
:10F93000070085047DB797000000E78060A2832759
:10F9400009000504CE972390070065D5814597F0FF
:10F95000FFFFE780C0BEF1BF1723FFFFE7028376FA
:10F9600083C7950041112A8A93F7F707A384F5000E
:10F9700032852E89328497C0FFFFE780005E93179F
:10F980000501C187635AF004AA89832A040097A05D
:10F99000FFFFE780405931E5835744008544014427
:10F9A000F11793B71700A301F10003483100D68780
:10F9B00052850147CE862686CA8597D0FFFFE7800D
:10F9C000806AA167F50748003EC42302910022C661
:10F9D00097D0FFFFE780402F41011723FFFF67000B
:10F9E000A371A2851306310097E0FFFFE78060292D
:10F9F0002A8489445DD99767FF1F9387E7519C4309
:10FA000081CF044997B0FFFFE7804052AA85268541
:10FA100097400000E78040DA1305040197000000DA
:10FA2000E780C0EA228597800000E78000338144A8
:10FA3000ADBF1723FFFFE702036883C7950041119D
:10FA4000AA8A93F7F707A384F5003285AE8932843A
:10FA50002311010097C0FFFFE78020509317050195
:10FA6000C1876354F0062A8AC145228597C0FFFFEB
:10FA7000E7804035AA8B5285032B040097A0FFFF37
:10FA8000E780604A21E98357440085440144F11727
:10FA900093B71700A300F10003481100035721009A
:10FAA000DA875685D2862686CE8597D0FFFFE780F7
:10FAB000805BA1679387270248003EC42302910020
:10FAC00022C697D0FFFFE780202041011723FFFFC8
:10FAD0006700E361A2851306110097E0FFFFE7804E
:10FAE000401A2A8489444DD99767FF1F9387C742DC
:10FAF00098433E8901CF044997B0FFFFE780004358
:10FB0000AA85268597400000E78000CB13050401F5
:10FB100097000000E78080DB97B0FFFFE78000419F
:10FB200095443DD9930521005E8597F0FFFFE7805E
:10FB300060B6AA8435F11C48035721002285239022
:10FB4000E70097800000E780402183270900A9D7BC
:10FB50000355210097400000E780A0BD35BF172363
:10FB6000FFFFE702435583C795004111AA8A93F727
:10FB7000F707A384F5003285AE89328497C0FFFF72
:10FB8000E780A03D93170501C1876351F0062A8ADB
:10FB9000228597C0FFFFE780403C2A895285032BCE
:10FBA000040097A0FFFFE780003831E58357440049
:10FBB00085440144F11793B71700A301F1000348EE
:10FBC0003100DA8756854A87D2862686CE8597D039
:10FBD000FFFFE7804049A167F90748003EC42302C0
:10FBE000910022C697D0FFFFE780000E4101172346
:10FBF000FFFF6700C34FA2851306310097E0FFFFA8
:10FC0000E78020082A8489445DD99167CA97C20792
:10FC10001167C1831307F7EF8544E362F7FA97672B
:10FC2000FF1F9387672F9843BE8B01CF044997B07E
:10FC3000FFFFE780A02FAA85268597400000E78078
:10FC4000A0B71305040197000000E78020C897B013
:10FC5000FFFFE780A02D95443DD11C4822858144BB
:10FC60002390270197800000E780200F83A70B00D7
:10FC7000B9D74A8597400000E780A0AB89B7172322
:10FC8000FFFFE702C3452A844105B28497000000C4
:10FC9000E780C0C311C5228597800000E780E00B94
:10FCA00081460146A685228597800000E780C04EE8
:10FCB0001C4C89C7DC4799C3228582971723FFFF15
:10FCC000670023449767FF1F938707069C430145FE
:10FCD00099C31385070182809767FF1F9387C70425
:10FCE000884382801723FFFFE702633F9317C60014
:10FCF000DD8DC2054111C1812A8432C697C0FFFF44
:10FD0000E780E0173246228511829375F60F97C07F
:10FD1000FFFFE780C01441011723FFFF6700633E28
:10FD20001723FFFFE702033A79713C083ED2B70779
:10FD30000C003ED43C083ED683C79500AE842A8989
:10FD400093F7F707A384F500A16593853504481060
:10FD500097A0FFFFE7804028C165FD150144176AA1
:10FD6000FF1F130AEA1C930A400EAE892E8B2EC683
:10FD700097B0FFFFE780801E420593170401418181
:10FD8000C183B24563E9A702C167FD176387F50028
:10FD9000481097C0FFFFE780800E50100147814652
:10FDA000A6854A8597A0FFFFE78060484561172335
:10FDB000FFFF670063343307540383270A0BBA97A6
:10FDC00003D6C701630A3601638A350148109700DC
:10FDD0000000E78060F1DA85050451BFB285EDBF10
:10FDE0001723FFFFE702232D79717C083EC8B70770
:10FDF00011003ECA7C083ECC83C79500AA89328593
:10FE000093F7F707A384F5002E8997C0FFFFE780DB
:10FE1000C01485676378F504A165AA84890508087C
:10FE200097A0FFFFE780401B268597400000E780F2
:10FE300060ED133415000A04A285080897C0FFFF7F
:10FE4000E780E001A685080897C0FFFFE780200350
:10FE500025CC014781461008CA854E8597A0FFFF33
:10FE6000E780E03C45611723FFFF67004328B307A5
:10FE700054030327CA0ABA9703D70700631C9700E5
:10FE800003D6270063806505080897000000E78017
:10FE9000A0E5DE8505042EC697B0FFFFE780000DC4
:10FEA0004205931704014181C183B245E3E1A7FCF8
:10FEB000C167FD17E38FF5F8080897C0FFFFE780DB
:10FEC00000FC41BFB285F9B7C165FD150144176A51
:10FED000FF1F130AEA05930A80022E8BAE8B65BFC3
:10FEE0001723FFFFE702A31F18418347170083462C
:10FEF0000700A207D58FD207D1832390F50083474F
:10FF00002700034717008D45A207D98F918323103F
:10FF1000F60097C0FFFFE780A0E91723FFFF670007
:10FF2000431E1723FFFFE702E319C1640144176969
:10FF3000FF1F1309E9FF93098002FD1497B0FFFF2B
:10FF4000E780C0026347A40001451723FFFF670055
:10FF5000A31A330534038327C90A3E958357050046
:10FF6000E38597FE0504D9BF1723FFFFE70283153A
:10FF70002A8AAE89B284B68A97400000E78080D88A
:10FF800019E591473E851723FFFF6700E3162A898D
:10FF90004E8597C00000E780E08E2A84638E0A04B5
:10FFA0008D476DD103570500C547E31D47FD034746
:10FFB000F9018546AD47E317D7FC8347450081CF5C
:10FFC0004146A6855D0597F00000E780C09E814709
:10FFD00055D9AD4745BF130965012302E500CA8520
:10FFE000268597100000E780606231C1A547E38B4A
:10FFF0000AF82302040079B705C183570500E3928C
:020000040001F9
:1000000047F94146A685190597F00000E780A09AB8
:1000100081472DD99947BDB74E8597000000E780ED
:1000200080F02A84954739DD130955004DBF4146BC
:10003000A68523104401231134011305190097F0FC
:100040000000E780A099228597800000E780A0EA61
:1000500081470DBF1723FFFFE702630879717C001A
:100060003ECCB7070A003ECE7C003ED083C7950049
:10007000B2842E8493F7F707A384F5001306A1003A
:100080002A892C00268597000000E780A0E5A1655D
:1000900028088D0597A0FFFFE78000F49040835566
:1000A000A10003558100854697000000E78000EC21
:1000B000AA84AA85280897C0FFFFE78040DA035684
:1000C000A10083558100280897000000E780C0C187
:1000D000300801478146A2854A8597A0FFFFE78047
:1000E0000015854748103ED42302910202D697D0CE
:1000F000FFFFE78060BD45611723FFFF67006300D6
:100100001723FFFFE702A3FD79717C003ECCB70700
:100110000A003ECE7C003ED083C79500B2842E8478
:1001200093F7F707A384F5001306A1002A892C0092
:10013000268597000000E780E0DAA16528088D0594
:1001400097A0FFFFE78040E990408355A100035549
:100150008100814697000000E78040E1AA84AA85DB
:10016000280897C0FFFFE78080CF0356A100835582
:100170008100280897000000E78000B73008014799
:100180008146A2854A8597A0FFFFE780400A481074
:100190002302910202D402D697D0FFFFE780C0B2BB
:1001A00045611723FFFF6700C3F51723FFFFE70231
:1001B00003F397000000E78060DB1723FFFF670071
:1001C00043F49767FF1F938767B68843828017239E
:1001D000FFFFE702C3F0835725004111AE842A8454
:1001E0002307B10017F5FFFF130525466C00231602
:1001F000F10097A0FFFFE780804591C4228597809A
:100200000000E780E0D6FD572310F400130620021B
:100210008145130554009720FFFFE78040EF41011F
:100220001723FFFF6700E3ED1723FFFFE70283E9D2
:1002300079717C003ECCB7070A003ECE7C003ED0F0
:1002400083C79500AA89AE8493F7F7073285A38404
:10025000F5001306A1002C0097000000E78080C87D
:1002600003558100114497400000E780A0A915C5FF
:100270000355A100014497B00000E780A06011CDB4
:10028000035705008357810045446318F7008545EF
:1002900097000000E780E0F30144216993053900ED
:1002A000280897A0FFFFE78020D3A285280897C0E1
:1002B000FFFFE780C0BA0356A100835581002808DC
:1002C00097000000E78040A2300801478146A685DC
:1002D0004E8597A0FFFFE78080F548104AD423029F
:1002E000810202D697D0FFFFE780009E4561172369
:1002F000FFFF670063E01723FFFFE702A3DC9767B8
:10030000FF1F938767A22A8488432E8915C5035748
:1003100045038357C4016311F702232605022318FE
:100320000502410597D00000E780209C6306090084
:1003300097800000E78060DB81449769FF1F938905
:1003400029BF130A800297B0FFFFE78020C263C471
:10035000A4049767FF1F9387E7A59C4399C703559C
:10036000C40197200000E780C0BD63070900228513
:1003700097800000E780C0A01306400E81452285CB
:100380009720FFFFE780A0D8FD57231EF400172316
:10039000FFFF670063D63385440383A7C90A3E95F0
:1003A000035705008357C4016317F700CA859700F8
:1003B0000000E78000E2850479B71723FFFFE7021A
:1003C00063D083C795004111AA8993F7F707A384E7
:1003D000F5003285AE8497C0FFFFE78000B88567DF
:1003E0006378F5042A8997400000E780A0910144D2
:1003F00001CD83D7040031446388270185459700E8
:100400000000E78080EF01444E85A2864A86A685DB
:1004100097D0FFFFE780A09CA1679387170448004F
:100420003EC42302810002C697D0FFFFE780C08947
:1004300041011723FFFF670023CC1723FFFFE702CB
:1004400063C89767FF1F9387278E804329C40145A0
:1004500097C00000E780002181470148C1641CDC8F
:10046000232E0403232004041769FF1F130949AC3A
:1004700001449309400EFD1497B0FFFFE78000AEE2
:10048000634FA400814517F5FFFF1305857F97A0F3
:10049000FFFFE780C01B1723FFFF6700E3C533059D
:1004A00034038327090B3E958357C5016387970063
:1004B000854597000000E78040E4050475BF935729
:1004C000050113D78700A380F50093170501C183A9
:1004D000A1832380E5002381F500A381A50082800C
:1004E0001723FFFFE702A3BF2300050083C7150002
:1004F000A300F50083C725002301F50083C735005D
:10050000A301F50083C745002302F50083C755000A
:10051000A302F50083C7650093059500A3030500BA
:100520002303F50023040500328597000000E780CF
:1005300040F91723FFFF6700C3BC1723FFFFE70243
:1005400063B84111E9540DCD85CD93F9C5FF2E84D3
:100550002A89AA84338AA900B7EA040063189A0298
:100560000D88854411CCB7E704009C5F82972AC6AA
:1005700022866C003305390197E00000E7800046D1
:10058000268541011723FFFF670003B783A78A036E
:100590009104829793170501C183A183A38EF4FE72
:1005A00093570501238FF4FEA183238EA4FEA38F0E
:1005B000F4FE6DB763E6D5021723FFFFE70223B20F
:1005C000B28741113686BE8536C697E00000E780C7
:1005D000E040B246410136851723FFFF670063B252
:1005E000814636858280838705001387F5003D05A7
:1005F000FD8793F77708834607007D158606B58F3C
:10060000A300F5006307B7007D17834717009D839C
:10061000DDB782801723FFFFE70263ACB7E7040072
:1006200083A7070932872A863A85829713351500F2
:100630001723FFFF6700E3AC15C181478DC1172366
:10064000FFFFE702C3A9414697E00000E7800039B9
:1006500085473E851723FFFF6700A3AA81473E8594
:1006600082801DCD1723FFFFE70263A74146814526
:100670002A849720FFFFE78080A941468145130522
:1006800004039720FFFFE78080A80147C16723226A
:10069000040438C87CC805451723FFFF670063A61C
:1006A0000145828081473DCDB5CD1723FFFFE7028D
:1006B00003A3B2842E891306800581452A849720DE
:1006C000FFFFE780C0A4CA8524C4268597000000E8
:1006D000E780C0F64146814522859720FFFFE780ED
:1006E00000A33044A285228597000000E780C0F275
:1006F00093040401A285268597000000E780E0EEC0
:10070000A6851305040297000000E78000EE22850D
:1007100097000000E78020F585473E851723FFFFFF
:100720006700239E3E8582801723FFFFE70283999F
:100730004111E9540DCD85CD93F9C5FF2E842A8949
:10074000AA84338AA900B7EA0400639844030D8899
:10075000814411CCB7E704009C5F82972AC62286A9
:100760006C003305390197E00000E78020272685DB
:1007700041011723FFFF6700239883A78A03910491
:10078000829793170501C183A183A38EF4FE93572B
:100790000501238FF4FEA183238EA4FEA38FF4FE14
:1007A0006DB765CD1723FFFFE702C391B28411E651
:1007B00005451723FFFF670023942A842E890145EE
:1007C000EDD93C487848B3E6E700E5D69386F7FFD5
:1007D000B3B7F6007D17032A4404BA9734C87CC81F
:1007E00063050A06C14913050A03B38949412295E5
:1007F000637D3601B2862E86A68597000000E780CD
:10080000A0DB7C40BE9464C065B7CE862E86CE85C4
:1008100097000000E78040DAC114D2944E99232259
:100820000404A2879306040103C7070003C6070355
:100830008507318FA38FE7FEE398F6FE3044A2854B
:10084000228597000000E78020DD2699C149330604
:10085000994063EC9900A9DCA686A68513050403DC
:1008600097000000E78040D579BF8147B306F400C8
:100870003307F6000347070083C5060085072D8F61
:100880002380E600E39437FF3044A2852285970059
:100890000000E78060D8C1145DBF014582800DC1B2
:1008A0001723FFFFE702A3831306800581459720E6
:1008B000FFFFE780C08505451723FFFF67006384BE
:1008C00001458280814749C5C1C51723FFFFE70263
:1008D0000381FC4141462E84AA846399C704138690
:1008E0000501A2878146C14503C7070003C5070369
:1008F0008507298F3305D600034505008506298F16
:10090000A38FE7FEE392B6FE3044A28526859700CA
:100910000000E78060D0228597000000E78060F843
:1009200085473E851713FFFF6700A37D13850703E7
:100930001D8E814522959710FFFFE780407D7C400A
:10094000130700F813060402A2972388E70251BF99
:100950003E8582801713FFFFE70263786D712E8456
:10096000B284AA8590102800368997000000E7809D
:10097000A0D309EDD55725A050400C402800970082
:100980000000E78040E27DD5FD142104F5F42C0041
:100990004A8597000000E78020F3814761DD3E85AE
:1009A00051611713FFFF6700C3751713FFFFE702BD
:1009B000037341112EC432C62C0005469700000077
:1009C000E78080F941011713FFFF67008373171356
:1009D000FFFFE702C37001112A842EC602C802CAB3
:1009E00002CC02CE97E00000E780C023B2462A8600
:1009F000A285080897000000E78060FB1375F50FDB
:100A000005611713FFFF6700C36F1713FFFFE702AE
:100A1000036D7971B2872A8421462308B10013053A
:100A20001101BE853AC436C697E00000E78000FB9E
:100A3000B24693059101368597000000E78060A8D3
:100A40002285141035460C0897000000E78020F638
:100A50002A84224701E921460C103A8597E00000DC
:100A6000E780C0F7228545611713FFFF67006369C0
:100A70001713FFFFE702A3667171AE84AA850A858A
:100A8000328497000000E78060BB11C90A86A68502
:100A9000228597000000E78020B8814711E1C54713
:100AA0003E854D611713FFFF6700A3651713FFFF16
:100AB000E702E35F1D712A8AB289BE843546854705
:100AC000130511012E8CB68A3A8BC28C468D2308F1
:100AD000F10097E00000E78060F010100C085285EC
:100AE000231F010097000000E780C0F82A843DED35
:100AF000A1476313FD089307900591E0E54735464C
:100B0000E2851305110113990A012308F100135915
:100B1000090197E00000E78060EC13578900939784
:100B20008A00D98F90080C085285231FF100970086
:100B30000000E78020F42A8415E9A1E49387FA00F5
:100B400091831379F9003EC6631309004149668B0E
:100B50008144C14B854DB247639F970C6A868C00D8
:100B600033855C0197E00000E78040E7228525613E
:100B70001713FFFF6700635793079004C9F0A54759
:100B8000BDBF834701050947C14B2308F1008347D7
:100B90001105A58FA308F10093872400814463E128
:100BA000FB04014714083386E6008C08B386E40092
:100BB000BA95DA9683C6060083C505000507AD8E93
:100BC0002300D600E390E7FE4147639CE7049008CA
:100BD0000C08528597000000E780C0E925D181A06C
:100BE000B3069B00BA871008B305F60090083E963E
:100BF00003C506000346060085078506298E238067
:100C0000C500E39277FF998F90080C085285BE9437
:100C100097000000E78000E68947014749D12A8410
:100C2000B1B790083E96034606001408BE9623808E
:100C3000C600850759BFB24785046387971481476B
:100C40001808B306F70098083E973386F900034763
:100C50000700034606008507318F2380E600E391F5
:100C600077FF90080C08528597000000E78080E02D
:100C70005DF53546E285130511012308B10197E0C2
:100C80000000E780A0D51397040141839397840067
:100C90002183D98F10180C085285231FF10097006B
:100CA0000000E78020DD25FD814710183387F9001B
:100CB0003E960347070003460600B306FB00850780
:100CC000318F2380E600E39277FF65A81808B3060A
:100CD000F70098083E973386F9000347070003465C
:100CE00006008507318F2380E600E3E127FFCA87EE
:100CF000639E770990080C08528597000000E780F2
:100D000060D711FD81479800B306F70090081810CE
:100D10003E973E9603470700034606008507318F3E
:100D20002380E600E39177FF3546E2851305110144
:100D30002308B10197E00000E78040CA139704013F
:100D40004183939784002183D98F10180C08528512
:100D5000231FF10097000000E780C0D1E31105ECEC
:100D6000814710183387F9003E9603470700034672
:100D70000600B306FB008507318F2380E600E3E21F
:100D800027FFC109410BC1BB814785B79408BE96B7
:100D900083C6060018083E972300D700850789BF41
:100DA000638006321713FFFFE702633059712A840C
:100DB000BE89B28B85473546130511022E8B468CB2
:100DC0004289BA8A368A2300F10297E00000E78060
:100DD000E0C010180C1022852317010297000000B4
:100DE000E78040C963180512A147631FFC069307FB
:100DF000900563930900E5473546DA85130511022E
:100E000093140A012300F102C18097E00000E780FB
:100E1000E0BC93178A0013D78400D98F90080C1078
:100E200022852317F10297000000E780A0C47DE12E
:100E3000639209049307FA00BD88918391E0C1444D
:100E4000C207C183DE8C814A3EC6414DB24763E290
:100E5000FA0E6286B3854B01881097E00000E780A8
:100E600080B54DC93D557DA093079004E39609F8E0
:100E7000A54759B7834701050947C14C2300F10233
:100E800083471105B3C7F900A300F1029387290036
:100E9000814963E1FC04814618103306D7008C08B1
:100EA0003387D900B69556970347070083C50500D9
:100EB00085062D8F2300E600E390D7FE414763901F
:100EC000E70690080C10228597000000E78080BAA2
:100ED00035D189A0B3863A01BA871010B305F60060
:100EE00090083E9603C50600034606008507850662
:100EF000298E2380C500E39297FF3387EC4090084A
:100F00000C102285BA9997000000E780A0B68947A7
:100F1000014741D165611713FFFF6700031D90086A
:100F20003E96034606001410BE962380C600850731
:100F300079B7B247850A93990A01939D8A0093D99C
:100F400009016391570F85473546DA85130511026C
:100F50002300F10293D9890097E00000E78000A800
:100F6000B3ED3D0190000C1022852317B1039700CB
:100F70000000E78020B059FD8147A68963EA970603
:100F800026860C084A8597E00000E78020A5814767
:100F90001810B306F700100898083E973E960347CE
:100FA0000700034606008507318F2380E600E3E152
:100FB00097FE639FA90590080C10228597000000FA
:100FC000E78040AB21F981479810B306F7009008FD
:100FD00018183E973E96034707000346060085070C
:100FE000318F2380E600E391A7FF4109C10CB9BD11
:100FF00018089000B306F7003E963387FC000347BD
:101000000700034606008507318F2380E600B5B749
:1010100098084E97034707001C10CE972380E700DF
:10102000850941BF85473546DA851305110223003E
:10103000F10293D9890097E00000E780209AB3ED90
:101040003D0190000C1022852317B103970000008A
:10105000E78040A2E31005EC814718089000B30632
:10106000F7003E963387FC0003470700034606005F
:101070008507318F2380E600E391A7FF41460C08E6
:101080004A8597E00000E780609581471810B30615
:10109000F700100898083E973E960347070003465E
:1010A00006008507318F2380E600E391A7FF9008B3
:1010B0000C10228597000000E780C09B1DD599BDCC
:1010C0007D5582801713FFFFE702630101112A8417
:1010D0002E8593055100328902C002C202C402C6A5
:1010E0009304740097F0FFFFE780A03D1D46A6859E
:1010F0001305910097E00000E780408E10088A8574
:101100004A8597000000E780E09619ED93071400E8
:10111000180883C607000346070085070507B18E38
:10112000A38FD7FEE397F4FE05611713FFFF670057
:1011300043FD1713FFFFE702E3F82E848C414111B2
:10114000AA89838715003289914463D30700A1449B
:101150009757FF1F938747149C43A1C7C1CA8D4768
:101160002310F10083C725004A852301F10083C7BE
:101170003500A301F10083C745002302F10083C7B6
:101180005500A302F10083C7650093059100A303F6
:1011900001002303F1002304010097F0FFFFE78023
:1011A00040320C404A860A8597F0FFFFE780803383
:1011B0000328040083564400A6881D088147014780
:1011C000E51642868A854E8597000000E780408EAE
:1011D0002A8919E5A685228597B0FFFFE780E0C13F
:1011E0004A8541011713FFFF670003F14A860A850C
:1011F00097F0FFFFE780002F6DB71713FFFFE7029F
:1012000063EC2E848C414111AA89838715003289B1
:10121000914463D30700A1449757FF1F9387C707E3
:101220009C43A1C7C1C68D472310F10083C7250089
:101230004A852301F10083C73500A301F10083C76C
:1012400045002302F10083C75500A302F10083C7C4
:10125000650093059100A30301002303F10023041B
:10126000010097F0FFFFE780C0250C404A860A8501
:1012700097F0FFFFE780002783564400032804000F
:101280008A85858EC2061D08C1822312D400A688D5
:1012900081470147E51642864E8597000000E780AA
:1012A00060B041011713FFFF670003E54A860A8516
:1012B00097F0FFFFE78000234DBF1713FFFFE70202
:1012C00003E2B335B000011185052A891315F60133
:1012D000336515012308B1009305110136843AC620
:1012E00032C03EC442C297F0FFFFE780801DA24794
:1012F0001248425593D68700230BF10093059101C4
:1013000093578800A30AD100A30BF100230C01011D
:1013100097F0FFFFE780E01A3247024603280400F7
:10132000B337E000835644009207914411C2A144B0
:101330004A85A68842860C0897F0FFFFE780407731
:101340002A8919E5A685228597B0FFFFE780E0AAE4
:101350004A8505611713FFFF6700A3DA1713FFFF24
:10136000E70243D601113EC68647B335B000850576
:10137000AA891315F6015D8D2308B10093051101AB
:1013800036843A89B28442C446C297F0FFFFE780B0
:10139000401322489248164593578800A30AF1004B
:1013A0009305910193D78800230B0101A30BF10052
:1013B000230C110197F0FFFFE780A0103247104087
:1013C00083564400B337E000920703280900914890
:1013D00091C0A1480C084E8597000000E780809CD2
:1013E000AA8401E9835544004A8597B0FFFFE7804E
:1013F000C0A0268505611713FFFF6700E3CFAA95FC
:101400009307F00F170701001307075B6317B50079
:1014100013C5F7FF1375F50F828005058346F5FFA9
:10142000B58FBA9783C70700D5B703574500144156
:101430009307F00F17060100130606583697420768
:101440004183139506014181631BE500AD8FB2977F
:1014500003C50700130515F31335150082808506B3
:1014600003C5F6FFA98FB29783C70700D9BF17132B
:10147000FFFFE702C3C6B28736842E86BA86AA85E6
:101480003E85BA8497F0FFFFE7806052634F050006
:10149000228597D00000E780E0782A86A686A2857C
:1014A000268597F0FFFFE78080501713FFFF670046
:1014B00043C51713FFFFE702E3C05D712A8BAE8AB5
:1014C000170501001305C54C2C00B284368ABA8971
:1014D0003E8997F0FFFFE780C04F2A845DE134101A
:1014E0004146DA85280097F0FFFFE780404C2A84C8
:1014F00049E98547A303F100A6C2930771002408B8
:10150000BEC4A68685470D462C18281002DC02DED4
:10151000D6C0BEC697F0FFFFE78000442A8435E1BD
:1015200083477102A6860D4693F7F7072300FA005A
:10153000C1473EDE2C188947281026DCA303F100A2
:1015400097F0FFFFE78040412A8405ED4146A685DC
:101550004E8597D00000E78060488D47A6860D46EF
:101560002C182810A303F10097F0FFFFE780C03E7E
:101570002A8401E94146A6854A8597D00000E78084
:10158000E045228561611713FFFF6700E3B617137B
:10159000FFFFE702C3B497F700009387E7A09843E3
:1015A00083C7470079712A89AE84170501001305A6
:1015B000A53E0C083AC42306F10097F0FFFFE78030
:1015C00040412A8405ED14104146CA85080897F069
:1015D000FFFFE780C03D2A8415E1140815462C0062
:1015E000081097F0FFFFE780803C2A8401E921463C
:1015F0002C08268597D00000E780403E2285456173
:101600001713FFFF6700E3AF1713FFFFE70223ADD8
:1016100097F70000938747999C477971AA842E8495
:10162000170501001305C5370C083EC697F0FFFFEC
:10163000E780203A0DE914104146A685080897F086
:10164000FFFFE780C03605E1140811466C00081062
:1016500097F0FFFFE780A03519E58347F10193F785
:10166000F7032300F40045611713FFFF670063A928
:101670001713FFFFE702A3A63688A1488147014759
:10168000E54697F0FFFFE780A0421713FFFF6700D2
:1016900043A71713FFFFE70283A43688A1488147B9
:1016A0000147E54697F0FFFFE780C06F1713FFFF84
:1016B000670023A51713FFFFE70263A201112A8425
:1016C0002E850C0832C697F0FFFFE780803009EDC9
:1016D0003247970601009386262B1008C1452285C4
:1016E00097000000E780E0D805611713FFFF67004F
:1016F00043A11713FFFFE702839E4111C1472EC08C
:1017000032C48A8509463EC23EC697F0FFFFE78095
:10171000A02441011713FFFF6700A39E1713FFFFCB
:10172000E702E39B4111AE8613061009AA850A85DC
:1017300002C002C202C402C697F0FFFFE780202762
:1017400041011713FFFF6700C39B1713FFFFE70259
:101750000399328797060100938606252E86930506
:10176000000297000000E780C0D01713FFFF67005A
:1017700043991713FFFFE70283967971C1472ACC7B
:101780002ED032D42C080D4628003ECE3ED23ED676
:1017900002C402C602C802CA97F0FFFFE780C01B5E
:1017A00045611713FFFF6700C3951713FFFFE7029B
:1017B00003930111AA842E84170501001305451F08
:1017C0008A8597F0FFFFE780C02015E514084146A1
:1017D000A6850A8597F0FFFFE780601D09ED834726
:1017E000E1010347F101A207D98FCA07C9836177D5
:1017F000D98F2310F40005611713FFFF6700639072
:1018000015CD1713FFFFE702838D9747FF1F9387BF
:10181000675690439745FF1F938505561745FF1F51
:101820001305455197D00000E78000C51745FF1FFD
:10183000130545501713FFFF6700A38C1745FF1FC3
:101840001305454F82808DCD1713FFFFE7022389D3
:101850009747FF1F93870752944301112E840A86EE
:101860009745FF1F9385455197D00000E78040C6FC
:101870000A850294014505611713FFFF670063881D
:101880007D5582801713FFFFE702638597D0000024
:10189000E78080D19747FF1F23AEA74C17F5FFFFC6
:1018A0001305E5C997B00000E780C0741713FFFF68
:1018B000670023851747FF1F1307074E931715006F
:1018C00008433E95FD572310F50082801713FFFF54
:1018D000E702E3802A84084009E51713FFFF670049
:1018E00043821C4158401CC06313E5005CC0834721
:1018F000550023200500F99BA302F50097A0FFFFE8
:10190000E780207CC9BF1703FFFFE702A37B97474F
:10191000FF1F9387674A98432A8411CB834735007A
:1019200093F7070289C703550500894502971305F8
:10193000440197B00000E780403B83550400035505
:10194000E40097300000E780A00C485819C597A024
:10195000FFFFE7800077232A040213058403970022
:101960000000E780E0F68144B1499790FFFFE780EF
:10197000206A63CBA402834734002320040493F736
:1019800027FCA301F40000489790FFFFE78040691F
:1019900013161500814522859700FFFFE780207709
:1019A0001703FFFF67004375B3873403032904035C
:1019B00085043E994A8597000000E78060F1230482
:1019C000090065B78347350093F7070299E301459E
:1019D00082808357E500E39CB7FEC167FD1763165D
:1019E000F60005458280054599A81703FFFFE70229
:1019F000036F93170601C187B2842A840149635992
:101A0000F002835705009DCB01456367F60003454F
:101A100084003E953325A6001375F50F0DA01C48D4
:101A200013171900BA9783D70700E38E97FA0509B1
:101A30009790FFFFE780C05EE343A9FE01451703CF
:101A4000FFFF6700036C1703FFFFE702A367AE8980
:101A5000AA849790FFFFE78060522A8497D0FFFF07
:101A6000E780A02EAA86014713068401970500008F
:101A7000938585E41745FF1F130545329790FFFFB7
:101A8000E780E0182A8925C98C441304C500228503
:101A90009E0593F5050897A0FFFFE780403CCC40EA
:101AA00083877400E18163DD070493E505082285DF
:101AB00097A0FFFFE780A03A0D469385440022855A
:101AC00097A0FFFFE780C03683D50400228597A04A
:101AD000FFFFE780E03D83D52400228597A0FFFF2C
:101AE000E780003D03D6490083A50900228597A021
:101AF000FFFFE780E0334A851703FFFF6700C35FFE
:101B000093F5F5076DB71703FFFFE702435D01117A
:101B10002A84328532C697A0FFFFE780E0279780AE
:101B2000FFFFE780C030835704001747FF1F1307EC
:101B300027403246231BF100930700F8A30DF10064
:101B40001C471843231AA1008983858BB307F740EC
:101B5000B28548083ECE231C0100230D01009700EA
:101B60000000E78080EE05611703FFFF67006359FF
:101B70001703FFFFE7020355004101453DC49304ED
:101B8000C40026853289AE8997A0FFFFE780C02474
:101B900095452A8A2685035B040197A0FFFFE7800D
:101BA0002021268597A0FFFFE780603E8D45AA8A09
:101BB000268597A0FFFFE780A01F268597A0FFFF3F
:101BC000E780E03C5C48420A135A0A01D2975CC4A1
:101BD00023186401814763983A0146054D81330615
:101BE00025419337160013F5F70F1703FFFF670022
:101BF000A3501703FFFFE702034C89692A8BAE8BC2
:101C0000328AB68A81440144314CFD199790FFFF16
:101C1000E780004063CDA4009790FFFFE78040423B
:101C2000018D33B5AA001703FFFF6700434C3389CA
:101C3000840383270B003E9963170A0083478900BA
:101C400085043E94E1B703560A00DE854A8533F6E3
:101C5000C90097000000E780E0F16DD10545E1B7CC
:101C60001703FFFFE702A34701112A847C000355F5
:101C7000E5003ECAB70707003ECC7C003ECE972069
:101C80000000E78020082A898545480897A0FFFFC3
:101C9000E78020399945480897A0FFFFE780E015C5
:101CA000AA844A8597200000E780A0082380A4002A
:101CB0009747FF1F9387C7279C434166130606F08B
:101CC0009396870113D78701558F93D68700F18E9E
:101CD000558FA207B706FF00F58FD98F11462C004C
:101CE000138514003EC497D00000E78020CF500831
:101CF000A38204008945228597000000E780E0E088
:101D000019C9AA851305840397A0FFFFE780E03176
:101D10003C4085073CC005611703FFFF6700633E39
:101D20001703FFFFE702A33B9790FFFFE7804031D7
:101D30002A8405049790FFFFE780802F3305A402D3
:101D4000F14791453305F50297200000E78020BA5E
:101D500011E565551703FFFF6700A33A9747FF1F7B
:101D600023A4A7049790FFFFE780802D2A84050411
:101D70009790FFFFE780C02B3305A4028945060535
:101D800097200000E780A0B669D59747FF1F23A5DD
:101D9000A7009790FFFFE780A02A2A840504979068
:101DA000FFFFE780E0283304A4029747FF1F239733
:101DB00087FE9790FFFFE780A0282A849790FFFF77
:101DC000E7800027930714003385A7029747FF1F7A
:101DD0002397A7FC97070100938747811747FF1FA9
:101DE0002322F7FC0145BDB71703FFFFE702832D50
:101DF000AA842E8901449749FF1F93896913130A06
:101E000080069790FFFFE780A0226347A40001456A
:101E10001703FFFF6700432E3305440383A709021E
:101E20004A86A6853E9597000000E780E0B919E153
:101E30000504C1BF0545E9BF1703FFFFE702A3275C
:101E4000AA8A2E8BB28B368C3A8A8144014481490E
:101E5000974CFF1F938CCC0D130D80069790FFFFBE
:101E6000E780001D63C9A40011E085494E85170372
:101E7000FFFF6700C3273389A40383A70C025E8694
:101E8000D6853E994A8597000000E780E0B31DC1E2
:101E90009790FFFFE780C01A0544636D4501D28625
:101EA0006286DA851305090397000000E780A0D455
:101EB00011C1854985045DB71703FFFFE702832041
:101EC000C16441112A8901449749FF1F938949063A
:101ED000130A8006FD1436C632C42EC29790FFFF47
:101EE000E780001592452246B2466348A4000145AA
:101EF00041011703FFFF670023203305440383A735
:101F000009023E9509C683473500C18B9DC791C61E
:101F10008347350093F707028DC363069900835703
:101F2000E500639C27010357050001CB63E7E5004B
:101F300083478500BA97E3CDF5FA050469BF170317
:101F4000FFFFE7022318C1642A8901449749FF1F54
:101F5000938909FE130A8006FD149790FFFFE7801E
:101F6000200D6346A4001703FFFF6700E318330545
:101F7000440383A709023E958357E500638A9700CF
:101F8000630499006396270197000000E780E097BB
:101F90000504E1B71703FFFFE702631189692A8A85
:101FA000AE8A328BB68B8144174CFF1F130C4CF852
:101FB000930C8006314DFD199790FFFFE780400795
:101FC00063C6A4001703FFFF67002312338994033D
:101FD00083270C028355CA015A863E994A85970089
:101FE0000000E780609E31C1814D15A03384AD03B0
:101FF0008327090303D60B00D68533F6C9003E9428
:10200000228597000000E780E0B609E9850D9790EA
:10201000FFFFE780E0FFE3CBADFC01A8228597003E
:102020000000E780E08A23040400850471B71703E9
:10203000FFFFE70243084169AA8A014A174BFF1FC5
:10204000130B0BEF7D19C14B054C9790FFFFE780F9
:1020500020FE6346AA001703FFFF670043099309A8
:102060008006B3073A0383290B02BE9983D7E900A0
:10207000638E270163842A01639A570103A48903AD
:1020800001E84E8597000000E780C0BD050A75BFD6
:1020900083570401639977099304C400268597A0A8
:1020A000FFFFE78060D385452A8D2685835C040188
:1020B00097A0FFFFE780C0CF268597A0FFFFE780AE
:1020C000A0E762056185635905048D45268597A0C3
:1020D000FFFFE780E0CD8945268597A0FFFFE780D9
:1020E00020CD8945268597A0FFFFE78060CC8545F8
:1020F000268597A0FFFFE780E0CC834705000947CE
:1021000093F7F707639AE7009945268597A0FFFFA5
:10211000E78040CBA30285014848337D2D01231879
:1021200094016A9548C40040A1BF1703FFFFE7026E
:1021300003FB37E404008327041D82979747FF1FA2
:1021400083C707CC1715FF1F1305453EA300F500F5
:102150008327441C82978327841C81461306F00F33
:102160008145014582971703FFFF670083F91747F1
:10217000FF1F1307E7B818439745FF1F83C545C8DE
:102180009747FF1F938747C68346870303469703F6
:102190006397D5009747FF1F2384C7C6828083C5F6
:1021A00087010347A7036317B6009747FF1F2389DB
:1021B000E7C4828003C687016317C7009747FF1FE4
:1021C0002380D7C4828083C6870113075002631916
:1021D000D700930760021747FF1F2303F7C28280CF
:1021E00083C68701130660026315D6009307700249
:1021F000DDB783C7870155BF9747FF1F9387C7BECA
:10220000D44B0947638DE6081703FFFFE70223ED70
:102210001749FF1F130989BA3E8483470900918B30
:102220009DCFB7E4040083A7041D829783A7441CB5
:102230001745FF1F130505B9829783A7841C8146A4
:102240001746FF1F034606BA81450145829721C5FF
:1022500083470900ED9B1747FF1F2301F7B683470C
:10226000040093F7F70F85CB91471747FF1F2327EC
:10227000F7B897000000E78080EB97000000E78048
:1022800040EFB7E70400BC4F414691451745FF1F9B
:10229000034505B682971703FFFF670083E6828038
:1022A0001703FFFFE702A3E38D4741116306F5041F
:1022B000C5476308F50285476310F5029747FF1F7E
:1022C0002382A7B4B7E70400BC4B93050010174561
:1022D000FF1F0345E5B1829741011703FFFF670028
:1022E00043E285471747FF1F230EF7B0B7E7040007
:1022F000BC4B93050020E1BF9747FF1F9387C7AEF4
:10230000D44B1147638DE600B7E7040083A7071D90
:102310008297B7E70400BC4B930500044DBF054905
:102320001747FF1F232C27AD83C7070032C62E8413
:1023300093F7F70FD5D3B7E4040083A7041D7D14EA
:102340001374F40F8297E37689FCB245994703C66C
:102350001500E3F0C7FCFC4409061745FF1F1305F1
:10236000A5AA8297BC48930500081745FF1F03459F
:1023700025A8829779BF1703FFFFE70243D61747C7
:10238000FF1F130767A64047184B1C409746FF1FC7
:1023900023A2F6A66316E4001747FF1F232EF7A417
:1023A000130584FE9790FFFFE78060A6035564FF46
:1023B0009780FFFFE780E06E97A0FFFFE78060D087
:1023C0001703FFFF6700E3D31703FFFFE70223D1E3
:1023D0009747FF1F938747A1D84BDC4789C79700D2
:1023E0000000E78080F985471747FF1F2328F7A0E3
:1023F0009747FF1F9387C7909C439305000217459B
:10240000FF1F0345E59E83C787031747FF1F230967
:10241000F79EB7E70400BC4B82971703FFFF6700E6
:1024200043CE9747FF1F23A3A79C82801703FFFF7C
:10243000E70243C937E404007C4CA1451745FF1F60
:102440000345059B82977C48A1451745FF1F03451F
:10245000259A9744FF1F938424998297DC4489EB43
:1024600097000000E78080D91703FFFF6700C3C80B
:1024700003D567FF9780FFFFE780A062AA896DD12F
:10248000D84891476310F7027C4C91451745FF1FD0
:102490000345059682977C4891451745FF1F0345E4
:1024A0002595829703A9490103D409018947B7E912
:1024B00004001747FF1F2323F79483A7091D210456
:1024C0004204829783C784011715FF1F1305050671
:1024D00061191717FF1FA30BF70483A7491C41803D
:1024E00082979747FF1F238F079083A7C91C8146B8
:1024F00009469375F40F4A85829711E99747FF1FA4
:1025000083C787A089C79700FF1FE780A06EB7E742
:102510000400BC4F2146A1451745FF1F0345458DCB
:10252000829799B71703FFFFE70263BB93F7052074
:1025300001112E8481CF97000000E78020E9134528
:10254000042005611703FFFF6700A3BB93F7051085
:10255000A9CF9744FF1F93842489DC48970000008B
:10256000E78020C11737FF1F13078779184383C7F8
:102570008401034787036318F700DC4489C7970089
:102580000000E78080DF85471747FF1F2328F78675
:10259000B7E70400BC4B930500021745FF1F034536
:1025A000258582971345041069BF93F70508BDC7B9
:1025B0009747FF1F83C75785E91719469745FF1FA0
:1025C0009385A5841305D10093F4F70F1749FF1FD6
:1025D0000349898397C00000E78040409397040136
:1025E000C1831747FF1F1307A782231DF100231C78
:1025F000F1009737FF1F9387277F3ACE3ACAD84317
:102600002306010009CBDC439315890154080D46CC
:10261000E185680082971345040825B793F72500E4
:10262000A5C39737FF1F9387277CD84B894763063D
:10263000F7029737FF1F83C7677813F7270011EF5B
:10264000918B99CFB7E70400BC4F1306000A894568
:102650001735FF1F0345C579829713452400D5B56B
:102660009737FF1F9387C7699C4383C78703173733
:10267000FF1F2307F77897000000E78060DBF1BFBA
:1026800093F7050281CB97000000E78060DA1345DD
:10269000040245BD93F7850081CB97000000E780D9
:1026A000E0D21345840071BD93F7150081CB9700EC
:1026B0000000E780A0B41345140061B593F745000E
:1026C00081CB97000000E78060B31345440095BDBF
:1026D00093F7050495C39737FF1F83C7E77091CB26
:1026E00097000000E780A0A491471737FF1F23271A
:1026F000F77013450404B1B593F705010145E38272
:1027000007E49737FF1F9387276ED84B91476310D5
:10271000F7049737FF1F9387676A9C4313D72700F7
:102720008583D98F858B91E7B7E7040083A7071DC1
:102730008297B7E70400FC4F91451735FF1F03450B
:10274000256B829785471737FF1F2329F76A1345A3
:102750000401C5BB9737FF1F2388A77A8280170320
:10276000FFFFE702C3979737FF1F23A50768973737
:10277000FF1F23A3076885471734FF1F130444581E
:102780001737FF1F232CF7661C4083C787031737B3
:10279000FF1F2307F7669790FFFFE780A08F29C5EB
:1027A0009717FF1F23A8A7D81C4017050000130583
:1027B000A5D783C787031737FF1F2303F7641717AE
:1027C000FF1FA305F7D69737FF1FA38F0760B7E753
:1027D000040083A7070882979737FF1F238AA76003
:1027E0001703FFFF6700E391B7C7898E938767EDF3
:1027F0001717FF1F2320F7D445BF1737FF1F0347C5
:10280000A75E795555E79737FF1F9387E75D03C7A5
:10281000170005079736FF1FA388E65C03C717005C
:102820008D463377D7029736FF1FA38FE65A83C6AC
:1028300017001737FF1F1307A74C184393F6F60F1F
:10284000A9EE834787031737FF1F230BF75A8547E6
:102850001737FF1F230AF7589737FF1F938707562D
:102860009C430145998BA9E71703FFFFE7022387E4
:1028700037E404007C48C1451735FF1F0345455721
:1028800082973C4885451735FF1F0345655682975B
:1028900001451703FFFF6700C38683C717008546FE
:1028A0006395F6008347970379BF8347A70361BF0A
:1028B00082809737FF1F83C72753A1CF1703FFFFDE
:1028C000E702E38137E404009737FF1F238E0750A8
:1028D0007C4885451735FF1F0345855182977C4C01
:1028E00091451735FF1F0345A55082977C489145B8
:1028F0001735FF1F0345C54F82973C48C145173523
:10290000FF1F0345E54E8297014517F3FEFF670061
:10291000437F7955828017F3FEFFE702437C2A84C8
:10292000035565FF9780FFFFE780A0179737FF1FCC
:102930009387874BD847BE841DEF9790FFFFE780B2
:1029400080779C48232004009DEB9737FF1F23A529
:10295000874A9737FF1F23AF8748B7E70400BC4B70
:1029600089451735FF1F0345A5488297014517F391
:10297000FEFF67000379630A8700184375BF80C3B1
:102980009737FF1F23AA8746C9BF7955CDB717F3DD
:10299000FEFFE702C3749737FF1F938727578843CB
:1029A0002326050023240500510597A00000E78099
:1029B000C03317F3FEFF6700C37417F3FEFFE7028F
:1029C00003721734FF1F130464541C40411199CF44
:1029D0009C472302B5002AC61CC197000000E7806F
:1029E00040FB1C409C4B99C332458297410117F331
:1029F000FEFF6700037117F3FEFFE702436E41110C
:102A0000444D328532842EC69790FFFFE780C05236
:102A10002AC422859790FFFFE780205403A8440032
:102A2000630C0800B245835744001840224683D502
:102A30004500AA8626850298410117F3FEFF67002C
:102A4000436C17F3FEFFE7028369404D1DC808C0C1
:102A500097050000938565031305440197A00000C6
:102A6000E78040169737FF1F9387474A9C430145ED
:102A700089E79737FF1F23AB874817F3FEFF6700EF
:102A800043687D55DDBF17F3FEFFE7024365011183
:102A900068009305F00F02C602C802CA02CC02CE3B
:102AA00097000000E780A0F1056117F3FEFF6700C3
:102AB00043659737FF1F938767459C43D847A167B6
:102AC0009D076319F70217F3FEFFE7024361011147
:102AD00032859790FFFFE7802046230AA1008145B9
:102AE000680097000000E78080ED056117F3FEFFA6
:102AF0006700236182809737FF1F938727419C439C
:102B0000D847A167938777036319F70217F3FEFF8E
:102B1000E702E35C011132859790FFFFE780C04137
:102B2000230AA1008145680097000000E78020E9A2
:102B3000056117F3FEFF6700C35C82809737FF1FB4
:102B40009387C73C9C43D84795476316F70417F310
:102B5000FEFFE702C3580111328532849790FFFFD0
:102B6000E780803D230AA10022859790FFFFE78040
:102B7000C03E83574400231BA10081453ECC1C402E
:102B800068003ECE97000000E78060E3056117F320
:102B9000FEFF670003578280930785FF8DC383275D
:102BA000C5FF91CFDC4B81CF17F3FEFFE702235324
:102BB000032585FF829717F3FEFF67008354828009
:102BC00017F3FEFFE702A3512A8432859790FFFF97
:102BD000E7808036BD4763EBA70018449377F50084
:102BE0000345B70041995D8DA305A70017F3FEFFCC
:102BF0006700235117F3FEFFE702634E01117C00CB
